:100000000C94B71A0C94E81A0C94E81A0C94E81A99
:100010000C94E81A0C94E81A0C94E81A0C94E81A58
:100020000C94E81A0C94E81A0C94E81A0C94E81A48
:100030000C94E81A0C94E81A0C94E81A0C94E81A38
:100040000C94E81A0C948BD10C94E81A0C94E81ACE
:100050000C94E81A0C94E81A0C9488BE0C9428AA04
:100060000C94E81A0C9457560C944D560C94E81ABC
:100070000C94E81A0C94E81A0C94E81A0C94E81AF8
:100080000C943D340C94E81A0C94E81A0C94E81A79
:100090000C94E81A0C94E81A0C94E81A0C94E81AD8
:1000A0000C94E81A0C94E81A0C940F340C94E81A87
:1000B0000C94E81A0C94E81A0C94E81A0C94E81AB8
:1000C0000C94E81A0C94E81A0C94E81A0C944B3728
:1000D0000C9415370C94E81A0C94E81A0C94E81A4E
:1000E0000C94E81A084AD73B3BCE016E84BCBFFD96
:1000F000C12F3D6C74319ABD56833DDA3D00C77FF8
:1001000011BED9E4BB4C3E916BAAAABE0000008090
:100110003F05A84CCDB2D44EB93836A9020C50B91F
:10012000918688083CA6AAAA2ABE000000803F004B
:100130000C9406FD0C94B8370C949AA40C94974236
:100140000C9405FC0C9421FC0C94A7FC0C94FCA8CA
:100150000C9409FC0C9495560C941DFC0D942101F3
:100160000C941B570C9401570D94540F0C94F0FBF6
:100170000C94F5370D94850B0D942E140C94F956B0
:100180000C94ED560C94F1370C942FFC0D944C010B
:100190000D94691F0C9479FC0C946CFC0D949410D4
:1001A0000C9425FC0C943BA90C94FCFC0C942BFCAB
:1001B0000D945A0C0D94AE0B0C94D3560C94C4565B
:1001C0000D947D0F0D94E50B0C9444420C94FFFBB1
:1001D0000C949FFC0C94FEA70C940FFC0D946D0CDA
:1001E0000C94D6370D94F90B0D9481090C94DEFC18
:1001F0000C94C5FC0C94F4FB0C948DFC0D94C8037A
:100200000D9449050C947EA80C941DA50D94EC0743
:100210000C94FCFB0C940DFF0C94DEFB0D94510A26
:100220000C94CC440D9465090C940EA90D944E0FBA
:100230000C94ED370C94F5560D9437000C94D9FBC3
:100240000C9407380C94C7370D94871F0C94E9372A
:100250000C9463A80C9493420D94C20B0C94044527
:100260000C94FC370D94B7020D94B5090C9405AAB3
:100270000C94FD560C941CA50C94E5370D949B0F23
:100280000C941FA80C94E2560C9489370D94170B0C
:100290000C9497FC0D9432090C94D4FC0C94F156F8
:1002A0000C94E9560C945F440C9413FC0C94B1FC30
:1002B0000C9474FC0D94180C0C948B440C940F3813
:1002C0000C94E8FC0D94E10A0D94570F0C9469A767
:1002D0000C94F2FC0C9413570C94BBFC0C94085730
:1002E0000D94870F0D9484100C9486A70D941D0D0A
:1002F0000D94A80F0D946F0F0D9457110D94270FA7
:100300000C94E1370C9417FC0C94DD370C9483FCAF
:100310000C94F8FB4E414E494E495459494E46CD36
:10032000CCCC3D0AD7233C17B7D13877CC2B3295AC
:1003300095E6241FB14F0A000020410000C842008A
:10034000401C4620BCBE4CCA1B0E5AAEC59D740054
:10035000407A10F35A00A0724E18090010A5D4E894
:100360000000E87648170000E40B54020000CA9A27
:100370003B000000E1F50500008096980000004079
:10038000420F000000A086010000001027000000BE
:1003900000E803000000006400000000000A000004
:1003A0000000000100000000002C76D888DC674FB8
:1003B0000823DFC1DFAE59E1B1B796E5E3E453C6E8
:1003C0003AE651997696E8E6C28426EB898C9B62E0
:1003D000ED407C6FFCEFBC9C9F40F2BAA56FA5F48A
:1003E00090055A2AF75C936B6CF9676DC11BFCE0B2
:1003F000E40D47FEF520E6B500D0ED902E03009405
:100400003577050080841E080000204E0A00000099
:10041000C80C333333330F986E12831141EF8D21A3
:1004200014893BE65516CFFEE6DB18D1844B381B0A
:10043000F77C1D901DA4BBE424203284725E2281CF
:1004400000C9F124ECA1E53D27434F4D4D554E49E0
:10045000434154494F4E0044525952554E00455263
:10046000524F525300494E464F004543484F0045B6
:1004700072726F722077726974696E6720746F2070
:10048000454550524F4D210A0053544F505045445A
:100490002E20005072696E7465722073746F7070D4
:1004A00065642064756520746F206572726F727365
:1004B0002E2046697820746865206572726F7220FC
:1004C000616E6420757365204D39393920746F2051
:1004D000726573746172742E202854656D70657234
:1004E00061747572652069732072657365742E205E
:1004F0005365742069742061667465722072657337
:1005000074617274696E67290A004E6F20436865D2
:10051000636B73756D2077697468206C696E6520F4
:100520006E756D6265722C204C617374204C696E1F
:10053000653A20004E6F20436865636B73756D20CC
:1005400077697468206C696E65206E756D6265727E
:100550002C204C617374204C696E653A20006368EE
:1005600065636B73756D206D69736D617463682C61
:10057000204C617374204C696E653A20004C696EA2
:1005800065204E756D626572206973206E6F7420F0
:100590004C617374204C696E65204E756D62657296
:1005A0002B312C204C617374204C696E653A20000D
:1005B0004D3131300053657269616C207374617420
:1005C0007573206D69736D617463680A0077616982
:1005D000740A0053442072656164206572726F7200
:1005E0000A002121204B494C4C20636175736564DE
:1005F00020627920746F6F206D75636820696E6169
:1006000063746976652074696D65202D2063757249
:1006100072656E7420636F6D6D616E643A20004880
:100620006F74656E642049646C652054696D656FF4
:10063000757400486F74656E642049646C6520545D
:10064000696D656F75740A003D3D6F6E46696C613A
:100650006D656E7452756E6F75743D3D0070617599
:100660007365004D363030002066696C616D656ED3
:10067000745F72756E6F7574200066696C616D656C
:100680006E745F72756E6F757420540046696C618C
:100690006D656E7452756E6F75742054002A2A2A27
:1006A000496E6974696E67206361726420697320A2
:1006B0004F4B2A2A2A004D6564696120496E736593
:1006C00072746564004D656469612052656D6F7672
:1006D0006564004D313030305300627573793A20D3
:1006E00070617573656420666F7220696E707574D1
:1006F0000A00627573793A207061757365642066CB
:100700006F7220757365720A00627573793A207092
:10071000726F63657373696E670A002A2A2A6B69B0
:100720006C6C2A2A2A00706F7765726F6666004BC0
:10073000494C4C45442E20005072696E74657220FD
:1007400068616C7465642E206B696C6C2829206369
:10075000616C6C6564210A0053544F505045442E1F
:1007600020005072696E7465722073746F707065CA
:10077000642064756520746F206572726F72732EC9
:100780002046697820746865206572726F722061F6
:100790006E6420757365204D39393920746F20726D
:1007A0006573746172742E202854656D7065726172
:1007B000747572652069732072657365742E205399
:1007C0006574206974206166746572207265737443
:1007D000617274696E67290A006563686F3A004543
:1007E00072726F723A0042696C696E656172204C78
:1007F0006576656C696E6720477269643A0A002104
:10080000212053544F502063616C6C6564206265F5
:100810006361757365206F6620424C546F75636821
:10082000206572726F72202D20726573746172740C
:100830002077697468204D3939390A002121205305
:10084000544F502063616C6C656420626563617510
:100850007365206F6620424C546F75636820657223
:10086000726F72202D2072657374617274207769C3
:100870007468204D3939390A002F2F616374696F0C
:100880006E3A0070726F6D70745F00656E64005335
:10089000656E64204D31303820746F207265737539
:1008A0006D650A00496E736572742066696C616DCE
:1008B000656E7420616E642073656E64204D313006
:1008C000380A005265686561742066696E697368EC
:1008D00065642E0052656865617420446F6E650022
:1008E000526568656174696E672E2E2E00526568C8
:1008F000656174004865617465722054696D656F47
:1009000075740053656E64204D31303820746F204B
:1009100068656174206E6F7A7A6C650A004E6F7A32
:100920007A6C65205061726B656400486F74656E07
:100930006420746F6F20636F6C640A00706175735C
:1009400065640050617573650044697361626C652C
:1009500052756E6F75740050757267654D6F726574
:10096000005061757365640073686F770062757419
:10097000746F6E00626567696E004C6F616420463B
:10098000696C616D656E74004C6F61642046696CC2
:10099000616D656E74205400496E736572742066D3
:1009A000696C616D656E7420616E642073656E6440
:1009B000204D3130380A00726573756D65640052E0
:1009C0006573756D696E670057616974696E67203C
:1009D000666F72206865617475702E0A004C6561DF
:1009E00076696E6720473236003F537065636966EB
:1009F00069656420582C5920636F6F7264696E6159
:100A00007465206F7574206F6620626F756E6473F5
:100A10002E0A003F28522965706561742076616C4A
:100A20007565206E6F7420706C61757369626C659A
:100A30003B206D757374206265206174206C656164
:100A4000737420312E0A003F285229657065617445
:100A5000206D7573742062652073706563696669C3
:100A60006564207768656E206E6F74207573696E9B
:100A70006720616E204C43442E0A003F537065632B
:100A80006966696564206E6F7A7A6C652074656D3D
:100A90007065726174757265206E6F7420706C6120
:100AA000757369626C652E0A003F537065636966F1
:100AB0006965642066696C616D656E742073697A1E
:100AC00065206E6F7420706C61757369626C652E41
:100AD0000A003F53706563696669656420707269D6
:100AE0006D65206C656E677468206E6F7420706C25
:100AF00061757369626C652E0A003F5072696D659D
:100B0000206C656E677468206D7573742062652053
:100B1000737065636966696564207768656E206EC9
:100B20006F74207573696E6720616E204C43442E8C
:100B30000A003F537065636966696564206E6F7A69
:100B40007A6C652073697A65206E6F7420706C61B1
:100B5000757369626C652E0A003F52657472616339
:100B600074696F6E204D756C7469706C6965722064
:100B70006D7573742062652073706563696669655D
:100B8000642E0A003F53706563696669656420528C
:100B9000657472616374696F6E204D756C746970F1
:100BA0006C696572206E6F7420706C617573696218
:100BB0006C652E0A003F5370656369666965642041
:100BC0006C6179657220686569676874206E6F74FE
:100BD00020706C61757369626C652E0A0043292E62
:100BE0000A003F53706563696669656420626564E5
:100BF0002074656D7065726174757265206E6F74B6
:100C000020706C61757369626C65202834302D002A
:100C1000473236207374617274696E672E2E2E0A05
:100C2000004F46460A00466164652048656967686A
:100C3000742000426564204C6576656C696E67209F
:100C4000004661696C656420746F20656E61626C3A
:100C50006520426564204C6576656C696E670A00A4
:100C6000496E76616C6964206D6573682E0A005068
:100C7000726F62696E6720506F696E740025532031
:100C800025692F2569002E0A002F0050726F6269B6
:100C90006E67206D65736820706F696E7420002028
:100CA0002844525952554E29004732392041757413
:100CB0006F20426564204C6576656C696E67003F05
:100CC00020284C2C522C462C4229206F7574206F02
:100CD0006620626F756E64732E0A003F2856296580
:100CE00072626F7365206C6576656C20696D706CDF
:100CF00061757369626C652028302D34292E0A00D5
:100D0000426164205A2076616C75650A004E6F203E
:100D100062696C696E65617220677269640A004479
:100D20006576696174696F6E0025533A20257300FA
:100D300046696E6973686564210A003A207A3A2030
:100D400000206F662000476F696E6720746F3A203D
:100D5000580043570A00206469723A0020616E67A8
:100D60006C653A00537461727420726164697573C2
:100D70003A004D343820506F696E740025533A2084
:100D800025642F256400506F736974696F6E696EF6
:100D900067207468652070726F62652E2E2E0A00BF
:100DA0003F4C656773206F66206D6F76656D656E6D
:100DB0007420696D706C61757369626C6520283090
:100DC0002D3135292E0A003F2028582C5929206F13
:100DD0007574206F6620626F756E64732E0A005002
:100DE000726F6265206F7574206F6620626F756E1A
:100DF0006473003F53616D706C652073697A652080
:100E00006E6F7420706C61757369626C6520283434
:100E10002D3530292E0A004D3438205A2D50726F4E
:100E20006265205265706561746162696C6974798C
:100E300020546573740A003F2856296572626F73E7
:100E400065206C6576656C20696D706C6175736981
:100E5000626C652028302D34292E0A005374616E8F
:100E60006461726420446576696174696F6E3A20CA
:100E7000002052616E67653A2000204D61783A206B
:100E800000204D696E3A2000205369676D613A2059
:100E9000004D65616E3A20005741524E494E472140
:100EA000204C6F77205A204A65726B206D61792043
:100EB0006C65616420746F20756E77616E74656413
:100EC000207061757365732E0A004F4646004F4EC1
:100ED0000020204D61783A2000200020204D696ECE
:100EE0003A2000536F667420656E6473746F70737C
:100EF0003A20003D3D4F6E506F7765724C6F7373B3
:100F0000526573756D653D3D004D32342053256C3F
:100F1000642054256C64004739322E3920452573EE
:100F200000473120462564004739322E39205A25A2
:100F300073004731205A302046323030004731208C
:100F400058257320592573204633303030004D34F6
:100F5000323020532569205A2573004D3130362018
:100F600050256920532569004D32303020442573C7
:100F70000047323852305859004739322E3920450F
:100F800030205A300A47315A2573004D313039200C
:100F9000532569004D31393020532569004D3432D5
:100FA00030205330205A300020496E76616C6964DD
:100FB000206578747275646572200047322F47335C
:100FC0002062616420706172616D65746572730A7C
:100FD00000536C6565702E2E2E005A2050726F6281
:100FE000652050617374204265640A005A20507273
:100FF0006F62652050617374204265640047323827
:101000004C30004D3131372050726F62652066617F
:10101000696C65642E0A4732380A0070726F626527
:101020005F72657769706500473239205265747266
:1010300079696E670050726F62696E6720466169F8
:101040006C6564004D31313720426564206C6576F3
:10105000656C696E67206661696C65642E0A47304D
:10106000205A31300A4D3330302050323520533839
:1010700038300A4D333030205035302053300A4D4F
:101080003330302050323520533838300A4D333029
:1010900030205035302053300A4D3330302050321C
:1010A0003520533838300A4D333030205035302019
:1010B00053300A47342053310070726F62655F66A7
:1010C00061696C6564004D31313720426564206C84
:1010D0006576656C696E6720646F6E652E00205AB8
:1010E0003A200020593A200042656420583A2000F6
:1010F0004D65736820706F696E74206F7574206F12
:10110000662072616E67650A004D302053746F70FF
:10111000004D312053746F7000436F6E74696E75AB
:101120006500436C69636B20746F20526573756D45
:10113000652E2E2E004E6F204D6F76652E00456E6B
:10114000642066696C65206C6973740A0042656787
:10115000696E2066696C65206C6973740A004E6F55
:10116000206D656469610A00526573756D696E670B
:1011700020534400286E6F2066696C652900437512
:101180007272656E742066696C653A2000507269EF
:101190006E742074696D653A20000A53746174732B
:1011A0003A2046696C616D656E7420757365643AAA
:1011B00020002C204C6F6E67657374206A6F623A52
:1011C0002000546F74616C2074696D653A2000537F
:1011D000746174733A20002C204661696C65643A2E
:1011E00020002C2046696E69736865643A200050BF
:1011F00072696E74733A200053746174733A2000FC
:10120000436F6F6C696E672E2E2E0048656174699E
:101210006E672E2E2E0045202553006F6B006F66E3
:1012200066006A0465045E04570449044445425557
:10123000473A004D31313320530042656420436FFB
:101240006F6C696E672E2E2E0042656420486561C2
:1012500074696E672E2E2E0044445820313053504E
:10126000726F5632204F46462E002F2F002052001C
:10127000416363656C65726174696F6E3A205000FA
:101280004D32303620580046523A0020466C6F7777
:101290003A20003A200020536572766F2000206FBC
:1012A0007574206F662072616E67650A00536572FF
:1012B000766F200020643A0020693A0020703A00DE
:1012C000496E76616C6964206578747275646572C4
:1012D0000A0020643A0020693A0020703A006469EC
:1012E0007300656E0043290A0061626C6564202802
:1012F0006D696E2074656D702000436F6C642065AD
:101300007874727564657320617265200050494479
:10131000204175746F74756E6500504944204175A5
:10132000746F74756E65206661696C656421204216
:101330006164206865617465722069640A004669A9
:101340006C616D656E742072756E6F757420646962
:101350007374616E636520286D6D293A20004669BB
:101360006C616D656E742072756E6F757420004DC2
:1013700034323120696E636F7272656374207061FC
:1013800072616D657465722075736167650A004DE1
:1013900065736820706F696E74206F7574206F6656
:1013A0002072616E67650A004F666673657473200C
:1013B0004170706C696564004572723A20546F6FB9
:1013C000206661722100546F6F2066617220667220
:1013D0006F6D207265666572656E636520706F69FA
:1013E0006E740A00454550524F4D204F4B0A005035
:1013F0006F7765722D6C6F7373207265636F76659E
:10140000727920004D383400446F6E652070726927
:101410006E74696E672066696C650A004D37370027
:101420004D3331004361703A004D454154504143C2
:101430004B00434F4F4C45525F54454D5045524130
:1014400054555245004348414D4245525F54454D25
:10145000504552415455524500424142595354451A
:101460005050494E470041524353004D4F54494F4D
:101470004E5F4D4F44455300544845524D414C5FDB
:1014800050524F54454354494F4E004C4F4E475FC6
:1014900046494C454E414D45004155544F524550EB
:1014A0004F52545F53445F53544154555300534477
:1014B0005F575249544500524550454154005344EA
:1014C000434152440050524F4D50545F5355505079
:1014D0004F525400454D455247454E43595F504188
:1014E0005253455200434153455F4C494748545F6E
:1014F0004252494748544E45535300544F47474C76
:10150000455F4C494748545300534F465457415246
:10151000455F504F574552004255494C445F504536
:101520005243454E54004C4556454C494E475F4446
:10153000415441005A5F50524F42450052554E4F60
:101540005554004155544F4C4556454C0050524956
:101550004E545F4A4F420050524F4752455353003A
:101560004155544F5245504F52545F54454D5000D1
:10157000564F4C554D455452494300454550524FE6
:101580004D0042494E4152595F46494C455F5452C5
:10159000414E534645520053455249414C5F584FC6
:1015A0004E5F584F4646004649524D574152455F9F
:1015B0004E414D453A4D61726C696E20322E302E8F
:1015C000375F4457372E3320426F6E64746563680B
:1015D0002053534D4442422028417072203239201A
:1015E000323032312031313A32363A3335292053D4
:1015F0004F555243455F434F44455F55524C3A68FF
:10160000747470733A2F2F6769746875622E636FF4
:101610006D2F496E73616E6974794175746F6D6178
:1016200074696F6E2F4D61726C696E2F747265658F
:101630002F437265616C6974794477696E5F322EED
:10164000302050524F544F434F4C5F5645525349F0
:101650004F4E3A312E30204D414348494E455F545C
:101660005950453A4444582031305350726F5632E5
:101670002045585452554445525F434F554E543AB5
:101680003120555549443A63656465326132662DAF
:10169000343161322D343734382D396231322D6393
:1016A00035356336326633363766660A0050726FF8
:1016B0006265204F6666736574205A0050726F62CF
:1016C00065204F6666736574205A00290A002074ED
:1016D0006F20003F5A206F7574206F662072616E14
:1016E0006765202800290A0020746F20003F5920D8
:1016F0006F7574206F662072616E676520282D00FB
:10170000290A0020746F20003F58206F7574206FE5
:10171000662072616E676520282D0050726F6265C9
:10172000204F666673657420580043616E6E6F7457
:10173000206F70656E207375626469722000256980
:10174000730025696D202569730025696820256966
:101750006D20256973002569642025696820256945
:101760006D20256973002569792025696420256924
:10177000682025696D20256973003D3D4477696EB9
:1017800020496E697420436F6D706C6574653D3DD2
:10179000002A2A2A4E6F7A7A6C6554656D705374EC
:1017A000617475735B325D203D003D3D4865617439
:1017B000696E6720446F6E65204368616E676520BF
:1017C00046696C616D656E743D3D002020737461E7
:1017D000727470726F677265737320003D3D77613C
:1017E000697477617920353D3D003D3D77616974CD
:1017F00077617920343D3D003D3D776169747761C3
:101800007920333D3D003D3D7761697477617920F2
:10181000313D3D003D3D6F6E5072696E7454696D8F
:10182000657253746F707065643D3D003D3D6F6E31
:10183000466163746F727952657365743D3D00272C
:101840000A0A0000272027002027002D006E6F7451
:10185000696669636174696F6E200063616E6365B8
:101860006C005072696E742041626F72746564001E
:101870004469736D6973730055492041626F7274D6
:10188000656400726573756D65004D3234002A2AF7
:101890002A43506C617920546F6E652A2A2A003DD4
:1018A0003D6F6E5072696E7454696D6572506175EA
:1018B0007365643D3D00486F6D696E6720466169E0
:1018C0006C6564006F70656E00545249474745521D
:1018D0004544003A200066696C616D656E74007A5B
:1018E0005F6D696E00795F6D696E00785F6D696E1E
:1018F000005265706F7274696E6720656E647374F0
:101900006F70207374617475730A0020746F6F2098
:101910006C6F6E6720657874727573696F6E207076
:10192000726576656E7465640A0020636F6C64206E
:10193000657874727573696F6E2070726576656E06
:101940007465640A00486F6D6520257325732573DF
:10195000204669727374005761726E696E673A202F
:10196000486F6D696E672042756D702044697669B5
:10197000736F72203C20310A000202040000000054
:10198000000000000000000000809D4300009B4319
:101990000000C8430000004100000041000000407A
:1019A000FFFFFF0000000100000001000080005563
:1019B0005555000000400033333300AAAA2A0049DD
:1019C00092240000002000C7711C0099991900D1D1
:1019D000451700555515003BB1130024491200115D
:1019E000111100000010000F0F0F00E3380E00432C
:1019F000790D00CCCC0C00C3300C00E8A20B0064C5
:101A0000210B00AAAA0A00703D0A009DD8090042D5
:101A10007B090092240900DCD308008888080010A4
:101A200042080000000800F0C10700878707007522
:101A3000500700711C07003EEB0600A1BC060069C0
:101A400090060066660600703E06006118060017E4
:101A5000F4050074D105005BB00500B2900500628A
:101A60007205005555050078390500B81E050005BA
:101A70000505004EEC040087D40400A1BD040090CD
:101A8000A7040049920400C17D0400EE690400C768
:101A9000560400444404005C320400082104004160
:101AA000100400000004003FF00300F8E0030026EB
:101AB000D20300C3C30300CCB503003AA803000A55
:101AC0009B0300388E0300C08103009F750300D084
:101AD000690300505E03001D530300344803009166
:101AE0003D03003333030016290300381F0300971A
:101AF000150300300C0300030303000BFA02004936
:101B0000F10200BAE802005CE002002DD802002DCC
:101B1000D0020059C80200B0C0020031B90200DA98
:101B2000B10200AAAA0200A0A30200BC9C0200FA13
:101B30009502005C8F0200DF88020082820200456D
:101B40007C02002776020027700200436A02007CB4
:101B5000640200D05E02003F590200C8530200FF39
:101B6000FDFCFAF8F6F4F2F0EEECEAE9E7E5E3E181
:101B7000E0DEDCDAD9D7D5D4D2D0CFCDCBCAC8C736
:101B8000C5C3C2C0BFBDBCBAB9B7B6B4B3B2B0AFBB
:101B9000ADACAAA9A8A6A5A4A2A1A09E9D9C9A9915
:101BA000989795949392908F8E8D8B8A898887864B
:101BB00084838281807F7E7D7B7A79787776757465
:101BC000737271706F6E6D6C6B6A6968676665645D
:101BD000636261605F5E5D5C5B5A59585857565549
:101BE0005453525150504F4E4D4C4B4A4A4948471E
:101BF0004646454443424241403F3E3E3D3C3B3BDE
:101C00003A39383837363535343332323130302F8F
:101C10002E2E2D2C2B2B2A29292827272625252433
:101C2000232322212120201F1E1E1D1C1C1B1B1ACA
:101C30001919181817161615151413131212111155
:101C4000100F0F0E0E0D0D0C0C0B0A0A09090808D7
:101C50000707060605050404030302020100003D10
:101C60003D6F6E5072696E7454696D657253746124
:101C7000727465643D3D0000809D4300009B4300FD
:101C800000C8430000000000000000000000003D0C
:101C90003D6F6E53746F726553657474696E6773CC
:101CA0003D3D003D3D6F6E436F6E666967757261C5
:101CB00074696F6E53746F72655772697474656E70
:101CC0003D3D0053657474696E67732053746F7281
:101CD0006564000A20696E6974207A70726F6265AB
:101CE0005F7A6F6666736574203D20003D3D6F6EC0
:101CF000436F6E66696775726174696F6E53746F56
:101D00007265526561643D3D00454550524F4D201E
:101D1000496E697469616C697A65640A003B2000E8
:101D20003A0A0020204D3630332000204400202085
:101D30004D34313220530046696C616D656E7420FC
:101D400072756E6F75742073656E736F723A0020D2
:101D500055004C0046696C616D656E74206C6F6156
:101D6000642F756E6C6F6164206C656E6774687348
:101D70003A0020204D3835312058005A2D50726FCE
:101D80006265204F66667365740020204D343133E0
:101D9000205300506F7765722D4C6F73732052651E
:101DA000636F766572793A00204400204900202054
:101DB0004D33303420500020440020490020204D75
:101DC0003330312050005049442073657474696E7B
:101DD00067733A00204A00202047323920572049B3
:101DE0000020204D3432302053004175746F204262
:101DF0006564204C6576656C696E673A0020204DFD
:101E0000323036205800486F6D65206F6666736506
:101E1000743A0020580020530020204D32303520E5
:101E20004200416476616E6365643A20423C6D69AC
:101E30006E5F7365676D656E745F74696D655F7500
:101E4000733E20533C6D696E5F66656564726174B4
:101E5000653E20543C6D696E5F74726176656C5F9F
:101E600066656564726174653E20583C6D61785F9B
:101E7000785F6A65726B3E20593C6D61785F795F6F
:101E80006A65726B3E205A3C6D61785F7A5F6A6565
:101E9000726B3E20453C6D61785F655F6A65726B71
:101EA0003E0020540020520020204D32303420507B
:101EB00000416363656C65726174696F6E2028759B
:101EC0006E6974732F7332293A20503C7072696EB8
:101ED000745F616363656C3E20523C72657472612D
:101EE00063745F616363656C3E20543C7472617619
:101EF000656C5F616363656C3E0020204D3230315C
:101F00002058004D6178696D756D20416363656C83
:101F100065726174696F6E2028756E6974732F73B2
:101F200032293A0020204D3230332058004D61785C
:101F3000696D756D206665656472617465732028CE
:101F4000756E6974732F73293A005374657073202A
:101F500070657220756E69743A0020440020204D2F
:101F60003230302053002044697361626C65640A2A
:101F70000046696C616D656E742073657474696E7A
:101F800067733A0020286D6D2900202047323120E8
:101F90002020203B20556E69747320696E206D6D82
:101FA000003D3D6F6E4C6F616453657474696E677C
:101FB000733D3D000000FA430000FA430000204159
:101FC00000008C420000A0420000A0420000C84374
:101FD0000080CF43EE020000EE020000640000002B
:101FE0003C00000024F4D43050C38E20C2A240171D
:101FF000828B7011127A910D816CD90AA861E10867
:10200000C7586607615143061E4B5D05C145A704CD
:102010001A411104093D9803713931034036DB023E
:1020200065339102D4305402802E1D02632CEE01E0
:10203000752AC501B028A001102781018F256401F0
:102040002B244B01E0223401AC211F018D200D0116
:10205000801FFC00841EED00971DDF00B81CD2001D
:10206000E61BC600201BBC00641AB200B219A8000F
:102070000A19A0006A189900D117910040178B0027
:10208000B516840031167E00B31579003A15730039
:10209000C7146F0058146A00EE13660088136300BB
:1020A00025135E00C7125B006C1257001512540016
:1020B000C111510070114F0021114B00D610490081
:1020C0008D1047004610440002104200C00F40002F
:1020D000800F3E00420F3C00060F3B00CB0E380045
:1020E000930E37005C0E3500270E3400F30D3200DE
:1020F000C10D3100900D3000600D2E00320D2D000D
:10210000050D2C00D90C2B00AE0C2900850C2900E4
:102110005C0C2700350C27000E0C2600E80B240071
:10212000C40B2400A00B23007D0B23005A0B2100BD
:10213000390B2100180B2000F80A1F00D90A1E00D5
:10214000BB0A1E009D0A1D00800A1D00630A1C00B8
:10215000470A1B002C0A1B00110A1A00F7091A0073
:10216000DD091900C4091900AB091900920917000B
:102170007B091800630917004C0916003609160080
:10218000200916000A091500F5081500E0081400DA
:10219000CC081400B8081400A40814009008130018
:1021A0007D0812006B081300580812004608120040
:1021B0003408110023081100120811000108110051
:1021C000F0071000E0071000D0071000C007100053
:1021D000B0070F00A107100091070E0083070F0042
:1021E00074070F0065070E0057070E0049070E0021
:1021F0003B070D002E070E0020070D0013070D00F2
:1022000006070D00F9060C00ED060D00E0060C00B7
:10221000D4060C00C8060C00BC060C00B0060C006E
:10222000A4060B0099060C008D060B0082060B001D
:1022300077060B006C060B0061060A0057060B00C0
:102240004C060A0042060A0038060A002E060A005A
:1022500024060A001A060A001006090007060A00EA
:10226000FD050900F4050900EB050900E205090078
:10227000D9050900D0050900C7050900BE050900F8
:10228000B5050800AD050800A50509009C05080076
:10229000940508008C050800840508007C050800EA
:1022A000740508006C050700650508005D0507005A
:1022B000560508004E0507004705070040050800C1
:1022C00038050700310507002A0507002305070028
:1022D0001C050600160507000F0507000805060087
:1022E00002050700FB040600F5040700EE040600E3
:1022F000E8040600E2040700DB040600D50406003B
:10230000CF040600C9040600C3040600BD0406008D
:10231000B7040600B1040500AC040600A6040600DC
:10232000A00405009B040600950405009004060027
:102330008A04050085040500800406007A0405006F
:1023400075040500700405006B04050066040500B3
:10235000610405005C0405005704050052040500F3
:102360004D04050048040500430405003E04040034
:102370003A04050035040500300404002C0405006F
:1023800027040400230405001E0404001A040400AA
:1023900016040500110404000D04040009040500DE
:1023A0000404040000040400FC030400F803040017
:1023B000F4030400F0030400EC030400E803040049
:1023C000E4030400E0030400DC030400D803040079
:1023D000D4030400D0030400CC030400C8030300AA
:1023E000C503030024F404D9201BC40C5C0E98041C
:1023F000C4095F0265077101F405F900FB04B3002D
:1024000048048700C10369005803550003034500D1
:10241000BE023A008402310053022A00290225003C
:1024200004022000E4011C00C8011900AF011700DC
:102430009801140084011300710110006101100063
:1024400051010E0043010D0036010B002B010B0062
:1024500020010B00150109000C010900030108000F
:10246000FB000800F3000800EB000700E400060092
:10247000DE000600D8000600D2000600CC000500F1
:10248000C7000500C2000500BD000400B90004003B
:10249000B5000400B1000400AD000400A900040070
:1024A000A5000300A20003009F0004009B0003009E
:1024B00098000300950002009300030090000300C1
:1024C0008D0002008B0003008800020086000200DD
:1024D00084000300810002007F0002007D000200F2
:1024E0007B00020079000200770001007600020004
:1024F0007400020072000100710002006F0002000F
:102500006D0001006C0002006A0001006900020019
:102510006700010066000100650001006400020020
:102520006200010061000100600001005F00020024
:102530005D0001005C0001005B0001005A00010029
:102540005900010058000100570001005600010029
:102550005500010054000100530000005300010029
:102560005200010051000100500001004F00010025
:102570004E0000004E0001004D0001004C00010023
:102580004B0000004B0001004A000100490001001F
:10259000480000004800010047000100460000001C
:1025A0004600010045000000450001004400010014
:1025B000430000004300010042000000420001000F
:1025C0004100000041000100400001003F00000008
:1025D0003F0001003E0000003E0001003D00000001
:1025E0003D0001003C0000003C0000003C000100F8
:1025F0003B0000003B0001003A0000003A000100EF
:1026000039000000390001003800000038000000E7
:1026100038000100370000003700010036000000DC
:1026200036000000360001003500000035000000D3
:1026300035000100340000003400000034000100C7
:1026400033000000330000003300010032000000BE
:1026500032000000320001003100000031000000B3
:1026600031000100300000003000000030000100A7
:102670002F0000002F0000002F0000002F0001009D
:102680002E0000002E0000002E0001002D00000092
:102690002D0000002D0000002D0001002C00000086
:1026A0002C0000002C0000002C0001002B0000007A
:1026B0002B0000002B0000002B0001002A0000006E
:1026C0002A0000002A0000002A0001002900000062
:1026D0002900000029000000290000002900010055
:1026E000280000002800000028000000280000004A
:1026F000280001002700000027000000270000003C
:10270000270000002700010026000000260000002E
:102710002600000026000000260001002500000021
:102720002500000025000000250000002500000015
:102730002500010024000000240000002400000007
:1027400024000000240001002300000023000000FA
:1027500023000000230000002300000023000000ED
:1027600023000100220000002200000022000000DF
:1027700022000000220000002200010021000000D1
:1027800021000000210000002100000021000000C5
:1027900021000000210001002000000020000000B6
:1027A00020000000200000002000000020000000A9
:1027B00020000000200001001F0000001F0000009A
:1027C0001F0000001F0000001F0000001F0000008D
:1027D0001F0001001E0000001E0000001E0000007F
:1027E0001E0000003930000033250000871900006A
:1027F000B00F0000DB080000BD0400007402000000
:102800003F01000020436F756E7420583A00236426
:102810006566696E652044454641554C545F00002D
:10282000626564004B6420004B6920004B702000FF
:10283000504944204175746F74756E652066696EE9
:102840006973686564212050757420746865206C14
:10285000617374204B702C204B6920616E64204B97
:102860006420636F6E7374616E74732066726F6D33
:102870002062656C6F7720696E746F20436F6E669F
:10288000696775726174696F6E2E680A00504944F9
:10289000204175746F74756E65206661696C65643E
:1028A000212074696D656F75740A00504944204198
:1028B00075746F74756E65206661696C656421203E
:1028C00054656D706572617475726520746F6F20E8
:1028D000686967680A00204B643A2000204B693A17
:1028E0002000204B703A200020436C6173736963B1
:1028F00020504944200A00204E6F206F7665727385
:10290000686F6F740A002054753A2000204B753AA6
:102910002000206D61783A2000206D696E3A200019
:1029200020643A200020626961733A2000504944D3
:10293000204175746F74756E652073746172740ACA
:1029400000504944204175746F74756E652066614E
:10295000696C6564212054656D706572617475726F
:102960006520746F6F20686967680A0042656400BB
:10297000453100626564002C2073797374656D20A5
:1029800073746F7070656421204865617465725F4F
:1029900049443A200048656174696E672046616960
:1029A0006C65640048656174696E67206661696C76
:1029B0006564004D3131322053687574646F776EF1
:1029C000001000C90210012C014001220170011801
:1029D00001B0010E01F00104015002FA00B002F052
:1029E000003003E600D003DC009004D2007005C87C
:1029F00000A006BE000008B400B009AA00D00BA0D9
:102A000000600E960060118C00001582002019787D
:102A100000C01D6E00A0226400B0275A00902C5008
:102A20000000314600E0343C0010383200903A2873
:102A300000603C1E00A03D1400803E0A00203F00C4
:102A400000544845524D414C2052554E4157415932
:102A500000546865726D616C2052756E61776179A2
:102A6000004572723A204D415854454D50004D4139
:102A70005854454D502074726967676572656400EB
:102A80004572723A204D494E54454D50004D494EC5
:102A900054454D5020747269676765726564002003
:102AA0002F002042403A0020403A0020573A0020B0
:102AB000573A00496E76616C696420657874727566
:102AC0006465720A007C3C3E5E2B3D3F2F5B5D3BA4
:102AD0002C2A225C0043616E6E6F74206F70656EED
:102AE000207375626469722000534420496E6974D2
:102AF000204661696C0053442063617264206F6BEF
:102B00000A006F70656E526F6F74206661696C6544
:102B1000640A00766F6C756D652E696E6974206647
:102B200061696C65640A004E6F20534420636172D2
:102B3000640A000A4D3234004D3233202573002ED2
:102B40000A006F70656E206661696C65642C2046B2
:102B5000696C653A200046696C652073656C656335
:102B60007465640A002053697A653A200046696CEE
:102B700065206F70656E65643A2000454E442053B1
:102B80005542524F5554494E450A002220706F73EA
:102B9000002220706172656E743A220053554252D1
:102BA0004F5554494E452043414C4C207461726747
:102BB00065743A220053756263616C6C204F7665D0
:102BC00072666C6F77004578636565646564206D37
:102BD000617820535542524F5554494E4520646503
:102BE0007074683A002E0A0044656C6574696F6EF3
:102BF000206661696C65642C2046696C653A20002A
:102C000046696C652064656C657465643A0053447C
:102C1000207072696E74696E672062797465200035
:102C20004E6F74205344207072696E74696E670A27
:102C30000057726974696E6720746F2066696C65ED
:102C40003A2000667265736800646F696E670020E1
:102C500066696C653A20004E6F7720002F617574AD
:102C60006F25632E67002020506C616E6E65724286
:102C7000756666657242797465733A200020467203
:102C80006565204D656D6F72793A2000436F6D70F8
:102C9000696C65643A2041707220323920323032DA
:102CA000310A00204C61737420557064617465644E
:102CB0003A20323032312D30342D3138207C2041D1
:102CC0007574686F723A20426F6E64746563682031
:102CD0002F20496E73616E6974794175746F6D61EF
:102CE00074696F6E0A00322E302E375F4457372ECC
:102CF000330A004D61726C696E0020536F66747701
:102D00006172652052657365740A002057617463AF
:102D100068646F672052657365740A002042726FA1
:102D2000776E206F75742052657365740A002045B4
:102D3000787465726E616C2052657365740A005018
:102D40006F77657255700A0073746172740A004778
:102D500039310A47315A350A4739300A4D38340A71
:102D60004D31303453300A4D3134305330004D3111
:102D7000303031006572726F722077726974696EDB
:102D80006720746F2066696C650A00446F6E652069
:102D9000736176696E672066696C652E0A004D3234
:102DA0003900456E6473746F70730025532025637A
:102DB00020256320256320256300205A3A002059EE
:102DC0003A0020583A00656E6473746F707320681F
:102DD00069743A200070012C0190012701B0012292
:102DE00001C0011D01F00118011002130130020E93
:102DF000016002090190020401C002FF000003FA11
:102E0000004003F5008003F000D003EB002004E64F
:102E1000007004E100E004DC004005D700C005D2EA
:102E2000004006CD00D006C8008007C3003008BEB1
:102E300000F008B900C009B400B00AAF00B00BAA96
:102E400000D00CA500000EA000500F9B00C01096F3
:102E5000005012910000148C00C0158700B017823A
:102E600000B0197D00D01B7800001E730040206E5A
:102E70000090226900F024640040275F0090295AE6
:102E800000E02B5500102E500020304B0010324631
:102E900000E033410090353C001037370070383285
:102EA00000A0392D00B03A2800A03B2300603C1E52
:102EB00000103D1900903D1400103E0F00703E0AB6
:102EC00000C03E0500003F0000403FFBFF803FF692
:102ED000FFC03FF1FF00000A0B02090C0D0E0807AE
:102EE00003040100000000000000000000000000DA
:102EF00000000000000000000000000000000000D2
:102F0000001211100000000000000000000000008E
:102F1000000000000000000000000050726F6269B5
:102F20006E67204661696C656400205A3A20002073
:102F3000593A200042656420583A20003D3D6F6EAA
:102F400055736572436F6E6669726D52657175690E
:102F50007265643D3D00220A00556E6B6E6F776EA0
:102F600020636F6D6D616E643A2022002042002064
:102F700050006F6B00204500205A00205900204D62
:102F8000393220580020453A00205A3A0020593A58
:102F900000583A0020746F6F206C6F6E6720657860
:102FA00074727573696F6E2070726576656E746584
:102FB000640A0020636F6C642065787472757369AD
:102FC0006F6E2070726576656E7465640A00436189
:102FD0006E6E6F7420656E746572207375626469BD
:102FE000723A20004D323520500A4D32340052657D
:102FF00073756D65005549205061757365004E6F9E
:10300000204D61746368203A004D32320A4D3231EE
:1030100000526566726573680050675570005067AE
:10302000446F776E0049732046696C6520004973D0
:10303000204469722000476F5570446972004861EE
:1030400073204D656469610046696C656E616D65EC
:103050002053656C6563746564004D3130303043D6
:10306000004D313030300046696C616D656E742002
:10307000537461742030202D20330046696C616DDB
:10308000656E7420537461742030202D2032004608
:10309000696C616D656E7420537461742030202DED
:1030A0002031002046696C616D656E742052657335
:1030B000706F6E7365204E6F00526573756D65207D
:1030C00059657320647572696E67207072696E74D9
:1030D000000A204E6F2046696C616D656E74004970
:1030E0006E76616C6964204F7074696F6E004D3547
:1030F00030300053746F72652053657474696E6765
:1031000073004265642050494420537461727465B1
:1031100064004D3939390A4D323830503053313628
:103120003000424C546F75636820526573657400BB
:103130004D3530320A4D35303000496E69742045C6
:103140004550524F4D00486F74656E64205049449D
:10315000205374617274656400456E676C697368AE
:1031600020416C726561647920536574004368691D
:103170006E657365204E6F7420537570706F727436
:10318000656400496E4C616E6743686F69636500F2
:103190000A202A2A2A7265636461742E646174614C
:1031A0005B305D203D004732380A473120463130E0
:1031B0003030205A313000556E737570706F7274F4
:1031C0006564204F7074696F6E2053656C6563741D
:1031D00065640047323652323535004D313930534F
:1031E00035350A4732380A4732390A4D3430300A09
:1031F0004D313034533231350A4732380A4D31308F
:1032000039533231350A4D34323053310A4731584F
:103210003130305931303046353030300A47315A4C
:10322000300A4D3530300A4D313137205365742026
:103230005A204F666673657400473120463130303E
:1032400030205A302E30004732380A47312046317C
:10325000303030205A302E30004D353030005A207A
:103260004F6666736574203A202573004D35303003
:10327000005A204F6666736574203A202573004714
:1032800032380A473146313530305A302E30004717
:1032900032385A0A473146313530305A302E3000F4
:1032A0004D383400473146313030305A302E3000FE
:1032B0004732380A473146313030305A302E3000EC
:1032C0004D616E75616C53657454656D7000526527
:1032D00071756573746564204F666673657420420A
:1032E00065796F6E64204C696D697473005A204F64
:1032F0006666736574203A20257300526F756E649C
:10330000696E6720746F2073746570005265717503
:103310006573746564204F6666736574200053742A
:103320006F70205472696767657265640053746FCB
:1033300070204E6F0053746F705072696E74004845
:10334000616E646C6520446174612041646A7573C8
:103350007420322053657474696E672053637265FC
:10336000656E200048616E646C6520446174612064
:103370005072696E7446696C6520332053657474AD
:10338000696E672053637265656E200048616E64E4
:103390006C652044617461205072696E7446696C7A
:1033A0006520322053657474696E672053637265BB
:1033B000656E20004D38340048616E646C652044B1
:1033C000617461205072696E7446696C6520506F3B
:1033D00073740048616E646C6520446174612050B0
:1033E00072696E7446696C6520507265004265674B
:1033F000696E537769746368003D3D204368656377
:103400006B6B65793D3D007265636461742E616428
:103410006472203D3D007265636461742E64617462
:10342000615B305D203D3D00776169747761792093
:103430003D3D0020202A2A2A2A2A2A2A5254535F54
:1034400048616E646C65446174612A2A2A2A2A2ABA
:103450002A2A2000526573656E643A20000000221B
:1034600000250028002B002E00310034000201004E
:1034700000050108010B0100002100240027002A9B
:10348000002D003000330001010000040107010A93
:103490000105050505070508080808020202020AD9
:1034A0000A080804040404010101010101010103E7
:1034B00003030303030303040707070C0C0C0C0CA2
:1034C0000C0C0C0202020206060606060606060B95
:1034D0000B0B0B0B0B0B0B0102102020080810200C
:1034E0004010204080020102010804020101020490
:1034F000081020408080402010080402018004024F
:1035000001804020100804020108040201010204A5
:1035100008102040800102040810204080444458D4
:103520002031305350726F56322052656164792ECB
:10353000005072696E74696E672E2E2E005072698B
:103540006E7420506175736564006E6F746966698E
:10355000636174696F6E20005049442054756E6534
:103560002046696E6973686564002401C8001124EF
:103570001FBECFEFD1E2DEBFCDBF00E00CBF14E035
:10358000A0E0B2E0E4EFF0E602E00BBF02C007907B
:103590000D92A230B107D9F726E1A2E0B4E001C054
:1035A0001D92AE32B207E1F71AE1C6EBDAE100E0B4
:1035B00006C021970109802FFE010F94A72CC53B5F
:1035C000D10780E00807A9F70F941E1A0D94683000
:1035D0000C9400009F92AF92BF92CF92DF92EF9235
:1035E000FF920F931F93CF93DF9300D01F921F92F0
:1035F000CDB7DEB7EFE5FBE10027BB27462F572FFE
:10360000A82FAA2341F4A52F542FB85FAA2319F499
:10361000A52F5527B85FA03138F45295A295452FB4
:103620004F70507FA42BBC5FA03428F4550FAA1F05
:10363000550FAA1FBE5FA03818F4550FAA1FB395E7
:10364000550FAA1FEA0FF01F449151E0AA27B85066
:1036500081F1C8F0B0FF02C0440F551FB1FF04C094
:10366000440F551F440F551FB2FF06C05295429597
:10367000142F1F70407F512BB3FF1BC0A52F542F59
:1036800044270C94591BB195B0FF02C0559547953E
:10369000B1FF04C05595479555954795B2FF05C0B4
:1036A0005295407F4295452B5F70B3FF02C0452F76
:1036B0005527DD24CC24BB24B2E0649FD018C10878
:1036C000B00AB00B749FC018B108B00B849FB0183B
:1036D000B109659FC018B108B00B759FB018B1094A
:1036E000859FB0196A9FB018B1097A9FB0194D9D96
:1036F000A12C99243327992722275D9DA00C911C8A
:10370000301F901F201FAD9D900C311D901F201F5A
:103710004C9DA00C911C301F901F201F5C9D900C95
:10372000311D901F201FAC9D300D911D201F4B9D02
:10373000900C311D901F201F5B9D300D911D201F8F
:10374000AB9D900D211D4B9F300D911D201F5B9F48
:10375000900D211DAB9F200DB1E0BB24CC24DD24B6
:10376000639FD018C108B00AB00B739FC018B1088E
:10377000B00B839FB018B109699FC018B108B00B96
:10378000799FB018B109899FB019629FB018B1092B
:10379000729FB019D61AC70AB80A20F0B1E03B0FE1
:1037A000901F201F1124792F632F90E0822F0F90FC
:1037B0000F900F900F900F90DF91CF911F910F916D
:1037C000FF90EF90DF90CF90BF90AF909F900895C3
:1037D000AF92BF92CF92DF92EF92FF920F931F931F
:1037E000CF93DF93C8E3DCE00BEE18E088E4A82E6B
:1037F0008CE0B82EC12CD12C7601C39469917991BB
:10380000899199910F94E525288939894A895B899D
:103810000F9446260F94232EF801619371938193A0
:1038200091938F01C616D706E806F90610F46B01CE
:103830007C01AC16BD0611F76FEF7FEFCB01A7013E
:1038400096010F94242C2093FB083093FC0840939E
:10385000FD085093FE08DF91CF911F910F91FF90CB
:10386000EF90DF90CF90BF90AF900895CF92DF920E
:10387000EF92FF928091F707882309F457C0C09018
:10388000F307D090F407E090F507F090F60720E0FA
:1038900030E0A901C701B6010F94E025882309F49F
:1038A00045C020E030E040E05FE3C701B6010F947F
:1038B00046269B01AC010F9446262BED3FE049E4E0
:1038C00050E40F9446269B01AC0160E070E080E874
:1038D0009FE30F94AA2D6B017C01C092800CD092C3
:1038E000810CE092820CF092830C609165027091E1
:1038F0006602072E000C880B990B0F94E7252AE02F
:1039000037ED43E25CE30F944626A70196010F943E
:1039100046266093610270936202809363029093E3
:103920006402FF90EF90DF90CF900895C12CD12CCE
:1039300080E8E82E8FE3F82ED0CF0F931F93CF931C
:10394000DF9350E0FC01E40FF51F8081440F551F09
:10395000440F551F43565A4FEA01882329F18881A5
:103960009981AA81BB81EB01088119812A813B8160
:103970000097A105B10569F40C591F4F2F4F3F4F18
:10398000DA010D931D932D933C9313978FEF808352
:1039900006C0081B190B2A0B3B0B37FDF7CFDF9135
:1039A000CF911F910F910895188219821A821B825C
:1039B000F6CFCF93DF9324E0829FC0011124EC0166
:1039C000C253D74FFC01EC5FF74F8850984FDC0192
:1039D0002D913D914D915C916081718182819381A6
:1039E0000F94B02C688379838A839B83DF91CF9176
:1039F00008958091980590919905A0919A05B091AC
:103A00009B058093410290934202A0934302B0939E
:103A10004402809196059091970590936802809357
:103A2000670208958091410290914202A091430261
:103A3000B09144028093980590939905A0939A05BC
:103A4000B0939B05809167029091680290939705CF
:103A50008093960584E690E09093680280936702D5
:103A600008958091881290918912891B877089F43A
:103A70008091900D81110DC08091840C9091850CE6
:103A8000892B39F481E09091A606911103C080E062
:103A9000089581E00895CF93DF93DB01F9019C91B4
:103AA0009130C1F0943080F094509C938830D1F4E0
:103AB00080819181009771F0019791838083480FF5
:103AC000591FEA01188206C08C3539F49C5F9C931B
:103AD000943041F4DF91CF9108958B3339F781E031
:103AE0008C93F8CF20813181B9016F5F7F4F718353
:103AF0006083420F531FEA018883808191818F3553
:103B000091056CF7E7CF0F931F9381E000912C1480
:103B100010912D1420912E1430912F1440912814BF
:103B20005091291460912A1470912B1404171507D1
:103B30002607370708F480E01F910F91089590E061
:103B400080E00895282F9091F207833021F495FDAD
:103B50000FC094FD0FC0892F90E0B0E0A0E004C03A
:103B6000B695A795979587952A95D2F78170089570
:103B700081E0089580E00895FC016591759185913B
:103B8000949108958F929F92AF92BF92CF92DF92BD
:103B9000EF92FF92CF93DF93EC018090CA08909050
:103BA000CB08A090CC08B090CD0820E030E0A9016F
:103BB000C501B4010F94E025882309F454C0C880DE
:103BC000D980EA80FB80A7019601C501B4010F945A
:103BD000E02518160CF04CC02091C2083091C308A3
:103BE0004091C4085091C508C701B6010F94E02563
:103BF000882331F1C092C208D092C308E092C40871
:103C0000F092C5082091C6083091C7084091C808B5
:103C10005091C908688179818A819B810F944626D9
:103C20009B01AC0160E070E080E89FE30F94AF2C53
:103C300060930F027093100280931102909312020E
:103C400060910F0270911002809111029091120206
:103C5000DF91CF91FF90EF90DF90CF90BF90AF902A
:103C60009F908F90089560E070E080E89FE3F0CF30
:103C700060E070E0CB01ECCFCF92DF92EF92FF9249
:103C8000CF93DF93EC01CC80DD80EE80FF8027E1D5
:103C900037EB41ED58EBC701B6010F94102F87FDAC
:103CA00023C023E030E04BE953E4C701B6010F9491
:103CB000E0251816CCF0C880D980EA80FB8027E187
:103CC00037EB41ED58EBC701B6010F94102F87FD7C
:103CD0000BC0C1E023E030E84DE953E4C701B60171
:103CE0000F94E02518160CF4C0E08C2FDF91CF91D3
:103CF000FF90EF90DF90CF9008952FEB280F2A319F
:103D000008F047C0E22FF0E080913505909136052C
:103D1000A0913705B091380504C0B695A795979541
:103D200087952A95D2F780FD02C081700895E95EDB
:103D3000FA4FE081EE2341F180918407909185074D
:103D4000E80FF92FF11D808190ED980F9A3030F037
:103D50008E3251F4818180538A3098F4F0930605B5
:103D6000E093050581E008958D3211F08B3249F41E
:103D7000818190ED980F9A3088F38E3211F4828110
:103D8000EACFF0E0E0E0EACF1092060510920505D8
:103D9000E9CF80E008950E947D1E882341F081E0F4
:103DA0002091050530910605232B09F480E0089544
:103DB0008F929F92AF92BF92CF92DF92EF92FF923B
:103DC000C090D405D090D505E090D605F090D705E9
:103DD00020E030E0A901C701B6010F94E025882357
:103DE000E1F1A701960160E070E080E89FE30F94A5
:103DF000AA2D6B017C018090D8059090D905A090E8
:103E0000DA05B090DB0520E030E0A901C501B4017E
:103E10000F94E025882329F1A501940160E070E06A
:103E200080E89FE30F94AA2DC092DE04D092DF04B5
:103E3000E092E004F092E1046093E2047093E30402
:103E40008093E4049093E504FF90EF90DF90CF908F
:103E5000BF90AF909F908F900895C12CD12C760188
:103E6000CACF60E070E0CB01DFCF129A08955F9A6D
:103E70008091360C8E7F8093360C8A9A8091360C16
:103E80008D7F8093360C809108018095817080939E
:103E900006018091360C8B7F8093360C0C94351F75
:103EA000269A2E9A08958C3221E0920714F08CE223
:103EB00091E09093ED118093EC110C944AFDE0E1B8
:103EC000F6E0108211821282138214820C944AFD51
:103ED0004F925F926F927F928F929F92AF92BF921A
:103EE000CF92DF92EF92FF920F931F93CF93DF93C6
:103EF000EC012091CC053091CD054091CE0550913B
:103F0000CF05688179818A819B810F94AF2C6B01E9
:103F10007C012091D0053091D1054091D20550917E
:103F2000D3056C817D818E819F810F94AF2C4B01D5
:103F30005C01A701960160910302709104028091D7
:103F40000502909106020F94E025882309F450C0E1
:103F5000C0920302D0920402E0920502F09206029F
:103F60002091DE043091DF044091E0045091E1049F
:103F7000C701B6010F9446262B013C010F94522E27
:103F80006B017C0120E030E0A9010F94E02587FD62
:103F900070C020E030E040E450E4C701B6010F9467
:103FA000102F18162CF4C12CD12CC0E4EC2EFE2CB2
:103FB000A7019601C301B2010F94AF2C6093D60400
:103FC0007093D7048093D8049093D904C701B601A5
:103FD0000F941C2E6093D404062E000C770B6F5F99
:103FE0007F4F6430710514F064E070E06093D20498
:103FF000D09101021091D404A501940160910702AF
:10400000709108028091090290910A020F94E025B4
:10401000811133C0D11381C02091BA043091BB0407
:104020004091BC045091BD046091D6047091D704B6
:104030008091D8049091D9040F9446262091BE0413
:104040003091BF044091C0045091C1040F94B02C32
:10405000DF91CF911F910F91FF90EF90DF90CF9064
:10406000BF90AF909F908F907F906F905F904F9098
:104070000895C12CD12C76019BCF8092070290929B
:104080000802A0920902B0920A022091E204309143
:10409000E3044091E4045091E504C501B4010F9498
:1040A00046264B015C010F94522E6B017C0120E0EF
:1040B00030E0A9010F94E02587FDF3C020E030E057
:1040C00040E450E4C701B6010F94102F18162CF4E9
:1040D000C12CD12CB0E4EB2EFE2CA7019601C5011A
:1040E000B4010F94AF2C6093DA047093DB048093D7
:1040F000DC049093DD04C701B6010F941C2E60937D
:10410000D504062E000C770B6F5F7F4F643071056E
:1041100014F064E070E06093D304C091D504D1132F
:1041200005C0809102028C1709F470C08091D404FC
:104130009091D50490930202809301020C2E000C02
:10414000DD0B25E01203C0011124FC01EC0FFD1F63
:10415000EE0FFF1FEE0FFF1FE257F84F2081318156
:10416000428153812093CE043093CF044093D004F6
:104170005093D1040091D304002E000C110BFC01CC
:10418000E00FF11FEE0FFF1FEE0FFF1FE257F84F7A
:1041900060817181828193810F94AF2C6093CA04F6
:1041A0007093CB048093CC049093CD042091D204DF
:1041B00035E02303F0011124CE0FDF1FCC0FDD1FEC
:1041C000CC0FDD1FC257D84F288139814A815B81CE
:1041D0002093C6043093C7044093C8045093C90485
:1041E000E00FF11FEE0FFF1FEE0FFF1FE257F84F1A
:1041F00060817181828193810F94AF2C6093C2049E
:104200007093C3048093C4049093C5048090DA042F
:104210009090DB04A090DC04B090DD042091CA04EF
:104220003091CB044091CC045091CD04C501B40130
:104230000F9446262091CE043091CF044091D004B3
:104240005091D1040F94B02C6B017C01C092BE043C
:10425000D092BF04E092C004F092C1042091C20445
:104260003091C3044091C4045091C504C501B40108
:104270000F9446262091C6043091C7044091C8048B
:104280005091C9040F94B02CA70196010F94AF2C44
:104290006093BA047093BB048093BC049093BD04F4
:1042A000BBCEC12CD12C760118CFCF92DF92EF92EA
:1042B000FF92CF93DF93EC0108960E94C21D6B0121
:1042C0007C0120E030E0A9010F94E02520E030E0FF
:1042D000A901882359F0CE010E94681F9B01AC01FF
:1042E000C701B6010F9446269B01AC01688579850C
:1042F0008A859B850F94AF2C688779878A879B87EF
:10430000DF91CF91FF90EF90DF90CF9008952F92A3
:104310003F924F925F926F927F928F929F92AF9255
:10432000BF92CF92DF92EF92FF920F931F93CF93A2
:10433000DF93D62FC72FFC0180809180A280B380AD
:10434000C501B40120E831E541E050E00F94242C90
:10435000C9016DE671E00F94932C6B017C01C501DE
:10436000B40120E13EE040E050E00F94242CCA016B
:10437000B90128E130E040E050E00F94242C362EC3
:10438000272E062F172F8CE3482E512C612C712CD1
:10439000C501B401A30192010F94242CB62EA72EBF
:1043A000CA01B901A30192010F94242CCB01C114BD
:1043B000D10479F1AF92BF927F936F932F923F9286
:1043C000FF92EF92DF92CF9286E697E19F938F93D1
:1043D000CF93DF930F9477258DB79EB70E960FB6C8
:1043E000F8949EBF0FBE8DBF8D2F9C2FDF91CF9174
:1043F0001F910F91FF90EF90DF90CF90BF90AF9003
:104400009F908F907F906F905F904F903F902F90F4
:104410000895E114F104C9F0AF92BF927F936F93B6
:104420002F923F92FF92EF9286E597E19F938F93B1
:10443000CF93DF930F947725EDB7FEB73C960FB679
:10444000F894FEBF0FBEEDBFCFCF012BB9F0AF92F6
:10445000BF927F936F932F923F928AE497E19F934D
:104460008F93CF93DF930F9477258DB79EB70A96DE
:104470000FB6F8949EBF0FBE8DBFB6CF892BA9F0A3
:10448000AF92BF927F936F9382E497E19F938F9354
:10449000CF93DF930F947725EDB7FEB738960FB61D
:1044A000F894FEBF0FBEEDBF9FCFAF92BF928EE3D9
:1044B00097E19F938F93CF93DF930F9477250F907E
:1044C0000F900F900F900F900F908ECFEF92FF9262
:1044D0000F931F93CF93DF93CDB7DEB78C01EDB66B
:1044E000FEB60F942D2501962DB73EB7281B390B2C
:1044F0000FB6F8943EBF0FBE2DBF8DB79EB7019685
:10450000B8010F9426250E946DF90FB6F894FEBEEF
:104510000FBEEDBEDF91CF911F910F91FF90EF90F5
:1045200008958C38910514F08CE890E090938211F6
:10453000809381110C94C0BEAB01BC0140932C143C
:1045400050932D1460932E1470932F1484E995E1E9
:104550000C9478AF2F923F924F925F926F927F921E
:104560008F929F92AF92BF92CF92DF92EF92FF9283
:104570000F931F93CF93DF93CDB7DEB760970FB63E
:10458000F894DEBF0FBECDBF8B876C87042F122F30
:10459000282F30E03E872D87462F50E05A874987E5
:1045A00085E0982E929EC001939E900D1124988BC9
:1045B0008F87FA01E80FF91FEE0FFF1FEE0FFF1FA5
:1045C000E257F84F60817181828193819B01AC0138
:1045D0000F94A22F882309F445C14B85400F6C85A9
:1045E000610F949EC0011124E985FA85E80FF91F37
:1045F000EE0FFF1FEE0FFF1FE257F84FC080D18074
:10460000E280F380040F909EA0011124E985FA85D1
:10461000E40FF51FEE0FFF1FEE0FFF1FE257F84FDD
:104620000081918082807380262F30E0EF85F889A9
:10463000E20FF31FEE0FFF1FEE0FFF1FE257F84FC1
:1046400020807181798372817A8373817B83610F8A
:1046500070E0EF85F889E60FF71FEE0FFF1FEE0FF2
:10466000FF1FE257F84FF88BEF87F081FC83EF854F
:10467000F889F181FD83EF85F889F281FE83EF856A
:10468000F889F381FF83FC01E20FF31FEE0FFF1F98
:10469000EE0FFF1FE257F84F20812887A180B280DC
:1046A0006380FA01E60FF71FEE0FFF1FEE0FFF1FEB
:1046B000E257F84F4080518032801381202F392DEE
:1046C000482D572D602F792D882D972D0F94A22FCF
:1046D000882321F000E0912C812C712C9601A701F8
:1046E000B601C7010F94A22F882321F0C02ED92C28
:1046F000E82CF72C2C813D814E815F816C817D817E
:104700008E819F810F94A22F882321F01C821D820D
:104710001E821F82222D39814A815B81622D79811F
:104720008A819B810F94A22F882339F02C803D81B0
:1047300039834E814A835F815B839201432D512FE0
:10474000B201832D912F0F94A22F882321F0412CA9
:10475000512C312C10E028853A2D4B2D562D688593
:104760007A2D8B2D962D0F94A22F882321F0488629
:10477000A52CB32C612E85E02D853E85829FF0010E
:10478000839FF00D112449855A85E40FF51FEE0F24
:10479000FF1FEE0FFF1FE257F84FFA87E9879601D8
:1047A000A701B601C7010F94B02C202F392D482D39
:1047B000572D0F94AF2C6B017C01222D39814A813A
:1047C0005B81622D79818A819B810F94B02C2C8131
:1047D0003D814E815F810F94AF2C9B01AC01C701DD
:1047E000B6010F94B02C6B017C0128853A2D4B2D1E
:1047F000562D68857A2D8B2D962D0F94B02C920115
:10480000432D512F0F94AF2C9B01AC01C701B60172
:104810000F94B02C20E030E040E450E40F94AA2D37
:10482000E985FA8560837183828393836C858B85A8
:1048300060960FB6F894DEBF0FBECDBFDF91CF916B
:104840001F910F91FF90EF90DF90CF90BF90AF90AE
:104850009F908F907F906F905F904F903F902F90A0
:104860000C9400F860960FB6F894DEBF0FBECDBF73
:10487000DF91CF911F910F91FF90EF90DF90CF903C
:10488000BF90AF909F908F907F906F905F904F9070
:104890003F902F900895809105059091060500970F
:1048A00031F04AE050E070E060E00D94FB2360E0FE
:1048B00070E0CB0108958091050590910605009761
:1048C00031F04AE050E070E060E00D94CD2260E00D
:1048D00070E0CB010895CF93DF93EB010E94CB1ED4
:1048E000882319F00E945B24EB01CE01DF91CF9168
:1048F00008950E945B2497FD0CC00E945B246F3FCB
:1049000071058105910509F034F40E945B24862F1E
:10491000089580E008958FEF0895CF93C62F0E94E9
:10492000CB1E882319F0CF910C9479248C2FCF9132
:1049300008958091050590910605892B41F00E940C
:10494000792491E0811101C090E0892F089591E0D0
:10495000FCCFCF93DF93C82FD62F0E94CB1E882386
:1049600021F0DF91CF910C9499248C2F0E947D1E11
:10497000811101C08D2FDF91CF9108950E945B249A
:10498000CB010895CF93DF93EB010E94CB1E8823C8
:1049900021F0DF91CF910C94BE24CE01DF91CF9115
:1049A00008950F931F93CF9380910505909106056D
:1049B0000097E9F0FC018F01C1912C2F2F7D81F030
:1049C000C53411F0C536B9F7F801108270E060E027
:1049D0000F946F21F801C083CF911F910F9108951B
:1049E00070E060E0CF911F910F910D946F2160E016
:1049F00070E0CB01F1CFCF92DF92EF92FF926A018C
:104A00007B010E94CB1E882331F0FF90EF90DF9056
:104A1000CF900C94D124C701B601FF90EF90DF90A6
:104A2000CF9008954F925F926F927F928F929F9254
:104A3000AF92BF92CF92DF92EF92FF921F93CF93EC
:104A4000DF9300D01F92CDB7DEB719821A821B8286
:104A50001C82CE0101964C0182E7C82E87E0D82E39
:104A600096E2E92E9CE0F92E2EECA22E28E0B22E42
:104A700010E088E5810F0E94CB1EF40181934F0165
:104A8000882309F4E0C00E94D1242B013C01812F2E
:104A90000E94A21D882309F4CCC0F7012081318136
:104AA00042815381C301B2010F94B02CF60160839F
:104AB0007183828393831F5FF4E0CF0ED11C84E067
:104AC000E80EF11C94E0A90EB11C133091F685E4B8
:104AD0000E94CB1E8C83882309F4C0C00E94D1247D
:104AE0006B017C0183E00E94A21D882371F020915C
:104AF000320C3091330C4091340C5091350CC7017D
:104B0000B6010F94B02C6B017C01C0927E07D0924D
:104B10007F07E0928007F09281078091CB05882380
:104B200059F18091301482FF27C08C81882321F1B4
:104B30008981811103C08A818823F1F02DEC3CEC3E
:104B40004CE45DE36091190870911A0880911B088C
:104B500090911C080F94B02C9B01AC0160912E0C1D
:104B600070912F0C8091300C9091310C0F94102F7C
:104B7000181614F40E9446F740E050E0BA0186E4AB
:104B80000E94FB2420E030E0A9010F94102F18169A
:104B900084F40E94D12420E030E040E752E40F94F6
:104BA000AA2D609341027093420280934302909336
:104BB00044028091E40B83FD28C0809191068823F4
:104BC00021F12091320C3091330C4091340C5091F2
:104BD000350C60917E0770917F07809180079091DE
:104BE00081070F94AF2C20919E0630919F06409133
:104BF000A0065091A1060F94B02C60939E0670936E
:104C00009F068093A0069093A1060F900F900F909F
:104C10000F90DF91CF911F91FF90EF90DF90CF9099
:104C2000BF90AF909F908F907F906F905F904F90CC
:104C30000895F5012081318142815381C301B20180
:104C40000F94AF2C33CFF70180819181A281B38182
:104C5000F60180839183A283B3832DCF8091320CA0
:104C60009091330CA091340CB091350C80937E0759
:104C700090937F07A0938007B09381074ECFCF9288
:104C8000DF92EF92FF926B017C0183E3C816D1049F
:104C9000E104F10470F082E3C81AD108E108F108D8
:104CA00062E370E080E090E00E940BFD0E943AC257
:104CB000ECCFC701B6010E940BFDFF90EF90DF9093
:104CC000CF900C943AC2CF92DF92EF92FF920F9363
:104CD0001F93CF93DF936B017A01EC01C656DB4F34
:104CE00028813CE0389F8001399F100D112427FF57
:104CF00024C0FB011182108288818F5F88838881A4
:104D00009801280F311D87FD3A95C9012091731232
:104D1000F6012817190629F024F088818C300CF44C
:104D20003CC080819181049680349C4908F475C010
:104D3000F60180819181049672C088819801280FC4
:104D4000311D87FD3A95C901209173122817190664
:104D500099F294F28881A801480F511D87FD5A9558
:104D6000FA01EE0FFF1FE40FF51FE55DFD4E808198
:104D700087FFC2CF8881F801E80FF11D87FDFA9502
:104D8000CF01EE0FFF1FE80FF91FE55DFD4E80819B
:104D900060E08F770E94A9FBAFCF8081918128814D
:104DA000A801420F511D27FD5A959A01FA01EE0FF5
:104DB000FF1FE20FF31FE55DFD4E21813281820F5F
:104DC000931FF7019183808388819801280F311DFB
:104DD00087FD3A95F901EE0FFF1FE20FF31FE55D26
:104DE000FD4E808187FF20C08881080F111D87FD3F
:104DF0001A95F801EE0FFF1FE00FF11FE55DFD4E64
:104E0000808161E08F77DF91CF911F910F91FF90AB
:104E1000EF90DF90CF900C94A9FB80E49CE9F70120
:104E2000918380838FEF8883DF91CF911F910F91C2
:104E3000FF90EF90DF90CF9008950F931F93CF9343
:104E4000DF930CE41CE0C5E6D1E1F801219131913A
:104E5000419151918F0160E070E080E89FE30F94F1
:104E6000AA2D6993799389939993F1E1C537DF0767
:104E700061F70E9485F5DF91CF911F910F910C94FE
:104E8000E81BCF92DF92EF92FF92CF93DF932091B6
:104E9000370C222329F1EC0108960E94C21D6B01F8
:104EA0007C0120E030E0A9010F94E02520E030E013
:104EB000A901882359F0CE010E94681F9B01AC0113
:104EC000C701B6010F9446269B01AC016885798520
:104ED0008A859B850F94B02C688779878A879B8702
:104EE000DF91CF91FF90EF90DF90CF9008952F92B8
:104EF0003F924F925F926F927F928F929F92AF926A
:104F0000BF92CF92DF92EF92FF920F931F93CF93B6
:104F1000DF93CDB7DEB76C970FB6F894DEBF0FBE48
:104F2000CDBF8C015B015A834983FC01EA5BFF4FD3
:104F3000208131814281538129873A874B875C8761
:104F4000CA01B9010F94E5256B017C01D5012D91B2
:104F50003D914D915C910F9446260F948E2D2B011F
:104F60003C01E981FA812081318142815381C7016D
:104F7000B6010F9446260F948E2D4B015C01C301A0
:104F8000B2010F94232E698B7A8B8B8B9C8B6837A5
:104F900071058105910540F428E730E040E050E0DC
:104FA000298B3A8B4B8B5C8BC501B4010F94232E5C
:104FB0006D877E878F87988B68377105810591058E
:104FC00040F448E750E060E070E04D875E876F870F
:104FD000788BF801EE5AFF4F4080518062807380D9
:104FE000C301B2010F94E72569837A838B839C8385
:104FF00069897A898B899C890F94E5256D8B7E8BD5
:105000008F8B988F20E030E0A90169817A818B81B4
:105010009C810F94E025882309F4E1C1A701960142
:10502000C701B6010F9446264B015C012D893E89CC
:105030004F89588DCA01B9010F9446269B01AC01D6
:10504000C501B4010F94AF2C4B015C0129813A8159
:105050004B815C81CA01B9010F94B02C9B01AC015A
:10506000C501B4010F94AA2D0F948E2D0F94232EF9
:105070006D837E838F83988766277727CB0164199A
:105080007509860997090F94E7254B015C016D8529
:105090007E858F8598890F94E5252B013C0120E0C2
:1050A00030E0A901C501B4010F94E025882309F47B
:1050B0009AC1A3019201C301B2010F944626698FE0
:1050C0007A8F8B8F9C8FA7019601C701B6010F9431
:1050D00046269B01AC01698D7A8D8B8D9C8D0F943A
:1050E000AF2C6B017C01A5019401C501B4010F94A3
:1050F000B02C9B01AC01C701B6010F94AA2D0F94EF
:10510000522ED80195968D909D90AD90BC90989719
:10511000750164012D813E814F815885C21AD30AE1
:10512000E40AF50A0F94232EC61AD70AE80AF90AE8
:10513000F7FE8EC02D893E894F89588DCA01B9016D
:105140000F9446266B017C0129813A814B815C8159
:10515000CA01B9010F94B02C69877A878B879C8725
:1051600020E030E0A90169817A818B819C810F94D4
:10517000E025882309F43BC1C501B4010F94E5255E
:1051800029853A854B855C850F944626A7019601B3
:105190000F94AF2C6D837E838F839887A301920138
:1051A000C301B2010F9446269B01AC016D817E8143
:1051B0008F8198850F94B02C2B013C0120E030E0CA
:1051C00040E850E469817A818B819C810F94462666
:1051D0009B01AC01C301B2010F94AA2D0F948E2D37
:1051E0002B013C0120E030E0A9010F94102F18168C
:1051F0001CF0412C512C3201C301B2010F94232E1B
:105200006D837E838F83988786169706A806B906D6
:1052100020F48D829E82AF82B8866D817E818F81DF
:1052200098850F94E52529853A854B855C850F94F3
:105230004626A70196010F94B02C0F945E2F0F9471
:10524000232E69877A878B879C87C12CD12C760186
:1052500069857A858B859C8529893A894B895C8902
:10526000621B730B840B950B0F94E52529813A8102
:105270004B815C810F94AA2D20E034E244EF59E485
:105280000F9446260F94232E4B015C0169857A8585
:105290008B859C852D853E854F855889621B730BB8
:1052A000840B950B0F94E52529813A814B815C8114
:1052B0000F94AA2D20E034E244EF59E40F944626DF
:1052C0000F94232E2B013C013FE683169104A10489
:1052D000B10408F090C0F401EE0FFF1FEE0FFF1FA6
:1052E000ED55F64E85919591A591B4918983292E1E
:1052F0003A2EBD8B4FE6441651046104710408F048
:1053000083C0F201EE0FFF1FEE0FFF1FED55F64EAB
:1053100045915591659174919A01CB014D815E81C2
:105320006F817885D80199964D935D936D937C93A9
:105330009C974C0D5D1D6E1D7F1DF80145A756A75E
:1053400067A770ABE65BFF4F49895A896B897C89F7
:105350004083518362837383D5968D929D92AD92E3
:10536000BC92D897F80141AE52AE63AE74AEFD96D2
:1053700049814083218232825D8953833496208320
:1053800031838283938369857A858B859C85D196C9
:105390006D937D938D939C93D4973D962D853E85FB
:1053A0004F85588920833183428353836C960FB68F
:1053B000F894DEBF0FBECDBFDF91CF911F910F914B
:1053C000FF90EF90DF90CF90BF90AF909F908F9025
:1053D0007F906F905F904F903F902F90089560E086
:1053E00070E0CB0141CE60E070E0CB0188CE60E0A0
:1053F00070E0CB01F3CEC501B4010E94EA1A6983C3
:10540000272E382E9D8B76CFC301B2010E94EA1A57
:105410009B0184CF8091881290918912891B87709B
:1054200019F490E080E0089590918512992351F04D
:10543000833030F48FEF890F19F080938512F1CF0C
:1054400010928512809189122CE5829FC00111244F
:105450008C5F964FFC01208120FDE3CF20918912C3
:105460002F5F277020938612309189122091871226
:10547000321304C0209186122093871208959091D0
:105480006F0081E091FD02C080E0089590916F006F
:105490009D7F90936F00089580FF04C090919C05BC
:1054A00090FD8E7F81FF05C090919C05969590FDA3
:1054B0008D7F82FF06C090919C059695969590FDF4
:1054C0008B7F08958F929F92AF92BF92CF92DF927F
:1054D000EF92FF92CF93DF9320914502222309F4AC
:1054E0009EC0EC0180919C05C82ED12CF12CE12CA2
:1054F00080FF2CC08090470290904802A090490203
:10550000B0904A02288139814A815B81C501B4018A
:105510000F94102F181624F488829982AA82BB82D5
:105520008090530290905402A0905502B090560281
:10553000288139814A815B81C501B4010F94E0253E
:1055400087FF04C088829982AA82BB82D701C601E4
:10555000B695A7959795879580FF2CC080904B02B4
:1055600090904C02A0904D02B0904E022C813D8153
:105570004E815F81C501B4010F94102F181624F4D9
:105580008C829D82AE82BF8280905702909058029A
:10559000A0905902B0905A022C813D814E815F81CA
:1055A000C501B4010F94E02587FF04C08C829D8261
:1055B000AE82BF8282E0F694E794D794C7948A952E
:1055C000D1F7C0FE2CC0C0904F02D0905002E090A6
:1055D0005102F0905202288539854A855B85C701C2
:1055E000B6010F94102F181624F4C886D986EA86BF
:1055F000FB86C0905B02D0905C02E0905D02F09070
:105600005E02288539854A855B85C701B6010F94FE
:10561000E02587FF04C0C886D986EA86FB86DF912D
:10562000CF91FF90EF90DF90CF90BF90AF909F9081
:105630008F900895CF92DF92EF92FF920F931F9376
:10564000C12CD12C76018C0122E33CE04EE25CE0DF
:105650006AE27CE086E29CE00E9481F41F910F9157
:10566000FF90EF90DF90CF9008950C9485F5809196
:10567000A306811105C080918207882309F463C0C5
:1056800080918905659B59C08160809389059091BF
:1056900003018091890591FF52C082608093890542
:1056A000809189054A9B4DC08460809389058091D3
:1056B000F00580FF10C08091A40680FF0CC080918F
:1056C000890580FF08C08091E60681608093E60628
:1056D00080E00E949AC68091F005869580FF11C0F7
:1056E0008091A406869580FF0CC08091890581FF7A
:1056F00008C08091E60682608093E60681E00E9401
:105700009AC68091F0058695869580FF1CC0809191
:10571000A4068695869580FF16C08091820788230F
:1057200091F08091890582FF0EC08091E606846029
:105730008093E60682E00C949AC68E7FA6CF8D7F7A
:10574000ADCF8B7FB2CF08958091A306811104C0A5
:1057500080918207882331F062E070E080E090E081
:105760000C943F2608950F931F938091231181304D
:1057700019F50E943EFD0091A5051091A605209106
:10578000A7053091A805601B710B820B930B28EEC7
:1057900033E040E050E00F94242C6091A905709113
:1057A000AA058091AB059091AC05620F731F841F11
:1057B000951F1F910F9108956091AD057091AE05F1
:1057C0008091AF059091B005D6CF10922311109221
:1057D000A5051092A6051092A7051092A805109293
:1057E000AD051092AE051092AF051092B005109263
:1057F000A9051092AA051092AB051092AC05089568
:10580000CF92DF92EF92FF92CF93DF93C62FFC01EE
:10581000C080D180E280F38020E030E0A901C701A0
:10582000B6010F94E02520E030E0A90187FD14C007
:1058300020E030E048EC52E4C701B6010F94102F8D
:1058400024E630E040E050E0181634F0C701B6011D
:105850000F941C2E9B01AC01C230A0F4D0E0C150CB
:10586000D74FAFEFB0E00F94652C24E630E040E076
:1058700050E00F94462C2F3F310519F010F02FEF18
:1058800030E02883DF91CF91FF90EF90DF90CF90B1
:1058900008958091090180FD06C08091301483FB3A
:1058A000882780F9089580E00895CF92DF92EF92E3
:1058B000FF92FC01C080D180E280F380663019F550
:1058C00010921506109216061092170610921806DE
:1058D000109219060E94C0BE20E030E0A901C70165
:1058E000B6010F94E02587FF1DC0C12CD12C760195
:1058F000C701B6010F941D2FCB01FF90EF90DF90F1
:10590000CF900C9491220E945F1F20E030E0A9010B
:10591000C701B6010F94E02587FF15C0C12CD12C1B
:10592000760121C020E030E04CE053E4C701B6012D
:105930000F94102F1816E4F6C12CD12C9CE0E92E00
:1059400093E4F92ED5CF20E030E046E953E4C701D7
:10595000B6010F94102F181634F4C12CD12C86E9FF
:10596000E82E83E4F82EC701B6010F941D2FCB015A
:10597000FF90EF90DF90CF900C94531F9091360CD6
:10598000977081E0973009F080E0089520918705B5
:1059900020FF14C020E83EE3629FA001639F500DEA
:1059A000729F500D1124CA019695879596958795FB
:1059B000009731F08A950000E9F708950C943F268E
:1059C0000895CF93DF931092E50B1092860C1092FE
:1059D000880C1092870C1092860510928505CFEFE7
:1059E000DFEF8091301485FD07C00E94D9AAD093C3
:1059F000AF12C093AE12F5CF8FEF9FEF9093AF121F
:105A00008093AE12DF91CF9108958F929F92AF92C3
:105A1000BF92CF92DF92EF92FF920F931F93CF939B
:105A2000DF9310923A05109239052FE32093340545
:105A300010923305109232051092310510923505FF
:105A40001092360510923705109238059C01F90125
:105A500090812F5F3F4F9032D1F39E34C9F4818102
:105A600090ED980F9A3020F08D3211F08B3281F446
:105A700032969F012F5F3F4F808180538A3008F418
:105A80007BC09F012F5F3F4F8081803209F476C039
:105A9000F0938507E09384078F010F5F1F4FC0814C
:105AA0006AE270E0C8010F94FE2F009731F0FC010C
:105AB000319780818032E1F31182CD3429F0C435F1
:105AC00019F0C73409F04BC0F80180810F5F1F4FF8
:105AD0008032D1F380538A3008F041C0C09334053E
:105AE00030E020E04AE0DF011196429FC001439F71
:105AF000900D11249C01205331098081280F311D04
:105B000087FD3A95818190ED980F9A30C8F13093D6
:105B10003305209332058E3261F4329690E04AE0EC
:105B2000DF0131968C9150ED580F5A3058F1909317
:105B30003105CD01DC0101964C914032D9F3CD34D1
:105B400089F52E31310539F018F52731310519F075
:105B50002C31310539F5B0933A05A0933905DF9121
:105B6000CF911F910F91FF90EF90DF90CF90BF905A
:105B7000AF909F908F900895F9017BCFF90181CF6D
:105B8000FD01B1CF949F800D112490ED980FC8CFE7
:105B90002537310538F027373105E8F2203A83E020
:105BA0003807C9F2D091840740E050E0BA0110E014
:105BB00000E0C12CD12C7601C394FD0131968C916B
:105BC000882309F47FC08132E1F4CD34D1F420324E
:105BD0003105B9F440933505509336056093370588
:105BE00070933805F0933A05E093390563E270E06D
:105BF000CF010F94FE2F009709F4B1CFFC01108262
:105C0000AECF81548A3108F058C0DF019D919032A7
:105C100091F0A0EDA90FAA30E8F09E3271F49181C5
:105C200090539A30B8F00115110519F48F01015005
:105C3000110990E013C0FD01E8CF9D3211F09B32B5
:105C400091F79181A0EDA90FAA3020F09E3259F76B
:105C50009281E6CF9E2F9D1B309759F3A82FB0E07D
:105C60004601570104C0880C991CAA1CBB1C8A95CC
:105C7000D2F7482959296A297B29A95EBA4F9C93F2
:105C800080818154DF018A3108F497CFDF0181914F
:105C9000882309F492CF90ED980F9A30B8F393EDE2
:105CA000980F923098F38B3289F3CD010196EC91E5
:105CB000E03209F082CFDC01F8CF0115110501F7C0
:105CC0008D01DECF10933A050093390540933505D9
:105CD00050933605609337057093380540CF4F9247
:105CE0005F926F927F928F929F92AF92BF92CF926C
:105CF000DF92EF92FF92CF93DF9300D000D01F92FC
:105D00001F92CDB7DEB75C01DB01CD90DD90ED9049
:105D1000FC90E0918312F0918412FE83ED838481E4
:105D20009581A681B78189839A83AB83BC839C01CB
:105D3000AD01C701B6010F94AF2C2B013C01F50159
:105D400080809180A280B380AD81BE818D919D9134
:105D50000D90BC91A02D8D839E83AF83B88727E1E2
:105D600037EB41ED58EBC301B2010F94102F87FDC3
:105D7000D0C023E030E04BE953E4C301B2010F94FB
:105D8000E02518160CF4C5C02D813E814F81588541
:105D9000C501B4010F94AF2C2B013C0127E137EB77
:105DA00041ED58EB0F94102F87FDB3C023E030E88E
:105DB0004DE953E4C301B2010F94E02518160CF429
:105DC000A8C020E030E0A9016D817E818F81988597
:105DD0000F94B02C2B013C0120E030E040E450E473
:105DE0000F94E02587FF05C0412C512C30E4632E31
:105DF000762C27E137EB41ED58E3C301B2010F9454
:105E0000AF2C9B01AC01C501B4010F94102F87FD8D
:105E100080C020E030E84DE953E46D817E818F81C0
:105E200098850F94B02C2B013C0120E030E844E928
:105E300053E40F94102F18163CF4412C20E8522EF6
:105E400024E9622E23E4722E27E137EB41ED58E37B
:105E5000C301B2010F94B02C9B01AC01C501B40188
:105E60000F94E02518160CF454C020E030E0A9018E
:105E700069817A818B819C810F94B02C4B015C01EC
:105E800020E030E040E051E40F94E02587FF05C0BA
:105E9000812C912CA12C91E4B92E27E137EB41ED17
:105EA00058E3C501B4010F94AF2C9B01AC01C701AD
:105EB000B6010F94102F87FD2CC020E030E04BE995
:105EC00053E469817A818B819C810F94B02C4B01C2
:105ED0005C0120E030E042E953E40F94102F1816E3
:105EE00034F4812C912C82E9A82E83E4B82E27E18A
:105EF00037EB41ED58E3C501B4010F94B02C9B0181
:105F0000AC01B1E0B983C701B6010F94E0251816C2
:105F10000CF41982898128960FB6F894DEBF0FBE63
:105F2000CDBFDF91CF91FF90EF90DF90CF90BF90EA
:105F3000AF909F908F907F906F905F904F9008955B
:105F4000E0E1F8E082EBDF011D928A95E9F7089520
:105F50008091CB05811104C00E94A02F0C943AB807
:105F60008091301482FD0C9446F7089580911008BA
:105F7000882361F09091C108891308C08091301482
:105F800083FF04C08EE498E00C9404B780E0089589
:105F9000FC01238121110C9439B30895EFE6F0E060
:105FA0008081826080830895CF92DF92EF92FF928A
:105FB000CF93DF93C82F0E943F2A94E0C99FE0014E
:105FC0001124FE01E250FA4FC080D180E280F380BC
:105FD00081110E94CE2FCB59DE4EC701B6010F941E
:105FE000E725288139814A815B810F944626DF911C
:105FF000CF91FF90EF90DF90CF9008958F929F9276
:10600000AF92BF92CF92DF92EF92FF921F93CF9306
:10601000DF93CDB7DEB760970FB6F894DEBF0FBE43
:10602000CDBF182F80E00E94D42F4B015C018092DD
:106030008A0590928B05A0928C05B0928D0581E027
:106040000E94D42F6B017C01C0928E05D0928F05E7
:10605000E0929005F092910582E00E94D42F609327
:1060600092057093930580939405909395051D86F2
:106070001E861F86188A89829A82AB82BC82CD8254
:10608000DE82EF82F88669877A878B879C8783E038
:106090000E94D42F6D877E878F87988B8091370CD5
:1060A000882321F0CE0101960E9455211E3FD9F48C
:1060B00080E1FE013196A6E2BCE001900D928A9546
:1060C000E1F760960FB6F894DEBF0FBECDBFDF914B
:1060D000CF911F91FF90EF90DF90CF90BF90AF9046
:1060E0009F908F90089584E0189FF0011124DF01A4
:1060F000AA5DB34F81E090E08C0F9D1FE80FF91F60
:1061000040815181628173814D935D936D937C9346
:106110001397D7CFCF92DF92EF92FF92CF93DF9377
:10612000C82F0E943F2A94E0C99FE0011124FE017C
:10613000EE50FA4FC080D180E280F38081110E943E
:10614000CE2FCB59DE4EC701B6010F94E72528812B
:1061500039814A815B810F944626DF91CF91FF9070
:10616000EF90DF90CF9008950E943F2A909189127E
:1061700090938812909387129093861294E690934E
:10618000851220ED33E03093030920930209811139
:106190000E94CE2F81E08093F1050895CF93DF9385
:1061A000CDB7DEB72C970FB6F894DEBF0FBECDBFCC
:1061B0000E9463F60E943F2A9CE0EEEFF5E0DE01CC
:1061C000119601900D929A95E1F781110E94CE2FC0
:1061D000CE0101960E947AC62C960FB6F894DEBFC7
:1061E0000FBECDBFDF91CF9108952F923F924F9276
:1061F0005F926F927F928F929F92AF92BF92CF9257
:10620000DF92EF92FF920F931F93CF93DF9300D013
:10621000CDB7DEB78090260C9090270CA090280C6C
:10622000B090290C40902A0C50902B0C60902C0CB4
:1062300070902D0CC0902E0CD0902F0CE090300C54
:10624000F090310C0E94E81B0E94361C03E81CE110
:1062500087E492E09B838A8387E7282E8CE1382E9F
:10626000198289810E94D91CC8010E94BC1DEA8143
:10627000FB816193719381939193FB83EA83C101C5
:106280000E94BC1DEA81FB816087718782879387AA
:10629000F981FF5FF9830C5F1F4F84E0280E311CEA
:1062A000F330F9F68CED95E00E94C8F60E94D81EF6
:1062B0000E941D27A50194016091260C7091270C66
:1062C0008091280C9091290C0F94E02581111CC01D
:1062D000A301920160912A0C70912B0C80912C0CDF
:1062E00090912D0C0F94E02581110EC020912E0C61
:1062F00030912F0C4091300C5091310CC701B601F8
:106300000F94E0258823B9F00F900F900F90DF9144
:10631000CF911F910F91FF90EF90DF90CF90BF90A2
:10632000AF909F908F907F906F905F904F903F9035
:106330002F900C94CE300F900F900F90DF91CF9153
:106340001F910F91FF90EF90DF90CF90BF90AF9093
:106350009F908F907F906F905F904F903F902F9085
:1063600008958091791190917A11892B79F4809117
:10637000791190917A11892B49F4209179113091FA
:106380007A1181E0232B19F480E0089581E00895CB
:106390001092EB048091220290912302A09124029A
:1063A000B09125028093E8059093E905A093EA0552
:1063B000B093EB0508959091901110929011923046
:1063C00071F0943079F0913099F4813089F48091B2
:1063D000EB04882369F0109226020C94C8311092C5
:1063E000250C08958AE898E19093850C8093840C9D
:1063F00008959091301493FB882780F993FF06C08D
:1064000081E090919715911101C080E00895CF939C
:10641000C0918805CF7739F50E94F931882319F1A9
:106420008091281490912914A0912A14B0912B14D2
:106430000097A105B105B9F0BC01CD016D597F4FA1
:106440008F4F9F4F24E630E040E050E00F94242C23
:1064500060912C1470912D1480912E1490912F1412
:106460000F94242CC22F8C2FCF910895EFEFF8E0DA
:1064700010821182089581E00895DC01EC918E2F45
:1064800090E0FC01EE0FFF1FE80FF91FE55DFD4EE8
:1064900080818F77808308958F929F92AF92BF9271
:1064A000CF92DF92EF92FF920F93CF93DF931F92E1
:1064B000CDB7DEB75C017B0149016B01C40ED51E6F
:1064C000F501808191810F94FE2B8983002311F0C7
:1064D000F7018083BE016F5F7F4FC4010E94E2E03D
:1064E000F50180819181019691838083FFEFEF1AFE
:1064F000FF0AEC14FD0421F780E00F90DF91CF91AB
:106500000F91FF90EF90DF90CF90BF90AF909F9052
:106510008F9008950F93AB010091E00521E00227D1
:1065200021EE35E0BC0181EC95E00E944C320F91E8
:106530000895009781F41092900082E0809391007A
:106540001092950010929400C19A8091710082601F
:10655000809371000895019761F41092A00082E089
:106560008093A1001092A5001092A40089BB809393
:10657000720008957F928F929F92AF92BF92CF92B6
:10658000DF92EF92FF920F931F93CF93DF93EC0173
:106590007B018881883108F0C3C090E0FC01EE0FD8
:1065A000FF1FE80FF91FE55DFD4E80818F770E9488
:1065B0002EE719821A8288812CE0622F0F94872C93
:1065C000829FB001112430E020E0AB01420F531F45
:1065D000FA01EE0FFF1FE40FF51FE55DFD4E908100
:1065E00097FD08C02F5F3F4F2C30310571F790E0C9
:1065F0000E9499327880072D10E06801CC0CDD1CD8
:10660000F601E00FF11FE55DFD4E8081806880831B
:1066100077FC86C080E2E81682E0F8060CF03FC006
:106620008A8128E532E0281B310987FD3395220F46
:10663000331F220F331F032E000C440B550B89818F
:1066400078E8872E912C881A910887FD9394880CFE
:10665000991C880C991C092C000CAA08BB0860E046
:1066600070E0CB01F7FC0AC0B701653B710514F07F
:1066700064EB70E0072E000C880B990B2819390980
:106680004A095B090F94142C24EB30E040E050E001
:106690000F94462C820E931EA41EB51E740187E132
:1066A0008715D8F0298188E890E0821B910927FDA1
:1066B0009395880F991F880F991FE816F90604F51E
:1066C00002972FB7F894E601C00FD11FC55DDD4ECC
:1066D000880F991F9A8389832FBF62E370E080E05F
:1066E00090E0DF91CF911F910F91FF90EF90DF909D
:1066F000CF90BF90AF909F908F907F900C943F264B
:106700002A8188E592E0821B910927FD9395880FE5
:10671000991F880F991FE816F90694F6C701D0CF84
:10672000DF91CF911F910F91FF90EF90DF90CF906D
:10673000BF90AF909F908F907F900895CF93DF93FD
:10674000EB01682F70E084E792E10E94BA32688121
:1067500079818A819B81643F21E0720781059105DF
:1067600020F464EF71E080E090E00E943F2689B160
:1067700082FB882780F9DF91CF910895CF93DF9333
:1067800000D01F92CDB7DEB78EEE92E0A0E0B0E071
:1067900089839A83AB83BC83BE016F5F7F4F8AE599
:1067A0000E949E330F900F900F900F90DF91CF912A
:1067B0000895CF93DF9300D01F92CDB7DEB78EEE52
:1067C00092E0A0E0B0E089839A83AB83BC83BE01F2
:1067D0006F5F7F4F8AE00E949E330F900F900F9063
:1067E0000F90DF91CF910895CF93DF9300D01F9248
:1067F000CDB7DEB784EF91E0A0E0B0E089839A8363
:10680000AB83BC83BE016F5F7F4F80EA0E949E33E3
:106810000F900F900F900F90DF91CF9108951F92DE
:106820000F920FB60F9211240BB60F922F933F9336
:106830004F935F936F937F938F939F93AF93BF9388
:10684000EF93FF9348EA50E064EA70E081E090E063
:106850000E946326FF91EF91BF91AF919F918F911D
:106860007F916F915F914F913F912F910F900BBE50
:106870000F900FBE0F901F9018951F920F920FB69A
:106880000F9211240BB60F922F933F934F935F9368
:106890006F937F938F939F93AF93BF93EF93FF93E8
:1068A00048E950E064E970E090E080E00E946326EF
:1068B000FF91EF91BF91AF919F918F917F916F91D8
:1068C0005F914F913F912F910F900BBE0F900FBE94
:1068D0000F901F9018959091D10095FD0CC090914C
:1068E000D00095FF08C08093D6008091D0008064CE
:1068F0008093D0000895209118042F5F2F770FB652
:1069000007FC27C090911904921328C09091D000E1
:1069100095FF1EC09091190440911804941306C06D
:106920009091D1009F7D9093D10012C0E92FF0E0AB
:10693000E85EFB4F32819F5F9F773093D600909344
:1069400019043091D00030643093D000491741F3DE
:10695000D9CF90911904921301C0FBCFE091180494
:10696000F0E0E85EFB4F8283209318048091D10011
:1069700080628093D10008958F929F92AF92BF92D0
:10698000CF92DF92EF92FF920F931F93CF93DF93FB
:106990007C0121E5E20EF11CD7014C914A3509F04A
:1069A000A4C06C01B2E5CB0ED11CF6013081353AA2
:1069B00009F09BC0EC01C05BDF4F2881233008F455
:1069C00094C08C0100561F4FD8014C93E15BFF4FE0
:1069D000308331962083EF54F1093081E05BFF4F23
:1069E00030833038B1F43196AC54B1093C913083E6
:1069F000E854F109AF5ABF4F50E040E02250330B4A
:106A000042175307CCF4808132968D934F5F5F4FCE
:106A1000F7CF233031F5313809F074C0FC01EC5563
:106A2000FF4FDC01AC5ABF4F2C9120833196885A1E
:106A30009F4FDC018C9180834801B12CA12C88816F
:106A400090E002968A159B050CF43FC0F4018191F9
:106A50004F010E946B340E94F8E0FFEFAF1ABF0AAB
:106A6000EECF323821F5FC01EC5AFF4F30814181E5
:106A7000E05BFF4F408331963083DC01AA55BF4F66
:106A800050E040E02350330B42175307ACF6FA01B5
:106A9000EE7FE45AFF4FE80FF91F608171817C930C
:106AA00011966C9311974E5F5F4F1296EDCF243085
:106AB00019F6333809F6FC01EC5AFF4F2081318179
:106AC000E05BFF4F30833196B0CF80E5DE011D9251
:106AD0008A95E9F78AE1F80111928A95E9F78AE542
:106AE000D7018C9385EAF6018083DF91CF911F91C6
:106AF0000F91FF90EF90DF90CF90BF90AF909F905D
:106B00008F900895323809F097CFADCFAF92BF92F2
:106B1000CF92DF92EF92FF920F931F93CF93DF9369
:106B2000EC0184E6C82E80E2D82EE12CF12C02E89C
:106B3000A12C90E2B92E15E00093BD13C092BE13B4
:106B4000D092BF13E092C013F092C113B092C7135A
:106B5000A092C6131093BA138AE693E10E94BC3444
:106B60008FEFC81AD80AE80AF80A88E7C81680E240
:106B7000D806E104F10401F724E630E240E050E0F9
:106B8000BE018AE693E1DF91CF911F910F91FF90B3
:106B9000EF90DF90CF90BF90AF900C94FDE0CF923C
:106BA000DF92EF92FF920F931F93CF93DF93CDB7B6
:106BB000DEB77C01CDB6DEB60F942D2501962DB73C
:106BC0003EB7281B390B0FB6F8943EBF0FBE2DBF42
:106BD0000DB71EB70F5F1F4FB701C8010F942625D1
:106BE000C8010E9486350FB6F894DEBE0FBECDBE3A
:106BF000DF91CF911F910F91FF90EF90DF90CF9099
:106C000008958F929F92AF92BF92CF92DF92EF92B0
:106C1000FF920F931F93CF93DF930E94E12C3AE0F2
:106C2000C32E30E2D32EE12CF12C15E002E8460110
:106C30005701CAE0D0E01092C7131092C613109308
:106C4000BA130093BD138092BE139092BF13A0920B
:106C5000C013B092C1138AE693E10E94BC3421971D
:106C60008FEF881A980AA80AB80A209721F78AE0B5
:106C7000C80ED11CE11CF11C82EDC81680E2D806BA
:106C8000E104F104A1F6C12C20E2D22EE12CF12C7A
:106C9000D5E0C2E81092C7131092C613D093BA136E
:106CA000C093BD13C092BE13D092BF13E092C01325
:106CB000F092C1138AE693E10E94BC341092C7138C
:106CC0001092C613D093BA13C093BD13D701C60157
:106CD0008C529F4FAF4FBF4F8093BE139093BF1303
:106CE000A093C013B093C1138AE693E10E94BC3411
:106CF0008FEFC81AD80AE80AF80A8AE0C81680E2B4
:106D0000D806E104F10431F69EEDC92E90E2D92EA9
:106D1000E12CF12CD5E0C2E81092C7131092C613F3
:106D2000D093BA13C093BD13C092BE13D092BF13B9
:106D3000E092C013F092C1138AE693E10E94BC3442
:106D40008FEFC81AD80AE80AF80A86EEC81680E259
:106D5000D806E104F10401F7CC24C39482E1D82ED3
:106D6000E12CF12C0AE010E0D5E0C2E81093C71343
:106D70000093C613D093BA13C093BD13C092BE1331
:106D8000D092BF13E092C013F092C1138AE693E150
:106D90000E94BC341093C7130093C613D093BA1348
:106DA000C093BD13D701C6018096A11DB11D80936C
:106DB000BE139093BF13A093C013B093C1138AE680
:106DC00093E10E94BC348FEFC81AD80AE80AF80A87
:106DD00085E1C81682E1D806E104F10439F682E1C2
:106DE00090E09093C7138093C613D093BA13C093C7
:106DF000BD1384E190E1A0E0B0E08093BE139093D6
:106E0000BF13A093C013B093C1138AE693E1DF913F
:106E1000CF911F910F91FF90EF90DF90CF90BF9097
:106E2000AF909F908F900C94BC341F920F920FB62E
:106E30000F9211240BB60F922F938F939F93EF9382
:106E4000FF938091190420911804821306C0809149
:106E5000D1008F7D8093D10012C0E82FF0E0E85E72
:106E6000FB4F92818F5F8F779093D60080931904A8
:106E70009091D00090649093D000281741F3FF9137
:106E8000EF919F918F912F910F900BBE0F900FBE9E
:106E90000F901F9018951F920F920FB60F9211240A
:106EA0000BB60F920F931F932F933F934F935F93C4
:106EB0006F937F938F939F93AF93BF93CF93DF9302
:106EC000EF93FF93C091D60000913C05D0913B0514
:106ED00011E01D0F1F7390911704913108F09FC0AE
:106EE000E92FF0E08827E858F84C8F4F0D94A72C35
:106EF0008937B837C737D637DD370F38E1370F381E
:106F0000E537E9370F38ED37F137F537FC370F380C
:106F10000738C03229F028F5CA3011F0CD3031F5EC
:106F2000011731F0ED2FF0E0E55CFA4FC283D12F6D
:106F3000D0933B05FF91EF91DF91CF91BF91AF913E
:106F40009F918F917F916F915F914F913F912F9181
:106F50001F910F910F900BBE0F900FBE0F901F90BF
:106F60001895CD3481F081E0CE3471F080E10CC011
:106F7000CA3338F4C033A0F6C03291F2CD32B1F743
:106F8000CFCFCD3499F782E080931704C9CFC133B6
:106F900059F018F4C03221F2E9CF88E0C433A1F3EC
:106FA0008BE0C83389F3E2CF83E0EECF84E0C033D7
:106FB00059F386E0C13341F3D9CF85E0C833B1F648
:106FC000E3CF87E0C23391F6DFCF89E0C13371F6BA
:106FD000DBCF8AE0C03351F6D7CF8CE0C73331F630
:106FE000D3CF8DE0C63311F6CFCFC03209F498CF9E
:106FF0008EE0C33549F2BACF80ED8C0F8A3008F0AD
:107000008FCF9FE0909317048093160489CFCA30E6
:1070100019F0CD3009F084CF1092170481CFCA3017
:1070200019F0CD3009F07CCF809124148823A1F38E
:10703000973089F038F4953079F710923C0210922D
:10704000250CEACF9A3059F09F3031F78091160421
:107050000E94DB31E1CF81E080930F06DDCF81E03C
:1070600080930E06D9CF9091C00095FFFCCF8093FE
:10707000C6000895CF93DF93EC018991882319F01E
:107080000E943338FACF8DE00E9433388AE0DF91D6
:10709000CF910C943338CF92DF92EF92FF92CF933F
:1070A0006B017C01C42F4A3069F4F7FE0BC0F094E9
:1070B000E094D094C094C11CD11CE11CF11C8DE261
:1070C0000E9433384C2FC701B601CF91FF90EF904B
:1070D000DF90CF900C9472AACF93DF93EC01FE0166
:1070E00084912196882319F00E943338F8CFDF91DC
:1070F000CF910895CF93DF93D09123118FE59CE139
:107100000E946C388AE00E9433388091A20C87304C
:1071100009F449C083E080939D0C81E080936E0266
:1071200080E190E09093C7138093C61385E080932D
:10713000BA13C2E8C093BD1384E190E1A0E0B0E0CF
:107140008093BE139093BF13A093C013B093C11349
:107150008AE693E10E94BC3461E070E080E090E058
:107160000E94C62C81E09AE59093C7138093C613C2
:1071700085E390E09093C9138093C81387E08093D0
:10718000BA13C093BD1384E890E0A0E0B0E0809310
:10719000BE139093BF13A093C013B093C1138AE69C
:1071A00093E10E94BC3480912311813089F18230B7
:1071B00061F50E94B32B6093A9057093AA05809393
:1071C000AB059093AC0581E0809323110E943EFDB6
:1071D0006093A5057093A6058093A7059093A805D5
:1071E000D23089F080919206909193060196909307
:1071F0009306809392061092B1051092B2051092F8
:10720000B3051092B40581E004C00E94E52BDBCFEA
:1072100080E0DF91CF910895CF93C82FCB010E94DA
:107220006C3883ED98E10E946C3884EC98E1CC23B3
:1072300011F089EC98E10E946C388AE0CF910C94AF
:107240003338CF93DF9300D01F92CDB7DEB784EFF2
:1072500091E0A0E0B0E089839A83AB83BC83BE0158
:107260006F5F7F4F8CE30E949E3381EF98E10E9415
:107270006C388CB16BEE78E185FB882780F90E9431
:107280000C398091030165EE78E1869581700E944A
:107290000C3989B16FED78E182FB882780F90E9473
:1072A0000C398CB166ED78E1829581700E940C39C1
:1072B0004A9909C00E94D9330F900F900F900F90F8
:1072C000DF91CF9108950E94BE330F900F900F90E1
:1072D0000F90DF91CF910895809123118130C1F5F6
:1072E0008FE998E10E946C388AE00E94333881E08F
:1072F0009AE59093C7138093C61387E590E0909327
:10730000C9138093C81387E08093BA1382E88093EF
:10731000BD1384E890E0A0E0B0E08093BE139093AA
:10732000BF13A093C013B093C1138AE693E10E94E8
:10733000BC3482E0809323110E943EFD6093AD0532
:107340007093AE058093AF059093B00581E00895EA
:1073500080E008950F931F930E943EFD00918D06DB
:1073600010918E0620918F0630919006011511051F
:107370002105310509F067C020919C12222309F4F0
:107380005FC0E0919A12215020939C1221E02E0FB1
:1073900020939A1230919D12231302C010929A12D8
:1073A00024E0E29FF0011124E256FD4E008111819C
:1073B000228133810093890610938A0620938B06DD
:1073C00030938C06600F711F811D911D60938D0697
:1073D00070938E0680938F069093900680918B0613
:1073E00090918C06892B61F11FB7F8948EE898E193
:1073F0000E946C388AE00E94333884E096E09093D3
:10740000C7138093C61380EA90E89093C9138093C2
:10741000C81387E08093BA1382E88093BD1380EA93
:1074200090E0A0E0B0E08093BE139093BF13A093D0
:10743000C013B093C1138AE693E10E94BC341FBF0E
:107440001F910F910895601B710B820B930B97FD99
:10745000F7CF409810928D0610928E0610928F06EC
:1074600010929006EDCF0F931F93CF93DF938C0173
:10747000EB0190919C1220919D12921305C00E94E5
:10748000AA390E943AC2F5CF80919B1234E0839FC3
:10749000F0011124E256FD4E11830083D383C28391
:1074A0009F5F90939C128F5F281739F080939B12F7
:1074B000DF91CF911F910F91089510929B12F8CFF9
:1074C000CF92DF92EF92FF921F93CF93DF93182F0B
:1074D000662351F01092EA041092E6041092E70439
:1074E0001092E8041092E9040E943EFD6B017C01B9
:1074F0008091E6049091E704A091E804B091E9043A
:10750000A7019601281B390B4A0B5B0BDA01C90155
:10751000B7FD3DC02091EA0417FD13C0412F012E95
:10752000000C550B4C5F5F4F822F022E000C990B05
:107530004817590764F184EF91E0A0E0B0E021170B
:1075400024F488EE93E0A0E0B0E08C0D9D1DAE1D0C
:10755000BF1D8093E6049093E704A093E804B093E2
:10756000E9042170C22F30E0D32F84E28C9FB00158
:107570008D9F700D7C1B112460597C4F82E390E03D
:107580000E94333A8091EA048F5F8093EA04DF918E
:10759000CF911F91FF90EF90DF90CF900895CF9300
:1075A000DF9300D01F92CDB7DEB784E198E10E944F
:1075B0006C388AE00E9433388091A20C8330D9F174
:1075C00019821A821B821C8260E0CE0101960E9401
:1075D000002C19821A821B821C8261E0CE01019666
:1075E0000E94002C81E080936D0210929C0C80938D
:1075F0006E0281E09AE59093C7138093C61383E3EC
:1076000090E09093C9138093C81387E08093BA13D6
:1076100082E88093BD1384E890E0A0E0B0E080931E
:10762000BE139093BF13A093C013B093C1138AE607
:1076300093E10E94BC340F900F900F900F90DF9158
:10764000CF9108956F927F928F929F92AF92BF9247
:10765000CF92DF92EF92FF920F931F93CF93DF931E
:10766000CDB7DEB764970FB6F894DEBF0FBECDBFBF
:107670001092D0008091D00082608093D000109250
:10768000D50080E18093D4008091D1008061809307
:10769000D1008091D10088608093D1008091D10089
:1076A00080688093D1008091D1008F7D8093D1003C
:1076B0008AE58093BB1380936B1385EA8093BC1398
:1076C00080936C13EAE0F4E18AE1DF011D928A9570
:1076D000E9F780919B0C882309F473C283E090E062
:1076E0009093C7138093C61385E08093BA1382E802
:1076F0008093BD138FE190E1A0E0B0E08093BE13D2
:107700009093BF13A093C013B093C1138AE693E183
:107710000E94BC3484E690E09093C7138093C61314
:1077200005E00093BA1312E81093BD1386E090E1D0
:10773000A0E0B0E08093BE139093BF13A093C0135A
:10774000B093C1138AE693E10E94BC348BE090E0D1
:107750009093C7138093C6130093BA131093BD136D
:1077600080E092E1A0E0B0E08093BE139093BF135D
:10777000A093C013B093C1138AE693E10E94BC3476
:107780001092C7131092C6130093BA131093BD132F
:1077900084E390E1A0E0B0E08093BE139093BF1328
:1077A000A093C013B093C1138AE693E10E94BC3446
:1077B0001092C7131092C6130093BA131093BD13FF
:1077C0008AE390E1A0E0B0E08093BE139093BF13F2
:1077D000A093C013B093C1138AE693E10E94BC3416
:1077E0008091EA119091EB119093C7138093C61387
:1077F0000093BA131093BD1386E390E1A0E0B0E0CC
:107800008093BE139093BF13A093C013B093C11382
:107810008AE693E10E94BC3480917F11909180119F
:107820009093C7138093C6130093BA131093BD139C
:107830008CE390E1A0E0B0E08093BE139093BF137F
:10784000A093C013B093C1138AE693E10E94BC34A5
:1078500082E090E09093C7138093C6130093BA130D
:107860001093BD138EE190E1A0E0B0E08093BE13D1
:107870009093BF13A093C013B093C1138AE693E112
:107880000E94BC3481E080936D0270E6C72E70E1E7
:10789000D72EE12CF12C1092C7131092C61300932F
:1078A000BA131093BD13C092BE13D092BF13E092CF
:1078B000C013F092C1138AE693E10E94BC34BFEF7B
:1078C000CB1ADB0AEB0AFB0AE4E7CE16E0E1DE06A0
:1078D000E104F10401F7CE0101967C0184E1D701B6
:1078E0001D928A95E9F781E08F9390E99F938F939A
:1078F0009CE29F938F939F9387E993E09F938F934D
:10790000FF92EF920F94383020E630E140E050E0F3
:1079100064EA73E08AE693E10E94FDE02AE630E142
:1079200040E050E061EB73E08AE693E10E94FDE005
:1079300024E730E140E050E0B7018AE693E10E949D
:10794000FDE02EE730E140E050E06DEB73E08AE6C9
:1079500093E10E94FDE01092C7131092C6130093AA
:10796000BA131093BD138EE090E1A0E0B0E08093D5
:10797000BE139093BF13A093C013B093C1138AE6B4
:1079800093E10E94BC341092C7131092C613009367
:10799000BA131093BD138FE090E1A0E0B0E08093A4
:1079A000BE139093BF13A093C013B093C1138AE684
:1079B00093E10E94BC340FB6F894DEBF0FBECDBF7A
:1079C0004AE0C42E40E2D42EE12CF12C55E0752E75
:1079D00062E8662E460157010AE010E01092C713D4
:1079E0001092C6137092BA136092BD138092BE13A8
:1079F0009092BF13A092C013B092C1138AE693E194
:107A00000E94BC3401501109FFEF8F1A9F0AAF0A80
:107A1000BF0A0115110511F78AE0C80ED11CE11C3F
:107A2000F11C92EDC91690E2D906E104F10491F639
:107A3000C12C30E2D32EE12CF12C05E012E810929B
:107A4000C7131092C6130093BA131093BD13C092BC
:107A5000BE13D092BF13E092C013F092C1138AE616
:107A600093E10E94BC341092C7131092C613009386
:107A7000BA131093BD13D701C6018C529F4FAF4F5D
:107A8000BF4F8093BE139093BF13A093C013B093C6
:107A9000C1138AE693E10E94BC34AFEFCA1ADA0A36
:107AA000EA0AFA0ABAE0CB16B0E2DB06E104F10416
:107AB00031F62EEDC22E20E2D22EE12CF12C05E083
:107AC00012E81092C7131092C6130093BA131093C2
:107AD000BD13C092BE13D092BF13E092C013F092B8
:107AE000C1138AE693E10E94BC34EFEFCE1ADE0A9E
:107AF000EE0AFE0AF6EECF16F0E2DF06E104F1042C
:107B000001F7CC24C39482E1D82EE12CF12C9AE029
:107B1000A92EB12C05E012E8B092C713A092C613AB
:107B20000093BA131093BD13C092BE13D092BF132B
:107B3000E092C013F092C1138AE693E10E94BC3434
:107B4000B092C713A092C6130093BA131093BD133B
:107B5000D701C6018096A11DB11D8093BE139093DD
:107B6000BF13A093C013B093C1138AE693E10E94A0
:107B7000BC348FEFC81AD80AE80AF80A95E1C9168A
:107B800092E1D906E104F10439F68AE797E10E940F
:107B90006C388AE00E94333864960FB6F894DEBFE2
:107BA0000FBECDBFDF91CF911F910F91FF90EF904E
:107BB000DF90CF90BF90AF909F908F907F906F900D
:107BC000089582E090E08CCD0E94223B10928405C3
:107BD00081E080936E028CE298E10E946C388AE02A
:107BE0000C9433380F931F93CF938C01C62F84E2EC
:107BF00094E10E946C38C8010E946C388AE30E94AC
:107C0000333880E38C0F0E9433388AE0CF911F9184
:107C10000F910C94333887EA95E10E946C3860E04C
:107C200087E995E10E94F23D60E082E895E10E94DB
:107C3000F23D61E08BE795E10E94F23D61E080E773
:107C400095E10E94F23D61E080E695E10E94F23DFF
:107C500060E087E595E10E94F23D61E08DE495E109
:107C60000E94F23D61E083E495E10E94F23D61E013
:107C70008CE395E10E94F23D61E084E395E10E948E
:107C8000F23D61E086E295E10E94F23D61E088E12B
:107C900095E10E94F23D60E089E095E10E94F23DAD
:107CA00060E08BEF94E10E94F23D60E085EE94E1AC
:107CB0000E94F23D61E084ED94E10E94F23D61E0BA
:107CC00085EC94E10E94F23D61E08EEB94E10E942C
:107CD000F23D60E087EB94E10E94F23D61E08EEAC4
:107CE00094E10E94F23D61E089E994E10E94F23D55
:107CF00061E08BE894E10E94F23D61E088E794E165
:107D00000E94F23D60E08BE694E10E94F23D61E06A
:107D100086E694E10E94F23D61E089E594E10E94EB
:107D2000F23D60E085E494E10E94F23D60E082E390
:107D300094E10E94F23D60E083E394E10E949F1D84
:107D4000682F617089E294E10C94F23D80913505D1
:107D5000827149F4809137058C7829F48091380537
:107D6000837009F475C082E40E947D1E882351F05F
:107D70000E944B246093480C7093490C80934A0CEA
:107D800090934B0C83E50E947D1E882351F00E9446
:107D9000D1246093780C7093790C80937A0C909333
:107DA0007B0C84E50E947D1E882351F00E94D12423
:107DB00060937C0C70937D0C80937E0C90937F0C71
:107DC00088E50E947D1E882351F00E94D124609393
:107DD000DB087093DC088093DD089093DE0889E56A
:107DE0000E947D1E882351F00E94D1246093DF08F9
:107DF0007093E0088093E1089093E2088AE50E947E
:107E00007D1E8823B1F00E94D1246093E308709313
:107E1000E4088093E5089093E6082DEC3CEC4CECEC
:107E20005DE30F94E025181624F088E99EE00E9497
:107E30006C3885E40E947D1E882351F00E94D12475
:107E40006093E7087093E8088093E9089093EA0844
:107E50000895AF92BF92CF92DF92EF920F931F934C
:107E6000CF93DF935B01EA016901882309F463C0C2
:107E700081E99EE00E946C38F50160817181828108
:107E8000938146E00E947ABAE1100BC088E89EE038
:107E90000E946C38688179818A819B8146E00E94CA
:107EA0007ABA81E89EE00E946C38F60160817181A7
:107EB0008281938143E00E947ABA8AE79EE00E9421
:107EC0006C38F801608171818281938143E00E9466
:107ED0007ABA81E79EE00E946C38F60120813181F8
:107EE00042815381F80160817181828193810F9475
:107EF000AF2C43E00E947ABAEE20F9F08AE00E94AB
:107F000033388CE59EE00E946C38688179818A81E3
:107F10009B8146E00E947ABA8AE00E9433388AE068
:107F2000DF91CF911F910F91EF90DF90CF90BF9095
:107F3000AF900C943338E110E4CFDF91CF911F91D3
:107F40000F91EF90DF90CF90BF90AF9008950F9377
:107F50001F93CF938C01C62F89E798E00E946C385D
:107F6000C8010E946C38CC2331F08AE0CF911F9178
:107F70000F910C943338CF911F910F9108950E9467
:107F800096E41092250C10923C020E94F93188234D
:107F900051F08091301482FD06C08AE898E19093F8
:107FA000850C8093840C61E083E898E10E94A73FF0
:107FB0000C947A380F931F93CF93DF938C016F3F0C
:107FC00019F41092641160E020916411862F062E3E
:107FD000000C990B2817190609F08CF560936411B1
:107FE00060E08DE498E10E94A73FC8010E946C38D0
:107FF0008AE00E943338C8010F942D25800F911F0D
:10800000EC01C01BD10BC034D1053CF00197FC0141
:108010002491207C2038D1F3F3CFDD27AE01B801C5
:1080200084E291E10F944E25CC5DDE4E188284E20D
:1080300091E1DF91CF911F910F910C948635DF91E3
:10804000CF911F910F9108951092250C10923C0230
:108050008091301480648093301461E08BE598E166
:108060000E94A73F40E758E168E778E185E00E9479
:108070001BE360E082E698E10C94DA3F0F931F93D4
:10808000CF938C01C62F60E083E898E00E94A73F61
:10809000C8010E946C38CC2331F08AE0CF911F9147
:1080A0000F910C943338CF911F910F91089561E097
:1080B0008BE898E00C943E40EF92FF920F931F9351
:1080C000CF937C018B01C42F60E083E898E00E948D
:1080D000A73FC7010E946C3880E20E943338C80174
:1080E0000E946C38CC2319F08C2F0E9433388AE020
:1080F000CF911F910F91FF90EF900C943338DF9246
:10810000EF92FF920F931F93CF93DF93D82E7B01B3
:108110008A01E9010E945740D092901140E0B701D6
:1081200084E799E00E945C400115110531F040E0C0
:10813000B8018DE699E00E945C40209731F040E064
:10814000BE018DE699E00E945C4061E088E699E01E
:10815000DF91CF911F910F91FF90EF90DF900C94E2
:108160003E40AF92BF92CF92DF92EF92FF920F9379
:108170001F93CF93DF9386EE97E00E946C38C0E0A8
:10818000D7E0D15021F080E20E943338FACF8C2F13
:108190000E9454E1CF5FC53099F78AE00E943338DE
:1081A0000EE817E0C0E080E20E9433388C2F0E9476
:1081B00054E15801D5E080E20E943338F501C080D7
:1081C000D180E280F380A7019601C701B6010F9428
:1081D000A22F882369F180E20E9433388DE30E9448
:1081E00033388DE30E9433388DE30E9433388DE3BA
:1081F0000E9433388DE30E943338D150F4E1AF0E42
:10820000B11CD111D8CF8AE00E943338CF5F0C5F08
:108210001F4FC53041F68AE0DF91CF911F910F913A
:10822000FF90EF90DF90CF90BF90AF900C943338D9
:1082300020E030E0A901C701B6010F94102F87FD9F
:1082400003C08BE20E94333843E0C701B6010E94AD
:108250007ABAD3CF811107C08AEC9EE00E946C38B5
:108260008AE00C9433388EEC9EE0F8CFCF93DF9306
:10827000EB010E946C38CE01DF91CF910C9412E299
:10828000CF93C62F0E946C388C2FCF910C9454E161
:10829000CF92DF92EF92FF926A017B010E946C38CD
:1082A00042E0C701B601FF90EF90DF90CF900C94B1
:1082B0007ABACF92DF92EF92FF926A017B010E941D
:1082C0006C384AE0C701B601FF90EF90DF90CF9085
:1082D0000C944B38CF93DF93EB010E946C38CE01A6
:1082E000DF91CF910C945BE14F925F926F927F92FE
:1082F0008F929F92AF92BF92CF92DF92EF92FF92B6
:108300000F931F93CF93DF9300D000D01F921F9243
:10831000CDB7DEB78091830581110AC480918105B4
:10832000909182059C012F5F3F4F309382052093EF
:1083300081058E3E924008F4FBC38091EA11909132
:10834000EB119093C7138093C61305E00093BA1303
:1083500012E81093BD1386E390E1A0E0B0E08093B3
:10836000BE139093BF13A093C013B093C1138AE6BA
:1083700093E10E94BC3480917F1190918011909381
:10838000C7138093C6130093BA131093BD138CE3E5
:1083900090E1A0E0B0E08093BE139093BF13A09350
:1083A000C013B093C1138AE693E10E94BC3480915C
:1083B000EC119091ED119093C7138093C613009325
:1083C000BA131093BD1384E390E1A0E0B0E0809372
:1083D000BE139093BF13A093C013B093C1138AE64A
:1083E00093E10E94BC34809181119091821190930D
:1083F000C7138093C6130093BA131093BD138AE377
:1084000090E1A0E0B0E08093BE139093BF13A093DF
:10841000C013B093C1138AE693E10E94BC3481E09B
:108420008093830510928205109281058091A20CA1
:10843000882339F10E94311D811123C0809180056C
:108440008F5F8093800580918005853620F01092A3
:1084500080051092A20CE091A20CE150E73008F0E8
:108460006AC00E2E000CFF0B8827E65CFD4B8F4F79
:108470000D94A72C444293425F448B44CC44044562
:10848000974210928005DFCF0E94BE2C882309F40A
:1084900052C081E080936E0286E098E10E946C38C1
:1084A0008AE00E94333880E190E09093C713809374
:1084B000C61385E08093BA1312E81093BD1384E1CC
:1084C00090E1A0E0B0E08093BE139093BF13A0931F
:1084D000C013B093C1138AE693E10E94BC3481E0DB
:1084E0009AE59093C7138093C61386E390E0909328
:1084F000C9138093C81387E08093BA131093BD13F8
:1085000084E890E0A0E0B0E08093BE139093BF13A6
:10851000A093C013B093C1138AE693E10E94BC34C8
:108520001092A20C08C00E94BE2C882321F00E9449
:10853000311D8823A9F380916E02882309F433C783
:10854000809184058111C0C284E096E09093C713A6
:108550008093C61380EA90E89093C9138093C81360
:1085600017E01093BA1302E80093BD1380EA90E07D
:10857000A0E0B0E08093BE139093BF13A093C0130C
:10858000B093C1138AE693E10E94BC3480916902E2
:1085900090916A02A0916B02B0916C020097A105C4
:1085A000B10509F03FC21092C7131092C61315E02F
:1085B0001093BA130093BD138AE890E1A0E0B0E0F5
:1085C0008093BE139093BF13A093C013B093C113B5
:1085D0008AE693E10E94BC3489E090E09093C7134F
:1085E0008093C6131093BA130093BD138CE890E1E7
:1085F000A0E0B0E08093BE139093BF13A093C0138C
:10860000B093C1138AE693E10E94BC348091690261
:1086100090916A02A0916B02B0916C020097F1E018
:10862000AF07B10508F441C2B093C713A093C613B6
:108630009093C9138093C81387E08093BA1382E89C
:108640008093BD1388E890E1A0E0B0E08093BE1372
:108650009093BF13A093C013B093C1138AE693E124
:108660000E94BC348091690290916A02A0916B02D1
:10867000B0916C02BA2FA92F982F8827009721E07C
:10868000A207B10508F417C2B093C713A093C6138D
:108690009093C9138093C81387E08093BA1312E8AC
:1086A0001093BD1381EA90E0A0E0B0E08093BE1388
:1086B0009093BF13A093C013B093C1138AE693E1C4
:1086C0000E94BC348091370C882309F4FAC183E0FE
:1086D00090E09093C7138093C61385E08093BA13FC
:1086E0001093BD1385E490E1A0E0B0E08093BE1349
:1086F0009093BF13A093C013B093C1138AE693E184
:108700000E94BC3480918405875E8093840520910B
:108710008405822F90E0253608F021C29093C7137C
:108720008093C61385E08093BA1382E88093BD13CB
:1087300080E090E1A0E0B0E08093BE139093BF137F
:10874000A093C013B093C1138AE693E10E94BC3496
:108750000E94311D811114C20E94F931811105C09E
:108760009091870591FD0E94311D9091870580FBB6
:1087700091F99093870591FD03C28091301482FD99
:10878000FFC1809123118150823008F4F9C16091BA
:10879000811170918211072E000C880B990B0F9498
:1087A000E7256B017C0120E030E0A9010F94E02572
:1087B000882309F4BBC660917F1170918011072E48
:1087C000000C880B990B0F94E7252B013C0120E04E
:1087D00030E040E050E4C701B6010F94AF2CA30194
:1087E00092010F94102F18160CF4C2C66091EA1172
:1087F0007091EB11072E000C880B990B0F94E72555
:108800006D837E838F8398876091EC117091ED1159
:10881000072E000C880B990B0F94E7254B015C0188
:1088200020E030E040E251E40F94AF2C2D813E81F6
:108830004F8158850F94102F18160CF499C620E01C
:1088400030E040E050E4C701B6010F94B02CA30122
:1088500092010F94E02587FD10C020E030E040E257
:1088600051E4C501B4010F94B02C2D813E814F819C
:1088700058850F94E02587FF6AC684E190E09093C5
:10888000C7138093C61385E08093BA1382E8809360
:10889000BD1384E190E1A0E0B0E08093BE1390931B
:1088A000BF13A093C013B093C1138AE693E10E9453
:1088B000BC3480919D0C81117CC682E07AC688EF21
:1088C00097E10E946C388AE00E94333881E09AE593
:1088D0009093C7138093C61380E490E09093C913DC
:1088E0008093C81317E01093BA1382E88093BD13E6
:1088F00084E890E0A0E0B0E08093BE139093BF13B3
:10890000A093C013B093C1138AE693E10E94BC34D4
:108910001093A20C10CE80918C0C882309F40BCEFE
:108920000E94BE2C882309F406CE0E94311D8111BD
:1089300002CE8AEE97E10E946C388AE00E943338BA
:1089400080918D0C90E0B0E0A0E0895B9F4FAE4F2E
:10895000B54A21E03AE53093C7132093C6139093AC
:10896000C9138093C81387E08093BA1382E8809379
:10897000BD1384E890E0A0E0B0E08093BE13909334
:10898000BF13A093C013B093C1138AE693E10E9472
:10899000BC3410928C0CC4CD0E94BE2C882309F4E8
:1089A000CACD0E94311D8111C6CD81E080936E0237
:1089B0001092A20C8CED97E10E946C388AE00E9424
:1089C000333881E09AE59093C7138093C6138EE401
:1089D00090E09093C9138093C81387E08093BA13F3
:1089E00082E88093BD1384E890E0A0E0B0E080933B
:1089F000BE139093BF13A093C013B093C1138AE624
:108A000093E10E94BC3497CD0E94311D811193CD1A
:108A100019821A821B821C8262E0CE0101960E949A
:108A2000E3F47ECD0196A11DB11D35E0B695A79565
:108A3000979587953A95D1F70197A109B1090097C4
:108A4000E1E0AE07B10548F1B093C713A093C61398
:108A50009093C9138093C8131093BA1312E810931C
:108A6000BD138AE890E1A0E0B0E08093BE1390933C
:108A7000BF13A093C013B093C1138AE693E10E9481
:108A8000BC3488E090E09093C7138093C61385E0D0
:108A90008093BA131093BD13A9CD9093C7138093FD
:108AA000C61385E08093BA13D9CF9093C7138093F0
:108AB000C61385E0C2CD9093C7138093C61385E09B
:108AC000ECCD82E090E005CE8A3F08F020CE8EEF1C
:108AD000809384058BEC97E10E946C388AE00E94B9
:108AE000333881E080936E0281E09AE59093C7135A
:108AF0008093C6138DE290E09093C9138093C813BE
:108B000087E08093BA1382E88093BD1384E890E0F5
:108B1000A0E0B0E08093BE139093BF13A093C01366
:108B2000B093C1138AE693E10E94BC34109283058E
:108B300028960FB6F894DEBF0FBECDBFDF91CF9160
:108B40001F910F91FF90EF90DF90CF90BF90AF906B
:108B50009F908F907F906F905F904F900895845674
:108B600091099093C7138093C61385E08093BA133D
:108B700082E88093BD1381E090E1A0E0B0E0DCCD1D
:108B80008CE090E09093C7138093C61315E0109388
:108B9000BA1382E88093BD1384E190E1A0E0B0E0D5
:108BA0008093BE139093BF13A093C013B093C113CF
:108BB0008AE693E10E94BC340E94B32B20E13EE0A0
:108BC00040E050E00F94242C2115310581E0480746
:108BD000510508F470C05093C7134093C6133093E7
:108BE000C9132093C81387E08093BA1312E8109337
:108BF000BD1380E190E1A0E0B0E08093BE139093BC
:108C0000BF13A093C013B093C1138AE693E10E94EF
:108C1000BC340E94B32B20E13EE040E050E00F94D2
:108C2000242C2CE330E040E050E00F94242C3093CF
:108C3000C7132093C61305E00093BA131093BD1316
:108C400082E190E1A0E0B0E08093BE139093BF1367
:108C5000A093C013B093C1138AE693E10E94BC3481
:108C60000E940732882309F45CC48F5F80937F05DC
:108C7000E82EF12C833330F5EE0CFF1CF092C71375
:108C8000E092C6130093BA131093BD138EE090E1E7
:108C9000A0E0B0E08093BE139093BF13A093C013E5
:108CA000B093C1138AE693E10E94BC341092C713BB
:108CB0001092C6132BC03093C7132093C613109382
:108CC000BA1394CF84E690E09093C7138093C613B1
:108CD0000093BA131093BD138EE090E1A0E0B0E0D2
:108CE0008093BE139093BF13A093C013B093C1138E
:108CF0008AE693E10E94BC34A2E3EA1AA0E8FA0AE9
:108D0000EE0CFF1CF092C713E092C6130093BA1347
:108D10001093BD138FE090E1A0E0B0E08093BE130C
:108D20009093BF13A093C013B093C1138AE693E14D
:108D30000E94BC340E94073290E09093C713809346
:108D4000C61385E08093BA1382E88093BD1386E151
:108D500090E1A0E0B0E08093BE139093BF13A09386
:108D6000C013B093C1138AE693E10E94BC3420E0A3
:108D700030E0A90160917F12709180128091811280
:108D8000909182120F94B02C20E030E048EC52E435
:108D90000F9446260F941C2E7093C7136093C6132E
:108DA00005E00093BA1312E81093BD1386E290E138
:108DB000A0E0B0E08093BE139093BF13A093C013C4
:108DC000B093C1138AE693E10E94BC34809165029E
:108DD000909166029093C7138093C6130093BA13C1
:108DE0001093BD1380E093E1A0E0B0E08093BE1348
:108DF0009093BF13A093C013B093C1138AE693E17D
:108E00000E94BC3420E030E040E251E460914C0C20
:108E100070914D0C80914E0C90914F0C0F94462602
:108E20000F94232E7093C7136093C6130093BA1345
:108E30001093BD1382E492E1A0E0B0E08093BE13F2
:108E40009093BF13A093C013B093C1138AE693E12C
:108E50000E94BC3420E030E040E251E46091500CCC
:108E60007091510C8091520C9091530C0F944626A6
:108E70000F94232E7093C7136093C6130093BA13F5
:108E80001093BD1386E492E1A0E0B0E08093BE139E
:108E90009093BF13A093C013B093C1138AE693E1DC
:108EA0000E94BC3420E030E040E251E46091540C78
:108EB0007091550C8091560C9091570C0F9446264A
:108EC0000F94232E7093C7136093C6130093BA13A5
:108ED0001093BD138AE492E1A0E0B0E08093BE134A
:108EE0009093BF13A093C013B093C1138AE693E18C
:108EF0000E94BC3420E030E040E251E46091580C24
:108F00007091590C80915A0C90915B0C0F944626ED
:108F10000F94232E7093C7136093C6130093BA1354
:108F20001093BD138EE492E1A0E0B0E08093BE13F5
:108F30009093BF13A093C013B093C1138AE693E13B
:108F40000E94BC3420E030E048EC52E4609177129B
:108F5000709178128091791290917A120F9446262E
:108F60000F941C2E7093C7136093C6130093BA130B
:108F70001093BD1386E392E1A0E0B0E08093BE13AE
:108F80009093BF13A093C013B093C1138AE693E1EB
:108F90000E94BC3420E030E048EC52E460917B1247
:108FA00070917C1280917D1290917E120F944626D2
:108FB0000F941C2E7093C7136093C6130093BA13BB
:108FC0001093BD138AE392E1A0E0B0E08093BE135A
:108FD0009093BF13A093C013B093C1138AE693E19B
:108FE0000E94BC3480917502909176029093C713D1
:108FF0008093C6130093BA131093BD1382E592E1D8
:10900000A0E0B0E08093BE139093BF13A093C01371
:10901000B093C1138AE693E10E94BC34809173023D
:10902000909174029093C7138093C6130093BA1360
:109030001093BD1384E592E1A0E0B0E08093BE13ED
:109040009093BF13A093C013B093C1138AE693E12A
:109050000E94BC3420E030E040E251E46091EF1126
:109060007091F0118091F1119091F2110F944626B8
:109070000F94232E7093C7136093C6130093BA13F3
:109080001093BD1386E592E1A0E0B0E08093BE139B
:109090009093BF13A093C013B093C1138AE693E1DA
:1090A0000E94BC342CEA35EC47E25EE36091F31198
:1090B0007091F4118091F5119091F6110F94AA2DF1
:1090C00020E030E040E251E40F9446260F94232E36
:1090D0007093C7136093C6130093BA131093BD1314
:1090E0008AE592E1A0E0B0E08093BE139093BF13B5
:1090F000A093C013B093C1138AE693E10E94BC34DD
:109100002CEA35EC47E25EE36091F7117091F811BB
:109110008091F9119091FA110F94462620E030E0E9
:1091200040E251E40F9446260F94232E7093C71308
:109130006093C6130093BA131093BD138EE592E1AA
:10914000A0E0B0E08093BE139093BF13A093C01330
:10915000B093C1138AE693E10E94BC3420E030E072
:1091600040E251E4609184117091851180918611E3
:10917000909187110F9446260F94232E7093C71356
:109180006093C6130093BA131093BD1382E692E165
:10919000A0E0B0E08093BE139093BF13A093C013E0
:1091A000B093C1138AE693E10E94BC342CEA35ECFB
:1091B00047E25EE3609188117091891180918A1174
:1091C00090918B110F94AA2D20E030E040E251E401
:1091D0000F9446260F94232E7093C7136093C613E3
:1091E0000093BA131093BD1386E692E1A0E0B0E0BD
:1091F0008093BE139093BF13A093C013B093C11379
:109200008AE693E10E94BC342CEA35EC47E25EE347
:1092100060918C1170918D1180918E1190918F11B0
:109220000F94462620E030E040E251E40F944626B9
:109230000F94232E7093C7136093C6130093BA1331
:109240001093BD138AE692E1A0E0B0E08093BE13D4
:109250009093BF13A093C013B093C1138AE693E118
:109260000E94BC348091960C811105C08091980CAD
:10927000882309F46DC06091EA117091EB11072EFB
:10928000000C880B990B0F94E72520E030E048ECA8
:1092900052E40F9446266B017C016091EC117091B1
:1092A000ED11072E000C880B990B0F94E7259B01FD
:1092B000AC01C701B6010F94AA2D0F94232E653679
:1092C000710510F064E670E07093C7136093C613E5
:1092D00005E00093BA1312E81093BD1384E290E105
:1092E000A0E0B0E08093BE139093BF13A093C0138F
:1092F000B093C1138AE693E10E94BC346091EA11F5
:109300007091EB11072E000C880B990B0F94E72539
:109310006B017C0120E030E04AE253E40F94102F0F
:10932000181624F48091960C811146C16091EC11BD
:109330007091ED11072E000C880B990B0F94E72507
:109340009B01AC01C701B6010F94102F87FFAFC17D
:1093500080918C0C882339F180918B0C91E0980FCF
:1093600090938B0C90E09093C7138093C61385E085
:109370008093BA1382E88093BD1382E490E1A0E069
:10938000B0E08093BE139093BF13A093C013B0932B
:10939000C1138AE693E10E94BC3480918B0C8A3021
:1093A00010F010928B0C0E94492C882309F4B5C14F
:1093B0006091A00C7091A10CEE24E394F12C611546
:1093C0007105A9F090E080E00F94E52520E030E001
:1093D00040E85EE30F9446260F948E2D20E030E0A7
:1093E00040E85FE30F94B02C0F94232E7B0101E043
:1093F00010E08091860C811102C010E000E08091A5
:10940000AE129091AF128F3F980711F40E94CFB324
:109410009093AF128093AE12080F191FB80190E01D
:1094200080E00F94E52520E030E040E85EE30F9413
:1094300046260F948E2D4B015C01F092C713E092EB
:10944000C61305E00093BA1312E81093BD1380E130
:1094500093E1A0E0B0E08093BE139093BF13A0937C
:10946000C013B093C1138AE693E10E94BC34C501D6
:10947000B4010F94232E7093C7136093C613009307
:10948000BA131093BD1382E193E1A0E0B0E08093A2
:10949000BE139093BF13A093C013B093C1138AE679
:1094A00093E10E94BC340AE014E1AAE1FA2E809113
:1094B0003B0590913C0520917D0530917E05891BEF
:1094C0008F7309F449C12A3131050CF0DBC1909149
:1094D0003B0580913C054FEF5FEF981749F0E82F6F
:1094E000F0E0E55CFA4F42818F5F8F7380933C051B
:1094F000F901E65FFB4E408380910A148A3509F03A
:10950000B3C162E070E080E090E00E94C62C8091E0
:109510007D0590917E05019690937E0580937D0553
:10952000C6CF1092C7131092C613ACCB6091EC114A
:109530007091ED11072E000C880B990B0F94E72505
:1095400020E030E0A9010F94E025811134C98CE0BE
:1095500090E09093C7138093C61385E08093BA136D
:1095600082E88093BD1384E190E1A0E0B0E0F3CB0A
:109570008DE090E09093C7138093C61385E08093AD
:10958000BA1382E88093BD1384E190E1A0E0B0E0DB
:109590008093BE139093BF13A093C013B093C113D5
:1095A0008AE693E10E94BC3480919D0C811101C038
:1095B00081E080939D0CDBCB1092960C20E030E094
:1095C00040E251E460918E0C70918F0C8091900C70
:1095D0009091910C0F9446260F941C2E7093C713F4
:1095E0006093C6130093BA131093BD1384E590E102
:1095F000A0E0B0E08093BE139093BF13A093C0137C
:10960000B093C1138AE693E10E94BC3420E030E0BD
:1096100040E251E46091920C7091930C8091940C13
:109620009091950C0F9446260F941C2E7093C7139F
:109630006093C6130093BA131093BD1388E590E1AD
:10964000A0E0B0E08093BE139093BF13A093C0132B
:10965000B093C1138AE693E10E94BC348AEA97E191
:109660000E946C388AE00E94333881E09AE590933A
:10967000C7138093C61381E490E09093C91380933D
:10968000C81387E08093BA131093BD1384E890E069
:10969000A0E0B0E08093BE139093BF13A093C013DB
:1096A000B093C1138AE693E10E94BC3451CE60911D
:1096B000980C662309F44CCE062E000C770B81E93A
:1096C00097E10E946A418AE00E9433381092980C18
:1096D00084E090E09093C7138093C61385E0809355
:1096E000BA1312E81093BD138EE890E1A0E0B0E049
:1096F0008093BE139093BF13A093C013B093C11374
:109700008AE693E10E94BC3481E09AE59093C71306
:109710008093C61383E590E0B0CF1092C7131092E8
:10972000C61305E00093BA1312E81093BD1380E14D
:1097300093E1A0E0B0E08093BE139093BF13A09399
:10974000C013B093C1138AE693E10E94BC34109217
:10975000C7131092C61393CE121613060CF492C0C0
:1097600080916E1390916F13A0917013B09171134B
:109770008C34E0E19E07A105B10509F4D7C98A340C
:109780009041A105B10509F4D1C920E030E040E2E3
:1097900051E46091260C7091270C8091280C9091D7
:1097A000290C0F9446260F941C2E7093C7136093B8
:1097B000C61305E00093BA1312E81093BD1388E4B2
:1097C00090E1A0E0B0E08093BE139093BF13A0930C
:1097D000C013B093C1138AE693E10E94BC3420E029
:1097E00030E040E251E460912A0C70912B0C8091A2
:1097F0002C0C90912D0C0F9446260F941C2E7093D8
:10980000C7136093C6130093BA131093BD138AE471
:1098100090E1A0E0B0E08093BE139093BF13A093BB
:10982000C013B093C1138AE693E10E94BC3420E0D8
:1098300030E040E251E460912E0C70912F0C809149
:10984000300C9091310C0F9446260F941C2E70937F
:10985000C7136093C6130093BA131093BD138CE41F
:1098600090E1A0E0B0E056C9121613060CF01FCE2E
:10987000F8012F2D11922A95E9F710927E0510928A
:109880007D0515CE90916B1380910A14981321C019
:1098900090916C1380910B1498131BC023303105E9
:1098A000C4F090910C1490936A1380910D148093DE
:1098B0006D139330D1F4982F9D7F9038B1F490912F
:1098C0000E149F3409F059C090910F149B3409F085
:1098D00054C0EAE0F4E18AE1DF011D928A95E9F7DC
:1098E00010927E0510927D053BCF833809F045C06C
:1098F00080910E1490910F14982789279827B0E033
:10990000A0E080936E1390936F13A0937013B093A5
:109910007113C0901014D12CF12CE12CC092721351
:10992000D0927313E0927413F092751321E134E135
:1099300040E050E0BA014C155D056E057F0508F06A
:109940004AC0DB01CA01B695A795979587950696FB
:10995000880F991FFC01E659FC4ED9018C91119694
:109960009C91892798278927918380834E5F5F4F39
:109970006F4F7F4F2E5F3F4FDECF813861F5809173
:109980000E1490E0B0E0A0E080936E1390936F13FC
:10999000A0937013B093711380910F14482F50E06F
:1099A00070E060E0409372135093731360937413EC
:1099B00070937513A0E1B4E1E6E7F3E190E030E0E5
:1099C00020E08217930739F04D9150E04193519375
:1099D0002F5F3F4FF6CFEAE0F4E18AE1DF011D920D
:1099E0008A95E9F710927E0510927D050E94EEFDA2
:1099F000B7CE3F924F925F926F927F928F929F92DB
:109A0000AF92BF92CF92DF92EF92FF920F931F938C
:109A1000CF93DF938091370587FD38C0809138055B
:109A20008370A1F5C0918312D0918412488159812D
:109A30006A817B818BE197E10E9448414C815D8185
:109A40006E817F818BE79FE20E94484140917F12A7
:109A500050918012609181127091821288E79FE28A
:109A60000E9448418AE0DF91CF911F910F91FF90B2
:109A7000EF90DF90CF90BF90AF909F908F907F90AE
:109A80006F905F904F903F900C94333860907712B6
:109A9000709078128090791290907A12A0907B1238
:109AA000B0907C1200917D1210917E12C0907F12B6
:109AB000D0908012E0908112F090821288E50E948E
:109AC000CB1EC82F882309F49AC00E94D124362EB9
:109AD000472E582ED92F20E030E046E953EC0F9462
:109AE000102F87FD0DC020E030E046E953E4632DE0
:109AF000742D852D9D2F0F94E02518160CF081C034
:109B00006CE271E088E097E10E946A416CE271E0EA
:109B100083E097E10E946A4180E097E10E946C38FF
:109B2000C0E089E50E94CB1E882361F10E94D12408
:109B3000362E472E582ED92F20E030E046E953EC40
:109B40000F94102F87FD0DC020E030E046E953E46C
:109B5000632D742D852D9D2F0F94E02518160CF084
:109B600055C06CE271E08DEE96E10E946A416CE2B4
:109B700071E088EE96E10E946A4185EE96E10E94CE
:109B80006C38C0E08AE50E94CB1E882309F443C0EC
:109B90000E94D1246B017C0120E030E040E151ECD7
:109BA0000F94102F87FD0AC020E030E040E151E41F
:109BB000C701B6010F94E02518166CF567EF7FEF2B
:109BC00083ED96E10E946A4169E070E08EEC96E1D7
:109BD0000E946A418BEC96E1DF91CF911F910F912A
:109BE000FF90EF90DF90CF90BF90AF909F908F90BD
:109BF0007F906F905F904F903F900C946C38C1E0D5
:109C000090CF632C742C852C9D2E8BCFA32CB42C41
:109C1000052D1D2FB7CFCC23E1F0C301D4018093D4
:109C2000771290937812A0937912B0937A12C501AB
:109C3000D80180937B1290937C12A0937D12B093F5
:109C40007E12C0927F12D0928012E0928112F09226
:109C50008212DF91CF911F910F91FF90EF90DF90D3
:109C6000CF90BF90AF909F908F907F906F905F90BC
:109C70004F903F9008958FED97E00C946C3889EDEC
:109C800097E00C946C3884E690E09093C205809342
:109C9000C1051092E2051092E1050C94C1DBEF9230
:109CA000FF920F931F93CF93DF93CDB7DEB76297E9
:109CB0000FB6F894DEBF0FBECDBF0E944C2A88239A
:109CC00009F43FC049EE53E082FF02C04DEC53E07F
:109CD00029EE33E081FF02C02FEC33E080FD2EC07F
:109CE00089EE93E05F934F933F932F939F938F93CE
:109CF00085E499E19F938F938E010F5F1F4F1F9310
:109D00000F930F9477250E943F4EC8010E943A3866
:109D1000C8010E945EE40FB6F894DEBF0FBECDBF4F
:109D200081E062960FB6F894DEBF0FBECDBFDF9123
:109D3000CF911F910F91FF90EF90089581ED93E0E7
:109D4000D1CF80E0EECFCF92DF92EF92FF928AE503
:109D50000E94CB1E882309F45AC00E94D12420E01F
:109D600030E040E050EC0F94E025C12CD12CE12CE8
:109D700090ECF92E87FD0FC00E94D12420E030E046
:109D800040E050E40F94102F18160CF462C00E94AB
:109D9000D1246B017C012091540C3091550C4091E1
:109DA000560C5091570CC701B6010F9446260F94DC
:109DB0001C2ECB010E9477FD80E50E947D1E811143
:109DC0004EC0A701960160917F1270918012809120
:109DD0008112909182120F94B02C60937F12709335
:109DE000801280938112909382120E943F4E409184
:109DF0007F125091801260918112709182128CEBCF
:109E000096E10E9448418AE00E94333805C083E50C
:109E10000E94CB1E8111A1CF8091370587FD24C000
:109E200080913805837001F50E943F4E40917F126A
:109E30005091801260918112709182128DEA96E1A8
:109E40000E9448418AE0FF90EF90DF90CF900C9401
:109E50003338C12CD12CE12C80E4F82E9CCF0E9409
:109E600099248111AECFD8CF82E50E947D1E811149
:109E7000DBCFFF90EF90DF90CF900895CF9384E5F4
:109E80000E94CB1EC0E08823D9F00E947924C82FFD
:109E90001816B4F40E943F4E8DE40E94333880912E
:109EA0003205909133050E9412E26C2FCC0F770B94
:109EB00088EA9FE00E946A418AE00E943338CFEF2F
:109EC0008C2FCF9108954F925F926F927F928F92D5
:109ED0009F92AF92BF92CF92DF92EF92FF92CF9379
:109EE000DF93CDB7DEB72C970FB6F894DEBF0FBE69
:109EF000CDBF4090CE085090CF086090D0087090B1
:109F0000D108209147023091480240914902509176
:109F10004A02C301B2010F94B02C69837A838B8308
:109F20009C838090D2089090D308A090D408B090E1
:109F3000D50820914B0230914C0240914D02509136
:109F40004E02C501B4010F94B02C6D837E838F83C4
:109F50009887C090D608D090D708E090D808F090A5
:109F6000D90820914F0230915002409151025091F6
:109F70005202C701B6010F94B02C69877A878B878C
:109F80009C87209153023091540240915502509188
:109F90005602C301B2010F94B02C2B013C01209159
:109FA0005702309158024091590250915A02C5010E
:109FB000B4010F94B02C4B015C0120915B023091F5
:109FC0005C0240915D0250915E02C701B6010F94A0
:109FD000B02C6B017C010E943F4E83EE9EE00E94FC
:109FE0006C3883E50E947D1E882321F00E9499240D
:109FF0008093450280914502811151C08AEC9EE018
:10A000000E946C388BED9EE00E946C3849815A8129
:10A010006B817C8183E19EE10E9448414D815E819C
:10A020006F8178858BE79FE20E94484149855A8578
:10A030006B857C8588E79FE20E94484189ED9EE020
:10A040000E946C3881ED9EE00E946C38B301A20141
:10A0500083E19EE10E944841B501A4018BE79FE2A4
:10A060000E944841B701A60188E79FE20E9448414B
:10A070008AE02C960FB6F894DEBF0FBECDBFDF91FD
:10A08000CF91FF90EF90DF90CF90BF90AF909F90D7
:10A090008F907F906F905F904F900C9433388EEC40
:10A0A0009EE0AECF5F926F927F928F929F92AF921F
:10A0B000BF92CF92DF92EF92FF920F931F93CF93B5
:10A0C000DF931F92CDB7DEB77C0139018B015B01B5
:10A0D000A40EB51ED12CC12CA016B10609F450C097
:10A0E000F70180809180F80151908F015982C4015D
:10A0F0000F94FE2B5816B9F1652DC4010F94062C50
:10A10000FFEFCF1ADF0AC6018F779927892B21F13C
:10A1100062E070E080E090E00E940BFDC4010F94CB
:10A12000FE2B99818917F9F00E943F4E8FE694E04B
:10A130000E946C3881E00F90DF91CF911F910F91B9
:10A14000FF90EF90DF90CF90BF90AF909F908F9057
:10A150007F906F905F90089562E070E080E090E003
:10A160000E943F26DBCFBE016F5F7F4FC3010E947D
:10A17000E2E0F70180819181019691838083ACCFE9
:10A1800080E0D9CFDF92EF92FF920F931F93CF938E
:10A19000DF93CDB7DEB7CA5AD1090FB6F894DEBF48
:10A1A0000FBECDBFCF55DF4F188219821A821B8296
:10A1B000C15AD0408091D3039091D403A091D5038C
:10A1C000B091D603CB55DF4F88839983AA83BB8395
:10A1D000C55AD04084E690E09093C2058093C105B3
:10A1E0001092E2051092E1051092E30521EE35E0B0
:10A1F00044E050E0BE016B557F4F81EC95E00E943A
:10A2000052508091C1059091C20502969093C2056B
:10A210008093C1051092E2051092E10581E0C655D8
:10A22000DF4F8883CA5AD040CE0186559F4F0E9487
:10A23000E6D121EE35E048E450E068E37CE081ECD3
:10A2400095E00E94525021EE35E040E150E06BED88
:10A2500078E081EC95E00E9452508AE097EDA3EA05
:10A26000BCE3CF55DF4F88839983AA83BB83C15A50
:10A27000D040CE018F559F4F0E94DDD184E098E001
:10A280000E94F8D186E292E00E94EFD182E292E051
:10A290000E94DDD18091CA089091CB08A091CC0892
:10A2A000B091CD0889839A83AB83BC838E010F5F05
:10A2B0001F4FC8010E94DDD1CF55DF4F1882198290
:10A2C0001A821B82C15AD0407E018DE6E80EF11C35
:10A2D00083E0D7018C938983CE018F559F4F0E94D5
:10A2E000DDD1C7010E94E6D1C8010E94E6D14AE053
:10A2F000D42EDA94DD2031F0CE018F559F4F0E948D
:10A30000DDD1F7CF87E792E10E94F8D1CF55DF4F3B
:10A31000188219821A821B82C15AD0403AE0D32E89
:10A32000DA94DD2031F0CE018F559F4F0E94DDD1B0
:10A33000F7CF85E0D82ED982F701D082C8010E94DC
:10A34000E6D1C7010E94E6D121EE35E048E050E0B9
:10A3500064ED75E081EC95E00E94525021EE35E00D
:10A3600048E050E06CEC75E081EC95E00E945250C2
:10A3700021EE35E044E650E06EE877E081EC95E0D0
:10A380000E94525019828FEFD7018C93C8010E940E
:10A39000EFD1C7010E94E6D121EE35E044E050E064
:10A3A00064EE72E081EC95E00E9452508091A50627
:10A3B0008983C8010E94EFD1198A1A8A1B8A1C8AD4
:10A3C00080E090E0A0E8BFE38D879E87AF87B88BE1
:10A3D0008091EF119091F011A091F111B091F211D3
:10A3E00089839A83AB83BC832CEA35EC47E25EE336
:10A3F0006091F3117091F4118091F5119091F61123
:10A400000F94AA2D6D837E838F8398872CEA35EC79
:10A4100047E25EE36091F7117091F8118091F911B4
:10A420009091FA110F94462669877A878B879C87CB
:10A4300021EE35E044E150E0B80181EC95E00E9466
:10A44000525084E190E09A838983C8010E94CBD165
:10A450008091841190918511A0918611B0918711FE
:10A4600089839A83AB83BC832CEA35EC47E25EE3B5
:10A47000609188117091891180918A1190918B114E
:10A480000F94AA2D6D837E838F8398872CEA35ECF9
:10A4900047E25EE360918C1170918D1180918E1175
:10A4A00090918F110F94462669877A878B879C87B6
:10A4B000C8010E94D4D18CE0EBE7F2E0D801019012
:10A4C0000D928A95E1F7C8010E94D4D11982C80182
:10A4D0000E94E6D18FE790E09A838983C8010E94A9
:10A4E000CBD1E7E8F2E0D80101900D92DA94E1F7E0
:10A4F00021EE35E045E050E0B80181EC95E00E94A6
:10A5000052508091CB058983C8010E94EFD180E22F
:10A51000ECE8F2E0D80101900D928A95E1F721EE86
:10A5200035E040E250E0B80181EC95E00E945250E5
:10A53000F7011082C7010E94EFD187EF97E00E94D8
:10A54000EFD183EF97E00E94DDD1CF55DF4F188226
:10A5500019821A821B82C15AD040CE018F559F4F5B
:10A560000E94DDD180E2D8011D928A95E9F721EEA3
:10A5700035E040E250E0B80181EC95E00E94525095
:10A58000FE01F99688E0DF011D928A95E9F744E61D
:10A5900050E060E070E049835A836B837C834D8395
:10A5A0005E836F83788783E090E0A0E0B0E08987E6
:10A5B0009A87AB87BC874D875E876F87788B498B7F
:10A5C0005A8B6B8B7C8B8D8B9E8BAF8BB88F898FCF
:10A5D0009A8FAB8FBC8F8D8F9E8FAF8FB8A38EE17C
:10A5E00090E0A0E0B0E089A39AA3ABA3BCA38DA3A5
:10A5F0009EA3AFA3B8A789A79AA7ABA7BCA78DA70F
:10A600009EA7AFA7B8AB89AB9AABABABBCAB8DABDE
:10A610009EABAFABB8AF21EE35E040E450E0B801FF
:10A6200081EC95E00E94525090E1D92EF8018D2DD9
:10A6300011928A95E9F721EE35E040E150E0B8014A
:10A6400081EC95E00E945250D8011D92DA94E9F70E
:10A6500021EE35E040E150E0B80181EC95E00E9448
:10A660005250CF55DF4F188219821A821B82C15A6D
:10A67000D040CE018F559F4F0E94DDD12CE0D22ECD
:10A68000F8018D2D11928A95E9F721EE35E04CE025
:10A6900050E0B80181EC95E00E9452508CE6D80160
:10A6A0001D928A95E9F721EE35E04CE650E0B801BD
:10A6B00081EC95E00E94525085EB95E00E94D4D148
:10A6C00021EE35E048E050E063EC75E081EC95E088
:10A6D0000E945250F7011192DA94E9F7C755DF4F03
:10A6E0001882C95AD04080E090E0A0E4B0E4C3569C
:10A6F000DF4F88839983AA83BB83CD59D040C7019C
:10A700000E94F8D1CE0187559F4F0E94E6D1CE011D
:10A7100083569F4F0E94DDD180E3D7011D928A9519
:10A72000E9F78FE89CE10E946C388AE00E94333898
:10A7300021EE35E040E350E0B70181EC95E00E9466
:10A7400052508091E305811128C00091C1051091FC
:10A75000C2058091E1059091E205F7019183808324
:10A7600084E690E09093C2058093C10521EE35E028
:10A7700044E050E064EF72E081EC95E00E945250BA
:10A78000C7010E94CBD191E00536134009F490E057
:10A790008091E305892B8093E3058091E305811186
:10A7A00005C060E083EC9CE10E94DA3F83EA9CE113
:10A7B0000E946C388AE00E9433389091E30581E072
:10A7C0008927C655DF4F0FB6F894DEBF0FBECDBF49
:10A7D000DF91CF911F910F91FF90EF90DF9008953F
:10A7E000CF93DF9300D01F92CDB7DEB78091910653
:10A7F0008823C1F083E390E09C838B831A821982C3
:10A800009E012F5F3F4F40E150E062E976E0CE01CC
:10A8100003960E94525083EA9CE10E946C388AE0C1
:10A820000E9433380F900F900F900F90DF91CF91CF
:10A830000895CF92DF92EF92FF92CF93C82F80912D
:10A8400023118150823008F069C00E94CF3A1092E3
:10A8500023110E943EFD6093AD057093AE05809379
:10A86000AF059093B005C090B105D090B205E090CF
:10A87000B305F090B4050E94B32BAB01BC0140932B
:10A88000B1055093B2056093B3057093B405809100
:10A89000960690919706A0919806B09199068C190A
:10A8A0009D09AE09BF09840F951FA61FB71F80938E
:10A8B000960690939706A0939806B0939906C111B7
:10A8C0000AC0C1E00E94F0538C2FCF91FF90EF900F
:10A8D000DF90CF900895809194069091950601960F
:10A8E00090939506809394060E94B32BC0909A068D
:10A8F000D0909B06E0909C06F0909D06C616D70669
:10A90000E806F906F0F60E94B32B60939A0670935E
:10A910009B0680939C0690939D06D3CFC0E0D2CF38
:10A9200081E00C9419540E94EDBE0E94905480E086
:10A930000E940DF98091E7068130A1F40E943B4E00
:10A9400082E697E00E946C3860E088E597E00E941C
:10A95000DA3F6EE571E080E090E00E943F2688E0FB
:10A960008093E7060895CF92DF92EF92FF921F93B4
:10A97000CF93DF9300D01F92CDB7DEB78EEEC82EF7
:10A9800082E0D82EE12CF12CC982DA82EB82FC82A3
:10A99000BE016F5F7F4F8AE50E949E3381110EC01A
:10A9A00010E0812F0F900F900F900F90DF91CF91BB
:10A9B0001F91FF90EF90DF90CF9008950E94F433A5
:10A9C000C982DA82EB82FC82BE016F5F7F4F8AE52B
:10A9D0000E949E33182F882319F30E943B4E8CE36C
:10A9E00098E00E946C380E949354DBCFCF92DF92A4
:10A9F000EF92FF921F93CF93DF9300D01F92CDB7BA
:10AA0000DEB78EEEC82E82E0D82EE12CF12CC98262
:10AA1000DA82EB82FC82BE016F5F7F4F8AE00E9488
:10AA20009E3381110EC010E0812F0F900F900F9078
:10AA30000F90DF91CF911F91FF90EF90DF90CF901B
:10AA400008950E94F4330E94BE330E94D9330E94BD
:10AA5000BE33C982DA82EB82FC82BE016F5F7F4F18
:10AA60008AE00E949E33182F8823E9F20E943B4E11
:10AA70008FEF97E00E946C380E949354D5CFCF930C
:10AA8000DF9300D01F921F92CDB7DEB781E0809395
:10AA9000910680E1E2E9F6E0DF011D928A95E9F78F
:10AAA0000E94F05386E18D8382E390E09C838B8348
:10AAB0001A8219829E012F5F3F4F41E050E0BE0194
:10AAC0006B5F7F4FCE0103960E9452500F900F9004
:10AAD0000F900F900F90DF91CF910895CF93DF9358
:10AAE000CDB7DEB7A8970FB6F894DEBF0FBECDBFC7
:10AAF0008C01F42E0E94EDBE0E943B4E88E397E04D
:10AB00000E946C380115110511F40FE217E08091D5
:10AB1000870580FD79C08160809387058BE197E090
:10AB20000E946C388AE00E943338CC24C3948AE5B2
:10AB3000D82ED092C713C092C6138FE090E09093A6
:10AB4000C9138093C81397E0792E7092BA1322E844
:10AB5000E22EE092BD1334E8832E912CA12CB12C6F
:10AB60008092BE139092BF13A092C013B092C113F3
:10AB70008AE693E10E94BC34D092C713C092C613F8
:10AB800088E590E09093C9138093C8137092BA132C
:10AB9000E092BD138092BE139092BF13A092C01397
:10ABA000B092C1138AE693E10E94BC348AE28983A1
:10ABB0008A838B838C83F801DE011596BE016F5F5B
:10ABC0007F4FCD01861B970B2491319621110CC02C
:10ABD000FB01E80FF91F8AE29F01261B370B283281
:10ABE000310524F48193F8CF2D93EBCF20E630E1AB
:10ABF00040E050E08AE693E10E94FDE06AE070E008
:10AC000080E090E00E94C62C61E086E297E00E941E
:10AC1000A73F89EE93E030E6019729F0232F2A958C
:10AC20000000E9F7F9CFF89489EE93E038EE019748
:10AC300029F0232F2A950000E9F7F9CF0E94EDBEF5
:10AC4000FF2031F00E94371F0E94501FA895FECFB1
:10AC50000E94351FF9CF8091E606882319F01092E3
:10AC6000E606089540E070E060E086EB98E10E941F
:10AC70006E558091A30C9091A40C2FEF3FEF981785
:10AC800051F0E92FF0E0ED55F34F228130E09F5F66
:10AC90009F779093A40CC90108951F920F920FB64D
:10ACA0000F9211240F900FBE0F901F9018951F92B6
:10ACB0000F920FB60F9211240BB60F920F931F93A2
:10ACC0002F933F934F935F936F937F938F939F93B4
:10ACD000AF93BF93CF93DF93EF93FF93C091C600E1
:10ACE0000091A40CD091A30C11E01D0F1F7790913F
:10ACF0001504913108F09FC0E92FF0E08827EC5748
:10AD0000F94A8F4F0D94A72C9556C456D356E25648
:10AD1000E9561B57ED561B57F156F5561B57F9567A
:10AD2000FD56015708571B571357C03229F028F515
:10AD3000CA3011F0CD3031F5011731F0ED2FF0E0D0
:10AD4000ED55F34FC283D12FD093A30CFF91EF9118
:10AD5000DF91CF91BF91AF919F918F917F916F9133
:10AD60005F914F913F912F911F910F910F900BBECB
:10AD70000F900FBE0F901F901895CD3481F081E099
:10AD8000CE3471F080E10CC0CA3338F4C033A0F681
:10AD9000C03291F2CD32B1F7CFCFCD3499F782E006
:10ADA00080931504C9CFC13359F018F4C03221F291
:10ADB000E9CF88E0C433A1F38BE0C83389F3E2CF55
:10ADC00083E0EECF84E0C03359F386E0C13341F332
:10ADD000D9CF85E0C833B1F6E3CF87E0C23391F62F
:10ADE000DFCF89E0C13371F6DBCF8AE0C03351F6A3
:10ADF000D7CF8CE0C73331F6D3CF8DE0C63311F611
:10AE0000CFCFC03209F498CF8EE0C33549F2BACF24
:10AE100080ED8C0F8A3008F08FCF9FE0909315045F
:10AE20008093160489CFCA3019F0CD3009F084CF51
:10AE30001092150481CFCA3019F0CD3009F07CCFC3
:10AE4000809124148823A1F3973089F038F4953049
:10AE500079F710923C021092250CEACF9A3059F003
:10AE60009F3031F7809116040E94DB31E1CF81E001
:10AE700080930F06DDCF81E080930E06D9CF8EBD83
:10AE80000DB407FEFDCF08958FEF8EBD0DB407FE04
:10AE9000FDCF8EB50895909164009B7F90936400E0
:10AEA000982F906A96959CBD80FD03C091E08630F6
:10AEB00009F490E09DBD0895CF93DF93EB010E94CC
:10AEC0006C38CE01DF91CF910C9437AF2F923F9227
:10AED0004F925F926F927F928F929F92AF92BF92AA
:10AEE000CF92DF92EF92FF920F931F93CF93DF9356
:10AEF000009709F0AAC11092880C1092870C9093C9
:10AF0000860580938505BAE0CB2EB0E2DB2EE12CDE
:10AF1000F12C15E002E846015701C4E1D0E010929F
:10AF20000D1310920C1310930013009303138092CF
:10AF3000041390920513A0920613B092071380EBAE
:10AF400092E10E94BC3421972FEF821A920AA20A42
:10AF5000B20A209721F744E1C40ED11CE11CF11C78
:10AF60008AE5C81680E2D806E104F104A1F6C12CF6
:10AF7000A0E2DA2EE12CF12CD5E0C2E810920D13FC
:10AF800010920C13D0930013C0930313C0920413B8
:10AF9000D0920513E0920613F092071380EB92E132
:10AFA0000E94BC3410920D1310920C13D093001316
:10AFB000C0930313D701C6018C529F4FAF4FBF4FB1
:10AFC0008093041390930513A0930613B093071373
:10AFD00080EB92E10E94BC34EFEFCE1ADE0AEE0A5B
:10AFE000FE0AFAE0CF16F0E2DF06E104F10431F6E2
:10AFF000FEEDCF2EF0E2DF2EE12CF12CD5E0C2E801
:10B0000010920D1310920C13D0930013C0930313DE
:10B01000C0920413D0920513E0920613F092071326
:10B0200080EB92E10E94BC342FEFC21AD20AE20AEE
:10B03000F20A46EEC41640E2D406E104F10401F738
:10B04000CC24C394E2E1DE2EE12CF12C0AE010E0E6
:10B05000D5E0C2E810930D1300930C13D0930013A6
:10B06000C0930313C0920413D0920513E092061309
:10B07000F092071380EB92E10E94BC3410930D1301
:10B0800000930C13D0930013C0930313D701C60190
:10B090008096A11DB11D8093041390930513A09376
:10B0A0000613B093071380EB92E10E94BC348FEF3C
:10B0B000C81AD80AE80AF80AE5E0CE16E2E1DE0688
:10B0C000E104F10439F60091870C1091880C011508
:10B0D000110509F0D6C08091860C882309F4E1C0DF
:10B0E0002AE030E240E050E067ED73E080EB92E16F
:10B0F0000E94FDE0C1E0D0E003E010E0E090870CAA
:10B10000F090880C35E0332E42E8242E44244A94F3
:10B11000542C64E0662E712C7FE1C72E74E0D72E8C
:10B120008091870C9091880C800F911FE816F9068A
:10B1300008F0D5C0C7010E9418E2882309F481C035
:10B1400080919E1161E971E1882311F06EE971E14E
:10B15000FB0101900020E9F7CF010197861B970BB7
:10B16000F4E1FC9F9001FD9F300D1124265F3F4DBF
:10B1700050E040E0459710F0FB01128A80EB92E12D
:10B180000E94FDE0CE018F5F9D4EB0E0A0E02196D1
:10B190004E0124E0880C991C2A95E1F7FDEF8F1AE7
:10B1A000FFE99F0AB12CA12C2091301424FF7EC00E
:10B1B00070920D1360920C133092001320920313BF
:10B1C0008093041390930513A0930613B093071371
:10B1D00080EB92E10E94BC34D0920D13C0920C130C
:10B1E000309200132092031380920413909205135F
:10B1F000A0920613B092071380EB92E10E94BC3438
:10B20000B7018BE498E10E94364180919E116EE96E
:10B2100071E1811102C061E971E188E498E10E9465
:10B220005C5765EE7BE084E498E10E945C5761E93D
:10B2300071E183E498E10E945C578FE398E10E94FA
:10B240006C382FEFE21AF20A6BCF2091870C309105
:10B25000880CA901415051096091850570918605BE
:10B260006817790738F42C5F3F4F3093880C209390
:10B27000870C45CE4430510508F43DCE24503109A9
:10B28000F4CF0430110569F48091860C882331F0E5
:10B2900083E090E09093880C8093870CD0E0C0E02E
:10B2A0002DCFD0E0C0E004E010E028CF10920D13C5
:10B2B00010920C1330920013209203138093041306
:10B2C00090930513A0930613B093071380EB92E1BC
:10B2D0000E94BC3450920D1340920C1381CFDF9129
:10B2E000CF911F910F91FF90EF90DF90CF90BF9083
:10B2F000AF909F908F907F906F905F904F903F9016
:10B300002F900895AF92BF92CF92DF92EF92FF926B
:10B310000F931F93CF93DF93CDB7DEB7E6970FB6AA
:10B32000F894DEBF0FBECDBF0091390510913A05EC
:10B33000F80101900020E9F731976F01C01AD10A96
:10B34000F801CF01801B910B8C159D053CF4819178
:10B350008F32B9F7DF0111971C92F3CF8BE1E0E553
:10B36000F4E1DE015C9601900D928A95E1F7F12CF3
:10B37000E12CEC14FD040CF05DC0F801EE0DFF1D96
:10B380008081811103C08FEFE81AF80A5801AE0CD2
:10B39000BF1CF5018081882309F44CC0FFEFEF1A30
:10B3A000FF0AF801EE0DFF1D7F01E01AF10A8191FD
:10B3B0008111FACFCE014C960E94CAB38BE1FE01F7
:10B3C0007C96DE01119601900D928A95E1F7B50108
:10B3D000CE0101960E94D8ABCE0101960E94C82FE3
:10B3E0008FE20E94333880919E1181113BC084EE20
:10B3F00093E00E9437AF8091301484FF1BC0198204
:10B400001C8221E0A501BE01645E7F4FCE01019642
:10B410000E940CB6811129C08AE00E9433380E9434
:10B420003F4EB5018AE297E10E945C57CE0101963A
:10B430000E94C82F8AE00E943338CE014C960E94A9
:10B44000C82FE6960FB6F894DEBF0FBECDBFDF91D2
:10B45000CF911F910F91FF90EF90DF90CF90BF9011
:10B46000AF9008958EE991E1C4CFCE014C960E9431
:10B4700039B38BE1FE013196DE015C9601900D92AD
:10B480008A95E1F7CE0101960E94C82F72CF2F92C4
:10B490003F924F925F926F927F928F929F92AF9264
:10B4A000BF92CF92DF92EF92FF920F931F93CF93B1
:10B4B000DF9300D000D000D01F921F92CDB7DEB72F
:10B4C000B82E8091900D843008F0D1C10E943EFDCD
:10B4D0006B017C018091900D811108C08091A30CBB
:10B4E0009091A40C891B8F7709F4A4C681E6A82E3D
:10B4F00013C08A3019F08D3009F0F6C010928B0D10
:10B500008091290D90912A0DFC01EB5DF24F16827E
:10B51000892BF1F40E943AC28091900D843008F09A
:10B52000ECC08091A30C9091A40C891B8F7709F437
:10B53000E4C00E94395697FFDCCF0E943B4E85EB5A
:10B5400095E00E946C388091A30C8093A40CE4CF0A
:10B5500010922A0D1092290D0BE21DE0F801819145
:10B56000803209F446C08E3409F0A9C060EB75E062
:10B57000C8010F945D254C01892B41F06EE470E009
:10B58000C80104960F94FE2F009709F4C8014AE001
:10B5900050E070E060E001960F94CD222B013C0159
:10B5A0008091250D9091260DA091270DB091280D29
:10B5B0000196A11DB11D481659066A067B0629F0A1
:10B5C00060E08DE795E0892851F16AE270E0C801FA
:10B5D0000F942D309C01009729F1982F901B912CEE
:10B5E000992349F09150F801E90FF11D80819826C7
:10B5F000F7CF8F01B3CF4AE050E070E060E0C901BF
:10B6000001960F94CD22292D30E050E040E06217E2
:10B6100073078407950751F060E08EE595E00E947E
:10B6200093E77ACF60E084E395E0F9CF4092250D6F
:10B630005092260D6092270D7092280D8091E7069A
:10B640008130E1F067E470E0C8010F94FE2F0097AD
:10B65000A9F04AE050E070E060E001960F94CD223E
:10B66000643071058105910548F483E994E00E94F6
:10B670006C3860E089E894E00E94DA3FC092860767
:10B68000D0928707E0928807F092890780912B0D6E
:10B690008B3309F441CF8091900D843008F03CCF7A
:10B6A0008091920D8A9DC00111246BE27DE08D5640
:10B6B000924F0F94093080E00E944DE72DCF80918A
:10B6C000301480FFBBCF6EE97DE2C8010F945D2589
:10B6D000009731F0FC01838180538A3008F0AECFAF
:10B6E00060E08AE095E09BCF29E23DE04BE25DE03F
:10B6F0006BE87DE00E944B1D0FCF8091301482FFDC
:10B70000B6C01A82198271E6F72EE0E1EE2EF9E654
:10B71000DF2E8091900D843008F0A9C00E94831D17
:10B720008111A5C041E050E0BE016B5F7F4F84E90D
:10B7300095E10E948CB10D8110E0019711F00FEF9F
:10B740001FEF80919C1590919D15A0919E15B09131
:10B750009F1580932C1490932D14A0932E14B093C6
:10B760002F140E94831D0F3F100749F4811107C059
:10B770000E943B4E83ED95E00E946C38CACF409109
:10B78000920D242F30E00A3061F00D3051F0882303
:10B7900009F45FC089819A81009719F001969A8314
:10B7A000898310929C0489819A81F29EF001F39E14
:10B7B000F00D1124E057F24FE80FF91F1382892B87
:10B7C00069F50E943AC20E94831D882309F4A1CF23
:10B7D0000E94B16184E995E10E9439B380912714F8
:10B7E000882391F18150809327148D9DC0011124ED
:10B7F00062E0815E994F0E948EB8E091271424E0A8
:10B80000E29FF0011124E55EF94F60817181828130
:10B8100093810E949C220E9441AB7BCF1A821982A5
:10B8200081E00E944DE780912C1490912D14A091FD
:10B830002E14B0912F1480938C0D90938D0DA093A6
:10B840008E0DB0938F0DBFCF0E9442B3E092E706FA
:10B8500060CF4F9DA00111244D56524F9E012F5F86
:10B860003F4F6CE974E0802F0E944B1D52CF0E9425
:10B870003EFD6B017C01B11004C080912211882330
:10B8800051F0C0927511D0927611E0927711F0923A
:10B890007811BB24B3948091110590911205A09169
:10B8A0001305B09114050097A105B105B1F04091C1
:10B8B0007511509176116091771170917811840F04
:10B8C000951FA61FB71FA7019601281B390B4A0B0E
:10B8D0005B0BDA01C901B7FF92C18091130290910D
:10B8E0001402A0911502B0911602892B8A2B8B2B82
:10B8F00009F099C10E943EFD4B015C018091250C2D
:10B90000811108C0209188129091891281E0291339
:10B9100001C080E02091EA113091EB1191E089277C
:10B920002A3A31050CF480E091E04091A104509155
:10B93000A2046091A3047091A404452B462B472BCD
:10B9400009F490E0981789F0882309F4BDC1D50166
:10B95000C40180569444A24FBF4F8093A10490939A
:10B96000A204A093A304B093A4044090320C50907E
:10B97000330C6090340C7090350C20919D04309104
:10B980009E0440919F045091A004C301B2010F9402
:10B99000E025882319F18091A1049091A204A0913F
:10B9A000A304B091A40440929D0450929E0460921E
:10B9B0009F047092A004892B8A2B8B2B09F449C019
:10B9C000D501C40180569444A24FBF4F8093A10477
:10B9D0009093A204A093A304B093A4048091A10423
:10B9E0009091A204A091A304B091A4040097A10592
:10B9F000B10579F1881A990AAA0ABB0AB7FC29C0CD
:10BA00001092A1041092A2041092A3041092A40414
:10BA100083E396E00E946C3860E08FE196E00E943C
:10BA2000DA3F8091EC119091ED111816190624F46B
:10BA300090E080E00E94531F8091811190918211CB
:10BA40001816190634F410928211109281110E9476
:10BA5000C0BE8091A9049091AA04A091AB04B091BA
:10BA6000AC0446015701881A990AAA0ABB0AD501F3
:10BA7000C401B7FDB9C120918812909189124091FB
:10BA80002D0280912C02291323C19091FF08899FD8
:10BA9000C0011124880F892F881F990B91958D83E0
:10BAA00080910009489FC0011124880F892F881FA9
:10BAB000990B91958E830E943EFD69837A838B83D7
:10BAC0009C8340E0BE016F5F7F4FCE0105960E94D0
:10BAD0009D1C6D8170E089E00E9435FC41E0BE0153
:10BAE0006F5F7F4FCE0105960E949D1C6E8170E0B6
:10BAF00087E00E9435FC80911A06882309F467C10B
:10BB00000091200210912102C80102972091EC11AE
:10BB10003091ED11281739070CF459C18090891222
:10BB20008F82188619861A861B86809188129F80BC
:10BB3000891509F4E7C0892D90E03CE5A32EA89E65
:10BB4000F001A99EF00D1124EC5FF64F458956894E
:10BB50006789708D452B462B472B81F4418D528D83
:10BB6000638D748D452B462B472B41F4458D568DA7
:10BB7000678D70A1452B462B472BE1F12CE5B22EAA
:10BB8000B89E9001B99E300D1124A9014C5F564F0B
:10BB90001A01FA0161817281838194810F945E2F71
:10BBA0004B015C01F10161A172A183A194A10F94E9
:10BBB000E5252B013C01F10165A176A187A190A5A6
:10BBC0000F94E5259B01AC01C301B2010F94AA2D8E
:10BBD000A50194010F9446264B015C012885398507
:10BBE0004A855B850F94102F181624F48886998651
:10BBF000AA86BB868F818F5F87708F8396CF0E94C6
:10BC00003B4E609184077091850782EE95E00E941B
:10BC10005C578AE00E94333840E070E060E090E0DA
:10BC200080E00E946E559091881280918912981739
:10BC300049F0C0927511D0927611E0927711F0928E
:10BC4000781158CEBB2019F01092AD0453CE0E944B
:10BC50003EFD009175111091761120917711309170
:10BC600078118090130290901402A0901502B09069
:10BC70001602080D191D2A1D3B1D601B710B820B3E
:10BC8000930B97FDE1CF8091AD04811133CE81E01C
:10BC90008093AD045F9A8091360C8E7F8093360C32
:10BCA0008A9A8091360C8D7F8093360C80910801A2
:10BCB00080958170809306018091360C8B7F8093F4
:10BCC000360C0E94351F16CE80E090E0DC0145CE98
:10BCD000209189125CE5259F900111242C5F364F3D
:10BCE000F901EA5AFF4F9081899FC0011124880F02
:10BCF000892F881F990B91958D83295A3F4FF90100
:10BD00008081D0CE20911A0230911B0240911C02FA
:10BD100050911D02688579858A859B850F944626FA
:10BD20004B015C01B801012E000C880B990B0F949C
:10BD3000E7259B01AC01C501B4010F94B02C6983C8
:10BD40007A838B839C8340911E0250911F02B8011D
:10BD5000CE0101960E94F8C189809A80AB80BC8098
:10BD60004090A5045090A6046090A7047090A80489
:10BD7000A3019201C501B4010F94E02587FF16C00D
:10BD800028E431EE4AE75FE3C301B2010F9446268F
:10BD900020E037ED43EA5CE30F94B02CA501940159
:10BDA0000F94462669837A838B839C8369817A8189
:10BDB0008B819C816093A5047093A6048093A70453
:10BDC0009093A8040F941C2ECB010E94531FF4E6FD
:10BDD000CF0ED11CE11CF11CC092A904D092AA0480
:10BDE000E092AB04F092AC040E943AC28091E70664
:10BDF000882309F4E0C180912602882309F4A3C0B6
:10BE00008091EB0481119FC080912211811108C0A3
:10BE100080912311813021F08091301482FF93C0F2
:10BE2000F894649B10C08091220290912302A0910B
:10BE30002402B09125028093E8059093E905A09330
:10BE4000EA05B093EB056091E8057091E9058091F2
:10BE5000EA059091EB05789420E030E0A9010F9479
:10BE6000E02587FF70C001E00093EB048091221170
:10BE7000811167C088E496E00E946C388AE00E94D5
:10BE8000333884E080939D0C82E08093890C81E0BC
:10BE90009AE59093C7138093C6138EE490E0909335
:10BEA000C9138093C81387E08093BA1382E8809304
:10BEB000BD1384E890E0A0E0B0E08093BE139093BF
:10BEC000BF13A093C013B093C1138AE693E10E94FD
:10BED000BC340E9457400093901140E36CE876E038
:10BEE00084E799E00E945C4061E088E699E00E9466
:10BEF0003E401091150560E010278CE399E069F44D
:10BF00008AE796E00E94A73F80E30E9433388AE0E8
:10BF10000E94333860E08DE596E00E94A73F88E6F6
:10BF200096E00E946C3880E30E9433388AE00E94D9
:10BF30003338112331F083E696E09093850C80939B
:10BF4000840C0E94B16190910901892F80958170C4
:10BF5000109100021817C9F020913014206220932C
:10BF600030148093000290FD3FC164EF71E080E0E7
:10BF700090E00E943F260E9464B38091301483FDBC
:10BF80007CC1111133C10E9401360E943EFD6B013C
:10BF90007C01109117021123F1F08091160588237E
:10BFA000D1F04091AE045091AF046091B004709113
:10BFB000B10446015701841A950AA60AB70AB501C9
:10BFC000A40177FD1AC0833009F42FC10CF01EC103
:10BFD00081300CF023C1212F30E0A8EEB3E00F94A4
:10BFE000782CC60ED71EE81EF91EC092AE04D09261
:10BFF000AF04E092B004F092B1048091231181303B
:10C0000009F073C00E943EFD6B017C018091B60473
:10C010009091B704A091B804B091B904A70196011A
:10C02000281B390B4A0B5B0BDA01C901B7FD3AC07B
:10C03000D701C601805F984DAF4FBF4F8093B604C4
:10C040009093B704A093B804B093B9048090B1055D
:10C050009090B205A090B305B090B4050E94B32BA8
:10C06000AB01BC014093B1055093B2056093B30599
:10C070007093B4058091960690919706A0919806CA
:10C08000B091990688199909AA09BB09840F951FCF
:10C09000A61FB71F8093960690939706A0939806C5
:10C0A000B09399068091B2049091B304A091B40426
:10C0B000B091B50446015701881A990AAA0ABB0A29
:10C0C000D501C401B7FD11C020E8C20E2EEED21E6C
:10C0D00026E3E21EF11CC092B204D092B304E092B7
:10C0E000B404F092B5040E94F0530E94AA390E9451
:10C0F000744180911005882379F10E943EFD6B0107
:10C100007C0180910C0590910D05A0910E05B091D8
:10C110000F0546015701881A990AAA0ABB0AD501D8
:10C12000C401B7FD19C02091100530E0A8EEB3E0BE
:10C130000F94782CC60ED71EE81EF91EC0920C056F
:10C14000D0920D05E0920E05F0920F0580E00E945E
:10C150001EBB8AE00E94333880910B05882359F179
:10C160000E943EFD6B017C018091070590910805BE
:10C17000A0910905B0910A05A7019601281B390B6A
:10C180004A0B5B0BDA01C901B7FD15C020910B0505
:10C1900030E0A8EEB3E00F94782CC60ED71EE81E50
:10C1A000F91EC0920705D0920805E0920905F092A9
:10C1B0000A050E94FFAA2B960FB6F894DEBF0FBEA9
:10C1C000CDBFDF91CF911F910F91FF90EF90DF9046
:10C1D000CF90BF90AF909F908F907F906F905F9027
:10C1E0004F903F902F9008950E9453B3123008F063
:10C1F000CCCE0E94013660E085EC96E056C083ED1F
:10C2000096E09093850C8093840CBFCE843009F027
:10C21000E2CE0E943F4E8AED96E004C00E943F4E5F
:10C2200089E097E00E946C38D6CE0E943F4E82EFA4
:10C2300096E0F8CF8091860790918707A0918807B4
:10C24000B0918907A7019601281B390B4A0B5B0B9C
:10C25000DA01C901885E9340A109B109B7FD46C959
:10C260008DEC95E00E946C38C0928607D0928707CB
:10C27000E0928807F092890739C91230C8F48DE935
:10C2800096E00E946C388AE00E9433380E94E12CCC
:10C2900090E080E00E9466571092A10C1092A00CD2
:10C2A00010929F0C60E086EB96E00E94DA3F6DCE24
:10C2B000123009F06ACE0E94BEB7882379F081E07F
:10C2C0000E9494B742EB50E060E178E085E394E1AE
:10C2D0000E948CB185E394E10E9439B30E94B62F8D
:10C2E00081118DCF0E94A02F0E943AB80E948FB773
:10C2F0004CCECF93DF938091881290918912891B45
:10C300008095877019F40E94475AF5CF8091881262
:10C310008F5F8770A09188129CE5A99FD00111249E
:10C32000FD01EC5FF64FEF0119929A95E9F798E05D
:10C330009083A75EB64F90E1EAE8F2E101900D929A
:10C340009A95E1F72091881290918912291303C0E0
:10C3500094E69093851280938812DF91CF910C948C
:10C36000CE2F9091881280918912981306C08091E7
:10C37000020990910309892B21F080E00E94475A1D
:10C38000F0CF0895FC012081318142815381609179
:10C39000580C7091590C80915A0C90915B0C0F9431
:10C3A00046260F941D2F60939612709397128093D8
:10C3B00098129093991290918812809189129813F3
:10C3C0000C9479610E94B1610E943F2A40919612BB
:10C3D00050919712609198127091991240930A06A9
:10C3E00050930B0660930C0670930D0681110C940C
:10C3F000CE2F08954F925F926F927F928F929F926D
:10C40000AF92BF92CF92DF92EF92FF920F931F9362
:10C41000CF93DF93EC018B015A01F9012091580C65
:10C420003091590C40915A0C50915B0C6081718194
:10C43000828193810F9446260F941D2F6B017C01FE
:10C440002091540C3091550C4091560C5091570C42
:10C45000F50160817181828193810F9446260F944A
:10C460001D2F4B015C012091500C3091510C4091DB
:10C47000520C5091530CF80160817181828193813B
:10C480000F9446260F941D2F2B013C0120914C0C3C
:10C4900030914D0C40914E0C50914F0C6881798138
:10C4A0008A819B810F9446260F941D2F60938A12D8
:10C4B00070938B1280938C1290938D1240928E12F7
:10C4C00050928F12609290127092911280929212FA
:10C4D00090929312A0929412B0929512C0929612DA
:10C4E000D0929712E0929812F0929912909188123D
:10C4F00080918912981791F0DF91CF911F910F9140
:10C50000FF90EF90DF90CF90BF90AF909F908F9073
:10C510007F906F905F904F900C9479610E94B16111
:10C520000E943F2A4091921250919312609194126E
:10C530007091951200918E1210918F12209190128D
:10C5400030919112C0908A12D0908B12E0908C1290
:10C55000F0908D12C092FE05D092FF05E092000689
:10C56000F09201060093020610930306209304063E
:10C57000309305064093060650930706609308061D
:10C5800070930906409196125091971260919812FB
:10C590007091991240930A0650930B0660930C0613
:10C5A00070930D06882391F0DF91CF911F910F9129
:10C5B000FF90EF90DF90CF90BF90AF909F908F90C3
:10C5C0007F906F905F904F900C94CE2FDF91CF9122
:10C5D0001F910F91FF90EF90DF90CF90BF90AF90A1
:10C5E0009F908F907F906F905F904F9008953F92B3
:10C5F0004F925F926F927F928F929F92AF92BF9273
:10C60000CF92DF92EF92FF920F931F93CF93DF931E
:10C61000CDB7DEB768970FB6F894DEBF0FBECDBFBB
:10C62000D82E2A013B01480159013E2C20E030E080
:10C63000A901C501B8010F94E025811110C081E066
:10C640008D1508F0B6C060E070E080E793E420E06C
:10C6500030E040E752E40F94AA2D4B015C018D8A33
:10C660009E8AAF8AB88E0D2D10E0F801E056F64E86
:10C67000E491BB24B3941E160CF4B12CCC24C394C7
:10C6800020E030E0A901C301B2010F94102F181669
:10C690000CF0C12CBC1471F092E0D9120BC0332005
:10C6A00049F081E00E940DF969E170E080E090E0DE
:10C6B0000E943F2680E00E94D42F69837A838B8377
:10C6C0009C8381E00E94D42F6D837E838F83988723
:10C6D00082E00E94D42F69877A878B879C8783E0CA
:10C6E0000E94D42F6D877E878F87988B000F111F34
:10C6F000000F111FE1E0F0E0EC0FFD1F0E0F1F1FF8
:10C70000F80110821182128213829E01235F3F4F33
:10C71000AE01475F5F4FBE016B5F7F4FCE01019659
:10C720000E94FA61F8014082518262827382198A02
:10C730001A8A1B8A1C8A8091020990910309892B0D
:10C7400091F4CE0141967C018E010B5E1F4F9E013C
:10C75000235F3F4FAE01475F5F4FBE016B5F7F4F6F
:10C7600040970E94B7E70E94B161BC1451F092E07B
:10C77000D91205C0332019F080E00E940DF90E9403
:10C780002B5668960FB6F894DEBF0FBECDBFDF9173
:10C79000CF911F910F91FF90EF90DF90CF90BF90BE
:10C7A000AF909F908F907F906F905F904F903F9051
:10C7B000089560E070E88BE395E449CF4F925F9273
:10C7C0006F927F928F929F92AF92BF92CF92DF92A1
:10C7D000EF92FF920F931F93CF93DF93CDB7DEB706
:10C7E0002C970FB6F894DEBF0FBECDBF2B013C01D6
:10C7F00029873A874B875C8747015801F601E0801B
:10C80000F1800281138120E030E0A901B701C80165
:10C810000F94E025882309F488C05E2D4F2D302F1A
:10C82000212F852F942FA32FB22F89839A83AB8337
:10C83000BC8320E030E0A901B701C8010F94E025D6
:10C84000811108C0E0903D02F0903E0200913F024D
:10C8500010914002C701D8018D839E83AF83B887B2
:10C86000A501940160912E0C70912F0C8091300CD9
:10C870009091310C0F94E02587FF0CC080922E0C14
:10C8800090922F0CA092300CB092310CCE010196F8
:10C890000E941A2B4092260C5092270C6092280C72
:10C8A0007092290C89859A85AB85BC8580932A0C6A
:10C8B00090932B0CA0932C0CB0932D0CCE010596CD
:10C8C0000E941A2BA501940160912E0C70912F0CDF
:10C8D0008091300C9091310C0F94102F181664F445
:10C8E00080922E0C90922F0CA092300CB092310CB2
:10C8F000CE0101960E941A2B0E94B1612C960FB6B0
:10C90000F894DEBF0FBECDBFDF91CF911F910F9185
:10C91000FF90EF90DF90CF90BF90AF909F908F905F
:10C920007F906F905F904F90089550E040E030E826
:10C9300020E477CFCF92DF92EF92FF920F931F9375
:10C940006A01E0902E0CF0902F0C0091300C1091A9
:10C95000310CFB012081318142815381FC016081D6
:10C960007181828193810E94DE631F910F91FF90FC
:10C97000EF90DF90CF900895CF92DF92EF92FF92E9
:10C980000F931F936B01FC01E080F1800281138102
:10C99000E6E2FCE024813581468157816081718126
:10C9A000828193810E94DE631F910F91FF90EF902F
:10C9B000DF90CF9008950F931F93CF93DF93EC01F7
:10C9C0008B0181E00E940DF969E170E080E090E068
:10C9D0000E943F26B801CE010E94BC64C091E606C9
:10C9E00080E00E940DF91092E60682E00E94FE2F80
:10C9F0000E94352BC2FBCC27C0F981E08C27DF9148
:10CA0000CF911F910F910895AF92BF92CF92DF9275
:10CA1000EF92FF920F931F93CF93DF9300D01F925B
:10CA2000CDB7DEB7FC01E080F18002811381611196
:10CA300012C0A0902E0CB0902F0CC090300CD09053
:10CA4000310C9501A601B701C8010F94E02587FFBD
:10CA500002C07501860120E030E048EC53E4B701E4
:10CA6000C8010F94E02587FD04C0E12CF12C08ECEF
:10CA700013E4C701D80189839A83AB83BC8360EE3A
:10CA800072E0CE0101960E94BC640F900F900F904F
:10CA90000F90DF91CF911F910F91FF90EF90DF905A
:10CAA000CF90BF90AF9008953F924F925F926F9258
:10CAB0007F928F929F92AF92BF92CF92DF92EF922E
:10CAC000FF920F931F93CF93DF9300D01F92CDB7A8
:10CAD000DEB7382E80E090E0A0E2B1E489839A834B
:10CAE000AB83BC83C0907F12D0908012E090811203
:10CAF000F090821220E030E0A901C701B6010F9446
:10CB0000E02587FF0CC0A701960160E070E080E29D
:10CB100091E40F94AF2C69837A838B839C8360E0CC
:10CB2000CE0101960E9404654090260C5090270C7F
:10CB30006090280C7090290C80902A0C90902B0CFF
:10CB4000A0902C0CB0902D0C332089F10E94F6544B
:10CB500019821A821B821C82E0902E0CF0902F0CFE
:10CB60000091300C1091310CCE0101966C01A501A1
:10CB70009401C301B2010E94DE63309282070E94D9
:10CB8000A42B0F900F900F900F90DF91CF911F91DA
:10CB90000F91FF90EF90DF90CF90BF90AF909F905C
:10CBA0008F907F906F905F904F903F9008950E947C
:10CBB000B354CECF80918207882319F080E00E9481
:10CBC000546580E008952F923F924F925F926F924A
:10CBD0007F928F929F92AF92BF92CF92DF92EF920D
:10CBE000FF920F931F93CF93DF93CDB7DEB7669776
:10CBF0000FB6F894DEBF0FBECDBFF82E282E312C15
:10CC0000F101E056F64ED49022E0821335C08091B7
:10CC10008207811103C081E00E9454650E94F6548E
:10CC2000811139C18CE999E10E94BC1D20E030E0FE
:10CC3000A9010F94E0258823F9F06D2DDD0C770B09
:10CC4000880B990B0F94E7252B013C018CE999E1A6
:10CC50000E94BC1D4B015C0120E030E040EA50E442
:10CC60000F94E02511E087FF1CC0812C912C90EAE5
:10CC7000A92E90E4B92E15C06D2DDD0C770B880B15
:10CC8000990B0F94E7252B013C01C101880F991FD7
:10CC9000880F991F8C56964E0E94BC1D4B015C015B
:10CCA00010E0A3019201C501B4010F9446264B0187
:10CCB0005C016101CC0CDD1CCC0CDD1CC60188576D
:10CCC000964E0E94BC1DEE24E394E12620E030E065
:10CCD00040EC5FE30F944626A30192010F94462691
:10CCE000AB01BC0100E010E098018F2D0E94F762BB
:10CCF00020E030E0A901C501B4010F94E025F60160
:10CD0000E458F64EFA8BE98B882309F44DC0F2E023
:10CD100000E010E020E431E4FF1619F000E010E03C
:10CD20009801B501A4017058E12C8F2D0E94F76283
:10CD3000A5019401C501B4010F94B02C6B8B7C8BC1
:10CD40008D8B9E8B22E0F216E9F0F101E758F64E4A
:10CD50006491611107C00E943F4E87E599E10E94EE
:10CD60006C386AE070E090E080E00F94E5259B016C
:10CD7000AC0160E070E088E492E40F94AA2D8B018E
:10CD80009C0104C000E010E020EC30E4EE24E394C9
:10CD90004B895C896D897E898F2D0E94F76232E014
:10CDA000F312D0C00E94B35481E090E0A0E0B0E064
:10CDB0000F2C04C0880F991FAA1FBB1F0A94D2F71B
:10CDC0002091360C282B2093360C20919C05822B29
:10CDD00080939C0589899A890E94BC1DF601EA5DB1
:10CDE000F34F608371838283938382E0F8121AC0C9
:10CDF00020917F12309180124091811250918212C5
:10CE000060912E0C70912F0C8091300C9091310C10
:10CE10000F94AF2C60932E0C70932F0C8093300CDA
:10CE20009093310CF601E850F84F10821182128273
:10CE300013828F2D0E94D91C0E94352BF601EA5DCA
:10CE4000F34F80819181A281B381F601EE58F84FB2
:10CE500080839183A283B38392E0F916A9F18CE0D9
:10CE6000ECEAF2E0DE01119601900D928A95E1F76D
:10CE7000E1E0F0E0EC0FFD1FEC0DFD1D80809180E6
:10CE8000A280B38020E030E0A901C501B4010F9475
:10CE9000E02581111EC066960FB6F894DEBF0FBE66
:10CEA000CDBFDF91CF911F910F91FF90EF90DF9059
:10CEB000CF90BF90AF909F908F907F906F905F903A
:10CEC0004F903F902F9008950E94DA658111E3CF33
:10CED000C6CF20E030E0A901C501B4010F94102FA6
:10CEE00087FF04C0B7FAB094B7F8B094F601EA5DD2
:10CEF000F34F6F01A3019201C501B4010F944626BF
:10CF00009B01AC01F60160817181828193810F9454
:10CF1000AF2CF6016083718382839383F2E080E01B
:10CF200090E0A0E4B1E4FF1621F080E090E0A8E4F6
:10CF3000B2E48D879E87AF87B88BCE010D960E9495
:10CF40001A2BA9CF81E090E0A0E0B0E00F2C04C044
:10CF5000880F991FAA1FBB1F0A94D2F72091360C85
:10CF6000282B2093360C20919C05822B80939C05C6
:10CF700089899A890E94BC1DF601EA5DF34F60839E
:10CF80007183828393834ECFCF93DF9300D01F9220
:10CF9000CDB7DEB780E090E0A0EAB0E489839A8361
:10CFA000AB83BC8361E0CE0101960E9404650F90C3
:10CFB0000F900F900F90DF91CF9108958F929F92D5
:10CFC000AF92BF92CF92DF92EF92FF920F931F9397
:10CFD000CF93DF93CDB7DEB72C970FB6F894DEBFB3
:10CFE0000FBECDBF8B0140E050E068E472E44D839A
:10CFF0005E836F83788740E050E060EA70E44987A1
:10D000005A876B877C878130B9F1823009F459C027
:10D0100020E030E040E050E460912E0C70912F0C45
:10D020008091300C9091310C0F94B02C4B017C010D
:10D0300020E030E048EC53E40F94102F181634F43D
:10D04000812C912C88ECE82E93E4F92EF801A08431
:10D05000B184C284D3849401A701B501C6010F94A1
:10D06000102F181614F054016701C501D6018983E9
:10D070009A83AB83BC8348C0BE01675F7F4FC80102
:10D0800008960E94BC64B8016C5F7F4FAE014B5F95
:10D090005F4FC8010E949A640E94CE302C960FB652
:10D0A000F894DEBF0FBECDBFDF91CF911F910F91DE
:10D0B000FF90EF90DF90CF90BF90AF909F908F90B8
:10D0C0000895F801208531854285538560912E0CA5
:10D0D00070912F0C8091300C9091310C0F94B02CEA
:10D0E0006B017C0120E030E048EC53E40F94E02534
:10D0F00087FD06C0C12CD12C28ECE22E23E4F22EB1
:10D10000C982DA82EB82FC82BE01675F7F4FCE016B
:10D110000196B7CFEF92FF920F931F93CF93DF93B8
:10D120007C018B010E94C831C6E2DCE020916102E3
:10D13000309162024091630250916402F701608174
:10D140007181828193810F94AA2D2C853D854E8516
:10D150005F850F94B02C6C877D878E879F87C80171
:10D160000E941A2BDF91CF911F910F91FF90EF90AA
:10D170000C94B1614F925F926F927F92AF92BF9287
:10D18000CF92DF92EF92FF920F931F93CF93DF9393
:10D1900000D000D01F921F92CDB7DEB75C0180E0B7
:10D1A00090E0A0E7B2E489839A83AB83BC8380E0FC
:10D1B00090E0A0E8B0EC8D839E83AF83B887BE017A
:10D1C0006F5F7F4FCE0105960E948A6868E873E121
:10D1D00080E090E00E943F26C12CD12C88ECE82E04
:10D1E00081E4F82EC982DA82EB82FC8280E090E052
:10D1F000A0E8B0E48D839E83AF83B887BE016F5FE4
:10D200007F4FCE0105960E948A6808E31CE0F80172
:10D2100040AC51AC62AC73ACC0AED1AEE2AEF3AEDA
:10D2200080E090E0A0EAB1E489839A83AB83BC8379
:10D23000F50180819181A281B3818D839E83AF832B
:10D24000B887BE016F5F7F4FCE0105960E948A6846
:10D25000F80140AE51AE62AE73AE129A64E670E071
:10D2600080E090E00E943F2681E028960FB6F89477
:10D27000DEBF0FBECDBFDF91CF911F910F91FF9009
:10D28000EF90DF90CF90BF90AF907F906F905F90C6
:10D290004F9008951F93CF93DF93CDB7DEB72C97B0
:10D2A0000FB6F894DEBF0FBECDBF182F882379F0DC
:10D2B00020E030E0A9016091D4057091D5058091FE
:10D2C000D6059091D7050F94E0258823F9F0809139
:10D2D000370C8117D9F00E94B1618CE0E8EBF2E0E5
:10D2E000DE01119601900D928A95E1F7CE0101962B
:10D2F0000E94681F8091370C882391F086E29CE0A1
:10D300000E9441271092370C0E94352B2C960FB6A5
:10D31000F894DEBF0FBECDBFDF91CF911F9108956E
:10D3200081E08093370C86E29CE00E945521ECCF8F
:10D330002F923F924F925F926F927F928F929F9225
:10D34000AF92BF92CF92DF92EF92FF920F931F9313
:10D35000CF93DF93CDB7DEB7CB54D1090FB6F89496
:10D36000DEBF0FBECDBF2DB73EB739AF28AF87E0C8
:10D370000E944F4E81110BC061E086E50E948D2412
:10D380008DA3853060F087E39EE00E946C38A8ADE5
:10D39000B9AD0FB6F894BEBF0FBEADBF40C33DA13F
:10D3A000332321F087E19EE00E946C386AE080E53B
:10D3B0000E948D24182F8CEF810F8F3218F083EF8D
:10D3C0009DE0E3CF60E085E40E94A924882309F46E
:10D3D00048C081E08FABE0908312F0908412D701B7
:10D3E0002D913D914D915C916091260C7091270C8F
:10D3F0008091280C9091290C0F94B02CAB01BC01AA
:10D4000088E50E94FB2469877A878B879C87F701D0
:10D41000248135814681578160912A0C70912B0CB3
:10D4200080912C0C90912D0C0F94B02CAB01BC0171
:10D4300089E50E94FB246D877E878F87988BBE01CC
:10D44000635F7F4FCE0109960E946F2E382E8111A7
:10D450000BC063E68FED9DE00E94DA3F87EC9DE014
:10D4600094CF92E09FABB7CF8CE40E947D1E082F33
:10D47000882309F431C10E9479248EA3803118F0E9
:10D4800080EA9DE082CFFEA1F13009F427C160E07F
:10D4900083E50E94A9248AAF882321F0011102C0EC
:10D4A00037E03EA38DA1833020F086E89DE00E9406
:10D4B0006C389091370C9DAF80E00E944A690E94C1
:10D4C000121D1D8A1E8A1F8A188E198E1A8E1B8E97
:10D4D0001C8E83EF9FE4A3ECB7E48D8F9E8FAF8FFC
:10D4E000B8A383EF9FE4A3ECB7EC89A39AA3ABA303
:10D4F000BCA3A12FB0E0BCA7ABA7EDB7FEB724E05B
:10D50000129FE019F10911240FB6F894FEBF0FBE67
:10D51000EDBF8DB79EB701969CAF8BAF2DA14FA9E4
:10D52000BE01635F7F4FCE0109960E949CF99B016B
:10D53000AC010F94A22F811162C20E943EFD6115C1
:10D5400071058105910511F00F946621212C1BAA0C
:10D550001CAA1DAA1EAAAEA1A150BB0B2C96BFAF40
:10D56000AEAF2C97E22DF0E0F8A7EFA32BA53CA5DA
:10D57000E217F3070CF074C23196FEA7EDA73F93B4
:10D580002F93FF93EF9382E79DE09F938F938CE718
:10D590009DE09F938F931F920E942BF98DB79EB7AA
:10D5A00009960FB6F8949EBF0FBE8DBF9EA199231A
:10D5B00009F458C10F9417212AE030E040E050E010
:10D5C0000F94462C0F94E72520E030E040EA50E429
:10D5D0000F94102F0FEF1FEF181614F001E010E05A
:10D5E0000F94172128E631E040E050E00F94462CDC
:10D5F0000F94E7252B013C010F94172120E230E026
:10D6000040E050E00F94462C6B5F7F4F8F4F9F4F51
:10D610000F94E7254B015C01ADA1A430D1F4BC010E
:10D62000A40184E69DE00E944841B301A2018CE57B
:10D630009DE00E94484186E59DE00E946C380130E3
:10D64000110519F483E40E94333882E59DE00E94BD
:10D650006C38312CC801110FAA0BBB0B2A968CAF6A
:10D660009DAFAEAFBFAF2A972C96AEADBFAD2C9796
:10D670003A161B060CF0F6C02A966CAD7DAD8EAD49
:10D680009FAD2A970F94E7256B017C01BAADBB23B0
:10D6900041F1AC019B010F94B02C20E030E040E957
:10D6A00052E40F9446269B01AC01C301B2010F94D2
:10D6B000B02C2B013C0120E030E044EB53E40F940C
:10D6C000102F1816FCF420E030E044EB53E4C301C3
:10D6D000B2010F94AF2CEDCF1EA2D9CE22E02EA323
:10D6E000D6CE0F94172124E130E040E050E00F94B3
:10D6F000462C675E7F4F8F4F9F4F0F94E725A70102
:10D700009601CFCF20E030E0A901C301B2010F9410
:10D71000E02587FF0BC020E030E044EB53E4C30179
:10D72000B2010F94B02C2B013C01ECCF009183127D
:10D7300010918412F80124813581468157816D85CD
:10D740007E858F8598890F94AF2C22966CAF7DAF24
:10D750008EAF9FAF22972BED3FE049E450E4C30129
:10D76000B2010F94462620E030E044E353E40F94E6
:10D77000AA2D6B017C010F94A52D6FA778AB89AB07
:10D780009AABD8012D913D914D915C9169857A8537
:10D790008B859C850F94AF2C26966CAF7DAF8EAF9A
:10D7A0009FAF2697A50194016FA578A989A99AA989
:10D7B0000F9446269B01AC0126966CAD7DAD8EADD7
:10D7C0009FAD26970F94B02C69837A838B839C83BB
:10D7D000C701B6010F94502FA50194010F9446265E
:10D7E00022962CAD3DAD4EAD5FAD22970F94B02C7F
:10D7F0006D837E838F8398874BE351E070E060E018
:10D80000CE0101960E94F8C146E351E070E060E06D
:10D81000CE0105960E94F8C1BDA1B43099F44981AA
:10D820005A816B817C8186E49DE00E9448414D8154
:10D830005E816F8178858BE79FE20E9448418AE094
:10D840000E943338198A1A8A1B8A1C8AAE014F5EDD
:10D850005F4FBE016B5F7F4FCE0101960E949A64BD
:10D86000339402CF20E04FA9BE01635F7F4FCE010A
:10D8700009960E949CF94B015C01312CAC019B0183
:10D880000F94A22F811102C033243394A501940177
:10D89000C501B4010F94A22F8111E2C0EFA1F8A538
:10D8A000EE0FFF1FEE0FFF1F2BAD3CADE20FF31F7E
:10D8B00080829182A282B382A50194016D8D7E8DBA
:10D8C0008F8D98A10F94102F181624F48D8E9E8E94
:10D8D000AF8EB8A2A501940169A17AA18BA19CA1E8
:10D8E0000F94E02587FF04C089A29AA2ABA2BCA234
:10D8F000A50194016BA97CA98DA99EA90F94B02CB8
:10D900006BAB7CAB8DAB9EABADA5BEA5BD01BB0F1C
:10D91000880B990B0F94E7256FA378A789A79AA77F
:10D920009B01AC016BA97CA98DA99EA90F94AA2D7E
:10D930002B013C014D8A5E8A6F8A788EEBADFCAD7F
:10D94000F8ABEFA710E0C12CD12C7601AFA5B8A998
:10D950006D917D918D919D91B8ABAFA7A30192017F
:10D960000F94AF2C9B01AC010F9446269B01AC0198
:10D97000C701B6010F94B02C6B017C011F5F21160B
:10D9800028F72FA138A549A55AA50F94AA2D0F94C1
:10D990005E2F698F7A8F8B8F9C8FBDA1B23068F11B
:10D9A0008DA59EA50E945BE16BA57CA581E49DE011
:10D9B0000E946A418BE39DE00E946C3843E0C50100
:10D9C000B4010E947ABA80E20E94333881E0EDA16E
:10D9D000E3300CF480E0E12C8E010F5D1F4F9E01BF
:10D9E000235E3F4FAE01475E5F4FBE016B5E7F4FD0
:10D9F0000E94293F8AE00E9433382394B3CD0E94CD
:10DA0000DA650E94F91C8DAD0E944A690E94CE30F1
:10DA100088AD99AD0FB6F8949EBF0FBE8DBFE8AD2F
:10DA2000F9AD0FB6F894FEBF0FBEEDBFC55BDF4F7B
:10DA30000FB6F894DEBF0FBECDBFDF91CF911F911F
:10DA40000F91FF90EF90DF90CF90BF90AF909F909D
:10DA50008F907F906F905F904F903F902F900895A0
:10DA60000E94DA65332069F280E39DE00E946C3801
:10DA700081E0FDA11F160CF080E0EE24E3948E01FE
:10DA80000F5D1F4F9E01235E3F4FAE01475E5F4F0C
:10DA9000BE016B5E7F4F0E94293F698D7A8D8B8D11
:10DAA0009C8D0052110926E042E00F94AD209F9317
:10DAB0008F938FE19DE09F938F9389E29DE09F93E9
:10DAC0008F931F920E942BF92DB73EB7295F3F4FCE
:10DAD0000FB6F8943EBF0FBE2DBF93CF2F923F924B
:10DAE0004F925F926F927F928F929F92AF92BF926E
:10DAF000CF92DF92EF92FF920F931F93CF93DF931A
:10DB0000CDB7DEB76A970FB6F894DEBF0FBECDBFB4
:10DB100083E50E947D1E182F3090370C882319F062
:10DB20000E949924382E4090260C5090270C60902B
:10DB3000280C7090290C80912A0C90912B0CA091AC
:10DB40002C0CB0912D0C8B8B9C8BAD8BBE8B809154
:10DB50002E0C90912F0CA091300CB091310C8F8B2A
:10DB6000988FA98FBA8F112329F0311003C080E05C
:10DB70000E944A6986E50E947D1E8A8B20E030E083
:10DB8000A9016091D4057091D5058091D605909139
:10DB9000D7050F94E025882309F4C9C083E40E94C7
:10DBA0007D1E882309F49DC00E94D1246B017C0155
:10DBB000AEE8B7E0B987A887BF83AE83F5E0FD8301
:10DBC0001D861E8628EC2F8702EC1A86212C88ECF5
:10DBD0008B8792E49C87AE81BF81B98BA88B15E0BF
:10DBE000E889F98981909190A190B190F98BE88BA7
:10DBF0002A85322D4B855C85C501B4010F94E02543
:10DC000087FF04C08A86292CAB86BC862D853E857D
:10DC10004F85502FC501B4010F94102F181624F40E
:10DC20008D869E86AF860B2D1150D1F6FD81F15069
:10DC3000FD838E819F8144969F838E83F111CBCF8C
:10DC40002D853E854F85502F6A85722D8B859C854D
:10DC50000F94B02C20E030E040E05FE30F944626C4
:10DC6000A70196010F94B02C4B015C012DEB37E31B
:10DC700046E855EB0F94102F87FD0AC02DEB37E3D4
:10DC800046E855E3C501B4010F94E02518164CF59C
:10DC900080E00E944A6910E0E884F98400E0D7013E
:10DCA0006D917D918D919D917D016D01B4E0CB1AB7
:10DCB000D108A50194010F94AF2CF6016083718304
:10DCC00082839383602F812F0E9400F80F5F0530BD
:10DCD00031F71F5F88859985449699878887153025
:10DCE000D9F6AA89AA2381F020E030E0A901609149
:10DCF000D4057091D5058091D6059091D7050F94E4
:10DD0000E02581110E94B1408AE50E947D1E882392
:10DD100051F00E94D12469837A838B839C83CE0146
:10DD200001960E94C8F6832D0E944A690BC03110EB
:10DD300003C09A89992341F30E943F4E80E69CE0FC
:10DD40000E946C38332051F08091370C811106C04D
:10DD50000E943B4E81E49CE00E946C380E943F4E42
:10DD600083E39CE00E946C388091370C0E942A412A
:10DD70000E943F4E86E29CE00E946C38C090CA0828
:10DD8000D090CB08E090CC08F090CD0820E030E0B7
:10DD9000A901C701B6010F94102F18160CF053C03B
:10DDA00042E0C701B6010E947ABA8DE00E94333882
:10DDB0008AE00E943338A30192016091260C709191
:10DDC000270C8091280C9091290C0F94E02581114B
:10DDD0001FC02B893C894D895E8960912A0C709106
:10DDE0002B0C80912C0C90912D0C0F94E02581111F
:10DDF0000FC02F89388D498D5A8D60912E0C7091EE
:10DE00002F0C8091300C9091310C0F94E0258111F2
:10DE10000E94CE306A960FB6F894DEBF0FBECDBF1B
:10DE2000DF91CF911F910F91FF90EF90DF90CF90F6
:10DE3000BF90AF909F908F907F906F905F904F902A
:10DE40003F902F90089581E29CE00E946C38B3CF00
:10DE50008F929F92AF92BF92EF92FF920F931F9378
:10DE6000CF93DF9380E00E944A691092D005109210
:10DE7000D1051092D2051092D3051092CC051092C4
:10DE8000CD051092CE051092CF051092D8051092B4
:10DE9000D9051092DA051092DB051092D405109284
:10DEA000D5051092D6051092D7050EE817E0C0E010
:10DEB000812C912C80ECA82E8FE7B82E7801D0E031
:10DEC000F70181929192A192B1927F016D2F8C2FD7
:10DED0000E9400F8DF5FD53099F7CF5F0C5E1F4FCF
:10DEE000C53061F7DF91CF911F910F91FF90EF90B7
:10DEF000BF90AF909F908F900895909188128091DD
:10DF00008912981308C08091020990910309892B06
:10DF100011F40C94371F80E00E94475AEECF83E53E
:10DF20000E94CB1E8823E9F00E943EFD609375118C
:10DF30007093761180937711909378110E94D12479
:10DF400020E030E04AE754E40F9446260F94232E55
:10DF5000609313027093140280931502909316023B
:10DF600008958091350584FD0AC08091370587FDAD
:10DF700006C080913805837011F40C947D6F0E9467
:10DF8000B16188E50E947D1E882331F05F9A8091FF
:10DF9000360C8E7F8093360C89E50E947D1E882387
:10DFA00031F08A9A8091360C8D7F8093360C8AE509
:10DFB0000E947D1E882359F0809108018095817010
:10DFC000809306018091360C8B7F8093360C85E41C
:10DFD0000E947D1E81110C94351F08952F923F924F
:10DFE0004F925F926F927F928F929F92AF92BF9269
:10DFF000CF92DF92EF92FF920F931F93CF93DF9315
:10E00000CDB7DEB7A6970FB6F894DEBF0FBECDBF73
:10E0100082E797E00E94622A8091E40B83FD7EC034
:10E020002091320C3091330C4091340C5091350CCE
:10E0300060917E0770917F078091800790918107A2
:10E040000F94E025882309F469C01091010911118A
:10E0500061C080915F029091600201972091EA1166
:10E060003091EB11281739073CF40E943F4E8AE2A9
:10E0700099E10E946C3811E02091320C3091330C00
:10E080004091340C5091350C60917E0770917F0760
:10E0900080918007909181070F94AF2C6B017C01D8
:10E0A00020E030E0A9010F94102F87FF04C0F7FA99
:10E0B000F094F7F8F094209161023091620240915F
:10E0C000630250916402C701B6010F94462620E016
:10E0D00030E84BE354E40F94102F1816ECF40E9430
:10E0E0003F4E8BE099E10E946C3880917E079091C1
:10E0F0007F07A0918007B09181078093320C9093A5
:10E10000330CA093340CB093350C8EE797E00E944B
:10E11000C26104C010E0B0CF1111E7CF2AE037EDA3
:10E1200043E25CE3609141027091420280914302BC
:10E13000909144020F9446266B017C016091670226
:10E1400070916802072E000C880B990B0F94E7253D
:10E150009B01AC01C701B6010F944626698B7A8BEF
:10E160008B8B9C8B8091370C882309F18090CA0897
:10E170009090CB08A090CC08B090CD08C0907A07C2
:10E18000D0907B07E0907C07F0907D0720E030E0A6
:10E19000A901C501B4010F94E0258823D1F1A7019D
:10E1A0009601C501B4010F94102F181694F1C12CDB
:10E1B000D12C76018E010F5E1F4F2EE737E04AE724
:10E1C00057E066E777E082E797E00E9481F480E11C
:10E1D000E2E7F7E0A6E2BCE001900D928A95E1F754
:10E1E000A6960FB6F894DEBF0FBECDBFDF91CF91DC
:10E1F0001F910F91FF90EF90DF90CF90BF90AF9065
:10E200009F908F907F906F905F904F903F902F9056
:10E2100008952091260C3091270C4091280C5091A4
:10E22000290C609172077091730780917407909127
:10E2300075070F94AF2C6D8B7E8B8F8B988F2091F1
:10E240002A0C30912B0C40912C0C50912D0C60918C
:10E2500076077091770780917807909179070F94EE
:10E26000AF2C698F7A8F8B8F9C8F20912E0C3091E1
:10E270002F0C4091300C5091310CC701B6010F9416
:10E28000AF2C6D8F7E8F8F8F98A32091320C3091A1
:10E29000330C4091340C5091350C60917E07709195
:10E2A0007F0780918007909181070F94AF2C6B01BD
:10E2B0007C0120E030E0A9016D897E898F89988DED
:10E2C0000F94E02581110CC020E030E0A901698D98
:10E2D0007A8D8B8D9C8D0F94E025882309F467CF70
:10E2E0002D893E894F89588DCA01B9010F94462660
:10E2F0004B015C01298D3A8D4B8D5C8DCA01B901B2
:10E300000F9446269B01AC01C501B4010F94B02CBB
:10E310004B015C012D8D3E8D4F8D58A1CA01B90175
:10E320000F9446269B01AC01C501B4010F94B02C9B
:10E330004B015C01A7019601C701B6010F94462667
:10E340009B01AC01C501B4010F94B02C0F945E2F5A
:10E350004B015C012DEB37E346E855E30F94E025D4
:10E3600087FF0FC020E030E0A901C701B6010F947C
:10E37000102F4601570187FF04C0B7FAB094B7F8D1
:10E38000B0942DEB37E346E855E3C501B4010F9493
:10E39000E02587FD1CCF20E030E040EA51E4C501D4
:10E3A000B4010F94AA2D0F94232E1B01672B19F48F
:10E3B00022242394312CB10190E080E00F94E525D4
:10E3C0009B01AC0160E070E080E89FE30F94AA2D10
:10E3D0002B013C01AC019B01C501B4010F94462601
:10E3E0004B015C01A30192016D897E898F89988D13
:10E3F0000F9446266D8B7E8B8F8B988FA301920195
:10E40000698D7A8D8B8D9C8D0F944626698F7A8FBE
:10E410008B8F9C8FA30192016D8D7E8D8F8D98A126
:10E420000F9446266D8F7E8F8F8F98A3A301920144
:10E43000C701B6010F94462669A37AA38BA39CA3B8
:10E4400080E1E6E2FCE08E010F5F1F4FD8010190F2
:10E450000D928A95E1F70E943EFD2B013C0128ECCC
:10E46000420E511C611C711C0DA31EA381E0281AD1
:10E47000310809F460C00E943EFD8B019C01041923
:10E4800015092609370937FD59C02B013C0128EC35
:10E49000420E511C611C711C80E00E94475A2D895C
:10E4A0003E894F89588D69817A818B819C810F9437
:10E4B000B02C69837A838B839C83298D3A8D4B8D15
:10E4C0005C8D6D817E818F8198850F94B02C6D83DA
:10E4D0007E838F8398872D8D3E8D4F8D58A16985C2
:10E4E0007A858B859C850F94B02C69877A878B877A
:10E4F0009C8729A13AA14BA15CA16D857E858F8562
:10E5000098890F94B02C6D877E878F87988B7501C3
:10E5100064018E010F5E1F4F9E01235F3F4FAE01CE
:10E52000475F5F4FBE016B5F7F4F8DA19EA10E9431
:10E5300081F481119BCF750164013CCE0E943AC2E7
:10E54000AECF8F929F92AF92BF92CF92DF92EF9217
:10E55000FF92CF93DF938090410290904202A0906F
:10E560004302B0904402FC01C080D180E280F3807D
:10E5700020E030E0A901C701B6010F94E02588230F
:10E5800041F0C0924102D0924202E0924302F092E6
:10E590004402C0916702D091680284E690E09093B3
:10E5A000680280936702C0906102D0906202E0909E
:10E5B0006302F090640280E090E0A0E8BFE3809303
:10E5C000610290936202A0936302B09364020E947E
:10E5D000EE6F8092410290924202A0924302B0926A
:10E5E0004402D0936802C0936702C0926102D09245
:10E5F0006202E0926302F0926402DF91CF91FF9099
:10E60000EF90DF90CF90BF90AF909F908F90089544
:10E610000F931F93CF93DF9300D01F92CDB7DEB738
:10E620009C0102E717E090E1E6E2FCE0D8010190EE
:10E630000D929A95E1F7F901208131814281538150
:10E64000F80160857185828593850F94B02CF8015F
:10E65000608771878287938780E090E0A0EAB0E4CA
:10E6600089839A83AB83BC83CE0101960E94A172F9
:10E670000F900F900F900F90DF91CF911F910F91FE
:10E6800008952F923F924F925F926F927F928F9256
:10E690009F92AF92BF92CF92DF92EF92FF921F9321
:10E6A000CF93DF93CDB7DEB72C970FB6F894DEBFCC
:10E6B0000FBECDBF7A011901DC012D913D914D9125
:10E6C0005C912D833E834F835887FB0140805180AE
:10E6D000628073808090260C9090270CA090280C6C
:10E6E000B090290CA50194016D817E818F81988560
:10E6F0000F94E02581110EC011E0A30192016091F9
:10E700002A0C70912B0C80912C0C90912D0C0F9455
:10E71000E025811110E0D1012D913D914D915C9149
:10E7200029873A874B875C87F701C080D180E280D8
:10E73000F38020910B0230910C0240910D02509118
:10E740000E02C701B6010F94E025882309F44EC0DC
:10E75000C0920B02D0920C02E0920D02F0920E02D7
:10E760008091320C9091330CA091340CB091350C07
:10E7700040912A0C50912B0C60912C0C70912D0C17
:10E780008092720790927307A0927407B0927507F7
:10E7900040937607509377076093780770937907D3
:10E7A000C0927A07D0927B07E0927C07F0927D07B7
:10E7B00080937E0790937F07A0938007B093810793
:10E7C00020E030E040E05FE36091640C7091650C04
:10E7D0008091660C9091670C0F94462669837A832A
:10E7E0008B839C83CE0101960E94A1722D813E8174
:10E7F0004F815885209372073093730740937407B5
:10E800005093750740927607509277076092780789
:10E8100070927907D1012D913D914D915C9160915C
:10E820007E0770917F0780918007909181070F94F8
:10E83000B02C60937E0770937F078093800790933E
:10E84000810711112FC020E030E0A90169857A8588
:10E850008B859C850F94E025811133C060E070E0CA
:10E8600088EC92E469837A838B839C83CE01019642
:10E870000E94A1722C960FB6F894DEBF0FBECDBFDA
:10E88000DF91CF911F91FF90EF90DF90CF90BF90DD
:10E89000AF909F908F907F906F905F904F903F9040
:10E8A0002F9008952AEF3EE74AE25FE36091680CFB
:10E8B0007091690C80916A0C90916B0C0F944626B4
:10E8C000D1CF60E070E080EA91E4CCCF0F931F934A
:10E8D000CF93DF9300D000D01F921F92CDB7DEB749
:10E8E0008B01FC0123A5211102C00E9489FB1D821E
:10E8F0001E821F82188620E030E040E05FE36091D6
:10E900002E0C70912F0C8091300C9091310C0F9443
:10E91000B02C69837A838B839C839E012B5F3F4F4E
:10E92000AE014F5F5F4F6AE27CE086E29CE00E94AE
:10E9300041731D821E821F82188620E030E040E075
:10E940005FE3F80160857185828593850F94B02C13
:10E9500069837A838B839C83B8016C5F7F4F9E01B0
:10E960002B5F3F4FAE014F5F5F4FC8010E94417365
:10E9700028960FB6F894DEBF0FBECDBFDF91CF91C2
:10E980001F910F9108959B01AC01485F5F4FBC013F
:10E990006C5F7F4F0C9441732F923F924F925F9226
:10E9A0006F927F928F929F92AF92BF92CF92DF929F
:10E9B000EF92FF920F931F93CF93DF93CDB7DEB704
:10E9C000A6970FB6F894DEBF0FBECDBF8C011B011A
:10E9D0005A8749874090260C5090270C6090280C4D
:10E9E0007090290C80902A0C90902B0CA0902C0CED
:10E9F000B0902D0CDB018D919D910D90BC91A02DBF
:10EA00008B8B9C8BAD8BBE8B9C01AD01C301B20186
:10EA10000F94AF2C6B017C01D10114968D919D91C7
:10EA20000D90BC91A02D8F8B988FA98FBA8F9C01D0
:10EA3000AD01C501B4010F94AF2C6B8F7C8F8D8F0E
:10EA40009E8FA985BA858D919D910D90BC91A02D29
:10EA50008B879C87AD87BE879C01AD01C301B20146
:10EA60000F94AF2C6F8F78A389A39AA3A985BA8539
:10EA700014968D919D910D90BC91A02D8F87988BB0
:10EA8000A98BBA8B9C01AD01C501B4010F94AF2CC9
:10EA90006BA37CA38DA39EA3A7019601C701B6011A
:10EAA0000F9446266B017C012B8D3C8D4D8D5E8D28
:10EAB000CA01B9010F9446269B01AC01C701B601FA
:10EAC0000F94B02C4B015C012B893C894D895E89E8
:10EAD0006B857C858D859E850F94AF2C2B013C0129
:10EAE0002F89388D498D5A8D6F85788989899A89C2
:10EAF0000F94AF2C6B017C01A3019201C301B20101
:10EB00000F9446262B013C01A7019601C701B601CF
:10EB10000F9446269B01AC01C301B2010F94B02CA7
:10EB20000F945E2F6B017C012F8D38A149A15AA152
:10EB3000CA01B9010F9446262B013C012BA13CA12F
:10EB40004DA15EA1CA01B9010F9446269B01AC01FB
:10EB5000C301B2010F94B02C9B01AC01C501B401FB
:10EB60000F94102F1816B4F520E030E0A901C7016A
:10EB7000B6010F94102F87FF2AC0C701B601905825
:10EB800020E030E040EA50E40F94102F181614F5FE
:10EB9000A10169857A85C8010E94CC74A6960FB63A
:10EBA000F894DEBF0FBECDBFDF91CF911F910F91C3
:10EBB000FF90EF90DF90CF90BF90AF909F908F909D
:10EBC0007F906F905F904F903F902F900895C70176
:10EBD000B601D6CF20E030E040E050E4C501B401FA
:10EBE0000F94102F181624F4B101C8010E94667406
:10EBF00019821A821B821C82BE016F5F7F4FC10186
:10EC00000E94C3742DEC3CEC4CEC5CE3C701B601F4
:10EC10000F9446269B01AC01F801608171818281CD
:10EC200093810F9446266D837E838F839887D801C6
:10EC30009B968C919B978823C9F02AE939E949E989
:10EC40005FE314966D917D918D919C9117970F9430
:10EC5000462669837A838B839C83BE016F5F7F4FD7
:10EC600082E797E00E94C374F80113A6BE016B5FB0
:10EC70007F4F89859A850E94C37490CF3F924F92AF
:10EC80005F926F927F928F929F92AF92BF92CF923C
:10EC9000DF92EF92FF920F931F93CF93DF93CDB745
:10ECA000DEB76C970FB6F894DEBF0FBECDBFDB01A9
:10ECB0000C91142F100F153008F067C11196DC90DD
:10ECC000C22ECD0CB4E0BC1508F45FC1ED2DF0E010
:10ECD000E450FB4F8080912CB12CA12C002E04C05D
:10ECE000B694A794979487940A94D2F780FE4DC166
:10ECF000EC2DF0E0E450FB4F8080912CB12CA12C46
:10ED0000012E04C0B694A794979487940A94D2F7DE
:10ED100080FE3BC1322E642F7C014090CC05509088
:10ED2000CD056090CE057090CF058091D40590916F
:10ED3000D505A091D605B091D705898F9A8FAB8F55
:10ED4000BC8F660F770B072E000C880B990B0F9466
:10ED5000E7254B015C01602F000F770B880B990BA7
:10ED60000F94E725298D3A8D4B8D5C8D0F944626A7
:10ED7000A30192010F94B02CA50194010F94B02C23
:10ED80006D877E878F87988B612F110F770B880B8C
:10ED9000990B0F94E725298D3A8D4B8D5C8D0F943F
:10EDA0004626A30192010F94B02CA50194010F9463
:10EDB000AF2C69837A838B839C834090D0055090DD
:10EDC000D1056090D2057090D3058091D8059091BF
:10EDD000D905A091DA05B091DB05898F9A8FAB8FA9
:10EDE000BC8F632D660F770B072E000C880B990BD9
:10EDF0000F94E7254B015C016D2DDD0C770B880B23
:10EE0000990B0F94E725298D3A8D4B8D5C8D0F94CE
:10EE10004626A30192010F94B02CA50194010F94F2
:10EE2000B02C698B7A8B8B8B9C8B6C2DCC0C770BDD
:10EE3000880B990B0F94E725298D3A8D4B8D5C8DAE
:10EE40000F944626A30192010F94B02CA5019401C2
:10EE50000F94AF2C6D837E838F839887F701808515
:10EE60009185A285B38589879A87AB87BC878D8B6F
:10EE70009E8BAF8BB88F45E351E061E070E0CE012F
:10EE800041960E94F8C145E351E061E070E0CE0197
:10EE900005960E94F8C14AE351E061E070E0CE01BE
:10EEA0000D960E94F8C14AE351E061E070E0CE01A6
:10EEB00001960E94F8C189889A88AB88BC8827E1AE
:10EEC00037EB41ED58EBC501B4010F94102F87FDCE
:10EED0005CC023E030E04BE953E4C501B4010F947A
:10EEE000E02518160CF451C08D849E84AF84B88838
:10EEF00027E137EB41ED58EBC501B4010F94102F1A
:10EF000087FD43C023E030E84DE953E4C501B40177
:10EF10000F94E0251816CCF18D809E80AF80B884C8
:10EF200027E137EB41ED58EBC501B4010F94102FE9
:10EF300087FD2BC023E030E04BE953E4C501B40169
:10EF40000F94E02518160CF189809A80AB80BC8064
:10EF500027E137EB41ED58EBC501B4010F94102FB9
:10EF600087FD13C023E030E84DE953E4C501B40147
:10EF70000F94E02518164CF0AE014F5F5F4FBE01B5
:10EF8000635F7F4FC7010E94CC746C960FB6F894F4
:10EF9000DEBF0FBECDBFDF91CF911F910F91FF90CC
:10EFA000EF90DF90CF90BF90AF909F908F907F9029
:10EFB0006F905F904F903F9008952F923F924F92A5
:10EFC0005F926F927F928F929F92AF92BF92CF92F9
:10EFD000DF92EF92FF920F931F93CF93DF93CDB702
:10EFE000DEB7CC58D1090FB6F894DEBF0FBECDBF47
:10EFF00080E19CE00E946C3887E00E944F4E8111B6
:10F000006EC084E50E94CB1E882329F00E94BE2496
:10F0100081110E9468BA80E090E0A0E8BFE3898394
:10F020009A83AB83BC838D839E83AF83B8878DEC3B
:10F030009CECACE4BEE389879A87AB87BC8780E011
:10F0400090E0A0E2B1E48D879E87AF87B88B8CE318
:10F0500090E09A8B898B8DEC90E09C8B8B8B8DEC68
:10F060009CECACECBEE38D8B9E8BAF8BB88F80E0BD
:10F0700090E0A0EEBFE3898F9A8FAB8FBC8F1BA669
:10F080001CA64AE959E969E97EE38FE40E94FB2462
:10F090006D8F7E8F8F8F98A360E083E40E94A924F8
:10F0A00089A360E08BE40E94A9248AA382E40E94E1
:10F0B000CB1E882381F10E94BE24009761F19C0140
:10F0C000285231092536310520F16CE870E082EED6
:10F0D0009BE00E946A418DED9BE00E946C38C45712
:10F0E000DF4F0FB6F894DEBF0FBECDBFDF91CF91DB
:10F0F0001F910F91FF90EF90DF90CF90BF90AF9056
:10F100009F908F907F906F905F904F903F902F9047
:10F1100008959A8B898B8CE40E94CB1E8823E1F0A2
:10F120000E94D1246B017C01C986DA86EB86FC86BD
:10F1300020E030E0A9010F94102F87FD0AC020E0E5
:10F1400030E040E050E4C701B6010F94E025181606
:10F150001CF485EB9BE0C1CF81E50E947D1E8823D6
:10F1600031F18091050590910605892BE9F00E9407
:10F17000D1246B017C01CD82DE82EF82F8862DECFA
:10F180003CEC4CE45DE30F94102F87FD0AC020E0B7
:10F1900030E040E751E4C701B6010F94E0251816AE
:10F1A00034F484E89BE099CF89E59BE096CF83E532
:10F1B0000E94CB1E8823E9F00E94D1246B017C01C0
:10F1C000CD8ADE8AEF8AF88E2DEC3CEC4CEC5DE3C8
:10F1D0000F94102F87FD0AC020E030E040E050E49B
:10F1E000C701B6010F94E02518161CF482E39BE0DA
:10F1F00074CF80E50E947D1E882341F18091050532
:10F2000090910605892B19F48AEF9AE066CF8BA5B9
:10F210008F5F8BA70E94D1246B017C01CD86DE8697
:10F22000EF86F88A20E030E0A9010F94102F87FDC7
:10F230000AC020E030E048EC51E4C701B6010F9469
:10F24000E02518161CF482ED9AE047CF86E40E9470
:10F25000CB1E8823E9F00E94D1246B017C01C98E6A
:10F26000DA8EEB8EFC8E20E030E040E85FE30F9416
:10F27000102F87FD0AC020E030E040E850E4C701CD
:10F28000B6010F94E02518161CF489EA9AE025CF00
:10F29000C98CDA8CEB8CFC8C8D889E88AF88B88CFE
:10F2A000A7019601C701B6010F9446269B01AC0148
:10F2B00060E070E084E490E40F94AA2D29813A8103
:10F2C0004B815C810F9446262B013C01A5019401E2
:10F2D000C501B4010F944626A70196010F94462656
:10F2E0002CEE31E548EB5DE30F94AA2D9B01AC01B8
:10F2F000C301B2010F94462669837A838B839C8372
:10F3000088E40E94CB1E882379F00E94BE240097D7
:10F3100059F09C01255A31092838310518F08BE73E
:10F320009AE0DBCE9C8B8B8B85E50E947D1E88232B
:10F33000C9F00E943EFD611571058105910511F02E
:10F340000F9466218091050590910605892B91F017
:10F350000E94D124609301057093020580930305F8
:10F360009093040582E50E947D1E811108C087E408
:10F370009AE0B3CE60E070E088E492E4EBCF809155
:10F38000050590910605892B61F00E94BE24AD967B
:10F390009FAF8EAFAD97181619064CF083E19AE037
:10F3A0009CCE2AE130E0AD963FAF2EAFAD9789E518
:10F3B0000E94CB1E882381F10E94D1242091D20883
:10F3C0003091D3084091D4085091D5080F94AF2CB8
:10F3D0006B017C0188E50E94CB1E882331F10E94DD
:10F3E000D1242091CE083091CF084091D00850917F
:10F3F000D1080F94AF2C6BA37CA38DA39EA3CFA2A7
:10F40000D8A6E9A6FAA6CE0183960E943C1E8111D9
:10F4100015C089EE99E061CEC0902A0CD0902B0CDB
:10F42000E0902C0CF0902D0CD5CF6091260C7091B3
:10F43000270C8091280C9091290CDDCF84E40E9448
:10F440007D1E91E089270E944A6980E090E0A0EA51
:10F45000B0E48DA79EA7AFA7B8AB60E0CE018D96B4
:10F460000E9404653091F707CD57DF4F3883C358AA
:10F47000D0401092F7070E94361C88EC99E00E9459
:10F480006C3889899A898A3191050CF044C08B893E
:10F490009C890E94531F61E080E00E9408BD811199
:10F4A00042C06FEF8DED99E00E94DA3F8CA581118B
:10F4B00004C0CE0101960E9489FB80E090E0A0EAA2
:10F4C000B0E480937A0790937B07A0937C07B09376
:10F4D0007D071DA61EA61FA618AABE01635D7F4F4D
:10F4E00082E797E00E94C374CD57DF4F5881C3581D
:10F4F000D0405093F7070E94361C8AA18111EFCDAE
:10F5000010928211109281110E94C0BE90E080E0A2
:10F510000E94531FE4CD0E94912281E00E9491BB82
:10F520008111B5CFBECF1092320C1092330C1092D5
:10F53000340C1092350C82E39CE00E94C2618BA5D2
:10F54000882309F452C020E030E040E751E46091A4
:10F55000680C7091690C80916A0C90916B0C0F94FF
:10F56000AA2D6DA77EA78FA798AB80E1E6E2FCE00D
:10F57000A2E7B7E001900D928A95E1F72D853E85CF
:10F580004F85588960917E0770917F078091800731
:10F59000909181070F94B02C60937E0770937F0742
:10F5A0008093800790938107CE018D960E94A1726F
:10F5B0002D853E854F85588960917E0770917F0724
:10F5C00080918007909181070F94AF2C60937E0704
:10F5D00070937F0780938007909381078CA581119A
:10F5E00004C0CE0101960E9489FBECEFF4E085E0B7
:10F5F000DF011D928A95E9F780E1E6E2FCE0A2E7EF
:10F60000B7E001900D928A95E1F789859A85AB85DF
:10F61000BC8580937A0790937B07A0937C07B09377
:10F620007D071DA61EA61FA618AABE01635D7F4FFB
:10F6300082E797E00E94C374BE01635E7F4F82E75A
:10F6400097E00E94C37489A1882309F41CC4209107
:10F65000260C3091270C4091280C5091290CE596EE
:10F660002CAF3DAF4EAF5FAFE59780912A0C9091E4
:10F670002B0CA0912C0CB0912D0CE1968CAF9DAF72
:10F68000AEAFBFAFE197312C212C9FEFA4969FAF77
:10F69000A497AFEFA896AFAFA897BFEFC158DF4FC1
:10F6A000B883CF57D040EFE4C058DF4FE883C0584D
:10F6B000D040F3ECCF57DF4FF883C158D04027E458
:10F6C000CE57DF4F2883C258D04081E090E0A0E0C1
:10F6D000B0E0022C04C0880F991FAA1FBB1F0A9418
:10F6E000D2F7CC57DF4F88839983AA83BB83C45852
:10F6F000D040ACEFB4E0E796BFAFAEAFE79710E015
:10F7000000E09101032C000C440B550BC857DF4F50
:10F71000288339834A835B83C858D040C457DF4F5E
:10F720002882CC58D040E796AEADBFADE7978D911B
:10F73000E796BFAFAEAFE79790E0B0E0A0E0CC5760
:10F74000DF4F288139814A815B81C458D0408223B0
:10F750009323A423B523892B8A2B8B2B09F024C157
:10F76000C857DF4F688179818A819B81C858D04012
:10F770000F94E7252091D4053091D5054091D60509
:10F780005091D7050F9446262091CC053091CD0598
:10F790004091CE055091CF050F94B02CEB966CAFF5
:10F7A0007DAF8EAF9FAFEB97B801012E000C880B99
:10F7B000990B0F94E7252091D8053091D9054091F8
:10F7C000DA055091DB050F9446262091D005309143
:10F7D000D1054091D2055091D3050F94B02C6B0107
:10F7E0007C01EB962CAD3DAD4EAD5FADEB97E59654
:10F7F0006CAD7DAD8EAD9FADE5970F94AF2C2B0119
:10F800003C01A7019601E1966CAD7DAD8EAD9FAD3B
:10F81000E1970F94AF2C4B015C01A3019201C3014E
:10F82000B2010F9446262B013C01A5019401C501AC
:10F83000B4010F9446269B01AC01C301B2010F94A1
:10F84000B02C0F945E2F4B015C01EB962CAD3DADBF
:10F850004EAD5FADEB976BA17CA18DA19EA10F94E6
:10F86000AF2C2B013C01A70196016FA178A589A5BA
:10F870009AA50F94AF2C6B017C01A3019201C301E7
:10F88000B2010F9446262B013C01A7019601C70146
:10F89000B6010F9446269B01AC01C301B2010F943F
:10F8A000B02C0F945E2F20E030E040E751E40F943D
:10F8B000AA2DA50194010F94B02C6B017C018090BE
:10F8C000010590900205A0900305B090040520E08A
:10F8D00030E040E85FE3C501B4010F94102F181623
:10F8E000F4F4C501B4010F941C2E4B015C0160E0DF
:10F8F00070E0CB01181419041A041B0434F40F949B
:10F900001721A50194010F94462C0F94E7259B0124
:10F91000AC01B601C7010F94B02C6B017C01C1583A
:10F92000DF4F2881CF57D040C058DF4F3881C058B3
:10F93000D040CF57DF4F4881C158D040CE57DF4F1E
:10F940005881C258D040B601C7010F94E02587FF07
:10F950002BC0A4960FAFA497C457DF4F3881CC5863
:10F96000D040A8963FAFA897EC96CFAEEC97ED9617
:10F97000DFAEED97EE96EFAEEE97EF96FFAEEF9718
:10F98000C158DF4FC882CF57D040C058DF4FD88210
:10F99000C058D040CF57DF4FE882C158D040CE5733
:10F9A000DF4FF882C258D0400F5F1F4F053011055E
:10F9B00009F0B9CE4FEF241A340A55E02516310468
:10F9C00009F083CEA4968FADA497E82FF0E0E45021
:10F9D000FB4F208181E090E0A0E0B0E0A8960FAC62
:10F9E000A89704C0880F991FAA1FBB1F0A94D2F7BB
:10F9F000822B8083A8969FADA8976A969FAF6A973F
:10FA0000A496AFADA4976B96AFAF6B97EC968FAD06
:10FA1000EC97ED969FADED97EE96AFADEE97EF9626
:10FA2000BFADEF976F968CAF9DAFAEAFBFAF6F9787
:10FA3000A896BFADA897BF3F09F409C2A496EFAD41
:10FA4000A497EF3F09F403C26B2FBB0F770B880B12
:10FA5000990B0F94E7252091D4053091D50540915D
:10FA6000D6055091D7050F9446262091CC053091AC
:10FA7000CD054091CE055091CF050F94B02C162F97
:10FA8000072F382E292E862F902FA32DB22D659665
:10FA90008CAF9DAFAEAFBFAF6597A496FFADA497F7
:10FAA0006F2FFF0F770B880B990B0F94E725209191
:10FAB000D8053091D9054091DA055091DB050F94B6
:10FAC00046262091D0053091D1054091D205509124
:10FAD000D3050F94B02C6B017C016996CCAEDDAEE2
:10FAE000EEAEFFAE6997CE018F5A9F4F0E943C1E2B
:10FAF000882309F4B0C120E030E040EA50E4612FEF
:10FB0000702F832D922D0F94B02C4B015C01CB01F3
:10FB1000D50121968CAF9DAFAEAFBFAF2197259693
:10FB2000CCAEDDAEEEAEFFAE2597A8962FADA89772
:10FB30002111E3C1A4963FADA4973111B3C120E0D8
:10FB400030E040EA50E4C701B6010F94B02C6B01DD
:10FB50007C01A4964FADA497442309F4C5C1A49693
:10FB60008FADA49784300CF0BFC122ED422E23E567
:10FB7000522E2BE7622E21E4722E21968CAC9DAC86
:10FB8000AEACBFAC219725968CAD9DADAEADBFADF3
:10FB90002597A7968CAF9DAFAEAFBFAFA7979C013F
:10FBA000AD0169966CAD7DAD8EAD9FAD69970F943B
:10FBB000AF2CAB966CAF7DAF8EAF9FAFAB97A5016F
:10FBC000940165966CAD7DAD8EAD9FAD65970F943C
:10FBD000AF2C2D966CAF7DAF8EAF9FAF2D97AB96B0
:10FBE0002CAD3DAD4EAD5FADAB9761962CAF3DAF4B
:10FBF0004EAF5FAF6197A50194016091260C7091A3
:10FC0000270C8091280C9091290C0F94AF2C4B015C
:10FC10005C01A7962CAD3DAD4EAD5FADA797609151
:10FC20002A0C70912B0C80912C0C90912D0C0F9420
:10FC3000AF2CA7966CAF7DAF8EAF9FAFA797812FEC
:10FC4000902FA32DB22D8DA79EA7AFA7B8ABC9AAA1
:10FC5000DAAAEBAAFCAAC984DA84EB84FC84CDAAD4
:10FC6000DEAAEFAAF8AE2DEC3CEC4CEC5CE3C30151
:10FC7000B2010F94462629813A814B815C810F9411
:10FC800046262091320C3091330C4091340C509127
:10FC9000350C0F94B02C69AF7AAF8BAF9CAFA50138
:10FCA0009401C501B4010F9446264B015C01A7964F
:10FCB0002CAD3DAD4EAD5FADA797CA01B9010F9414
:10FCC00046269B01AC01C501B4010F94B02C20E085
:10FCD00030E040E050E40F94102F1816ACF420E010
:10FCE00030E040E05FE3C701B6010F94B02C2996E5
:10FCF0006CAF7DAF8EAF9FAF2997BE01635C7F4F26
:10FD0000CE0101960E94667489859A85AB85BC8573
:10FD100029968CAF9DAFAEAFBFAF2997A3961CAE0F
:10FD20001DAE1EAE1FAEA397BE01615A7F4FCE011E
:10FD3000CD960E94C3748CA58823C1F02AE939E9C5
:10FD400049E95FE36D817E818F8198850F94462616
:10FD5000A3966CAF7DAF8EAF9FAFA397BE01615AE4
:10FD60007F4F82E797E00E94C3741CA6E090600C6E
:10FD7000F090610C0091620C1091630CA0905C0CEF
:10FD8000B0905D0CC0905E0CD0905F0C9501A60108
:10FD9000B701C8010F94102F181614F475018601CD
:10FDA0008090410290904202A0904302B0904402A1
:10FDB0002DEC3CEC4CEC5DE3B701C8010F944626FA
:10FDC00060934102709342028093430290934402F5
:10FDD00040E0BE01675B7F4FCE018D960F941815F2
:10FDE00080E1E6E2FCE0A2E7B7E001900D928A959F
:10FDF000E1F78092410290924202A0924302B092B7
:10FE0000440220E04FEFBE01675A7F4FCE010196BA
:10FE10000E943E7620E041E0BE01675A7F4FCE014E
:10FE200001960E943E762FEF40E0BE01675A7F4F59
:10FE3000CE0101960E943E7621E040E0BE01675A65
:10FE40007F4FCE0101960E943E760E94B161809163
:10FE5000A30C8093A40CAD964EAD5FADAD97415011
:10FE60005109AD965FAF4EAFAD97452B09F419CB55
:10FE70006A968FAD6A9787FD14CB6B968FAD6B97A3
:10FE800087FFE1CB0ECB2BA13CA14DA15EA1E59656
:10FE90002CAF3DAF4EAF5FAFE5978FA198A5A9A559
:10FEA000BAA5EBCB812F902FA32DB22D21968CAF2D
:10FEB0009DAFAEAFBFAF219720E030E040EA50E405
:10FEC000C701B6010F94AF2C25966CAF7DAF8EAFF6
:10FED0009FAF2597A4965FADA49754300CF42FCE16
:10FEE000182D092D3A2C2B2C92ED492E93E5592EE5
:10FEF0009BEF692E90E4792E40CEA8969FADA897EF
:10FF000094300CF452C0A496AFADA497A4300CF179
:10FF100020E030E040EA50E4612F702F832D922DD5
:10FF20000F94AF2C21966CAF7DAF8EAF9FAF219712
:10FF300020E030E040EA50E4C701B6010F94AF2C56
:10FF40006B017C01A496EFADA497E4300CF40DCEC8
:10FF5000CBCF812F902FA32DB22D21968CAF9DAFAB
:10FF6000AEAFBFAF219720E030E040EA50E4C701D8
:10FF7000B6010F94B02C25966CAF7DAF8EAF9FAFBE
:10FF80002597A496BFADA497B111D2CF20E030E061
:10FF900040EA50E4612F702F832D922D0F94AF2CE7
:10FFA000162F072F382E292E9FCFA496FFADA4978A
:10FFB000F1110DC020E030E040E251E4B401C50190
:10FFC0000F94AF2C162F072F382E292ECECDA496A6
:10FFD0002FADA49724309CF020E030E040E251E4C3
:10FFE000B401C5010F94AF2C21966CAF7DAF8EAFDD
:10FFF0009FAF2197182D092D3A2C2B2CB6CD182DFB
:020000021000EC
:10000000092D3A2C2B2C82ED482E83E5582E8BEFB0
:10001000682E81E4782EB1CD2F923F924F925F925D
:100020006F927F928F929F92AF92BF92CF92DF9208
:10003000EF92FF920F931F93CF93DF93CDB7DEB76D
:10004000EE970FB6F894DEBF0FBECDBF8091370C90
:10005000888B87E50E947D1E882309F423C120E058
:1000600030E0A9016091D4057091D5058091D60545
:100070009091D7050F94E025811108C00E943B4E56
:100080008DE09DE00E946C3810E01FC18AE50E945F
:10009000CB1E882339F10E94D1242091D6083091BB
:1000A000D7084091D8085091D9080F94AF2C6B0114
:1000B0007C0120E030E040E251ECC701B6010F9432
:1000C000102F87FD0AC020E030E040E251E4C70174
:1000D000B6010F94E025181674F40E943B4E80E0A0
:1000E0009DE0D0CFC0902E0CD0902F0CE090300C23
:1000F000F090310CDECF40E050E060EC7FE788E527
:100100000E94FB242091CE083091CF084091D00866
:100110005091D1080F94AF2C2B013C0140E050E0EE
:1001200060EC7FE789E50E94FB242091D2083091A2
:10013000D3084091D4085091D5080F94AF2C4B01AF
:100140005C016FEF89E40E948D24182F6FEF8AE421
:100150000E948D24082FA3019201C301B2010F94C4
:10016000A22F81116EC0A5019401C501B4010F94A5
:10017000A22F811166C08BA19CA1ADA1BEA18BABAA
:100180009CABADABBEAB2091CC053091CD05409181
:10019000CE055091CF05C301B2010F94AF2C2B01B6
:1001A0003C0120E030E040E05FE36BA97CA98DA931
:1001B0009EA90F9446269B01AC01C301B2010F9486
:1001C000B02C2BA93CA94DA95EA90F94AA2D0F9480
:1001D0001C2E162F4FA058A469A47AA42091D005F4
:1001E0003091D1054091D2055091D305C501B4019C
:1001F0000F94AF2C4B015C0120E030E040E05FE366
:10020000C301B2010F9446269B01AC01C501B401A4
:100210000F94B02CA30192010F94AA2D0F941C2EC1
:10022000062F812F012E000C990B97FD33C00597E7
:100230009CF5802F002E000C990B97FD2FC0059781
:100240007CF5153008F020CF053008F01DCF80E098
:100250000E944A6995E01902F0011124E00FF11D96
:1002600007FDFA95EE0FFF1FEE0FFF1FE257F84F45
:10027000C082D182E282F382602F812F0E9400F837
:1002800088890E944A698889882309F4FDCE0E94E2
:10029000CE30FACE10E0CDCF14E0CBCF00E0D1CFFE
:1002A00004E0CFCF8AE40E947D1E182F811127C061
:1002B00070E060E086E50E94C2249A8389830597F6
:1002C00008F18BED9CE00E946C38812FEE960FB602
:1002D000F894DEBF0FBECDBFDF91CF911F910F917C
:1002E000FF90EF90DF90CF90BF90AF909F908F9056
:1002F0007F906F905F904F903F902F9008950E9455
:10030000286FC2CE60E084E40E94A9248F8740E079
:1003100050E0BA018AE50E94FB246BA77CA78DA759
:100320009EA740E050E86BE376E483E50E94FB245F
:1003300020E030E040E752E40F94AA2D60933D02A4
:1003400070933E0280933F0290934002E0908312AC
:10035000F0908412D7018D909D90AD90BC9020E0DC
:1003600030E0A901C501B4010F94B02C6BAF7CAF94
:100370008DAF9EAF20E030E040E450E40F94E025E4
:1003800087FF06C01BAE1CAEB0E4BDAFE0E4EEAF2D
:1003900020E030E84DE953E4C501B4010F94B02CDE
:1003A000662E7BAB8FAB98AF20E030E844E953E496
:1003B0000F94102F18163CF4612CF0E8FBAB24E9E5
:1003C0002FAB33E438AFD70114968D909D90AD904C
:1003D000BC90179720E030E0A901C501B4010F944B
:1003E000B02CD62EE72EF82E092F20E030E040E08A
:1003F00051E40F94E02587FF04C0D12CE12CF12CAF
:1004000001E420E030E04BE953E4C501B4010F946E
:10041000B02CB62EC72E89AF9AAF20E030E042E96B
:1004200053E40F94102F181634F4B12CC12CB2E9F8
:10043000B9AFE3E4EAAF88E40E947D1E882309F4A3
:1004400016C20E94D1240F941C2E1B0177FF02C0FC
:100450006F5F7F4F759567957195619571096A56C4
:100460007F4F072E000C880B990B0F94E725762EF3
:10047000872E982EA92E2D2D3E2D4F2D502F0F94C7
:10048000102F18161CF4D72C74010A2D2BAD3CAD7F
:100490004DAD5EAD672D782D892D9A2D0F94102FBF
:1004A000181624F07BAC8CAC9DACAEAC872D982D8F
:1004B000A92DBA2D8B8B9C8BAD8BBE8B8D2D9E2D3C
:1004C000AF2DB02F8F8B988FA98FBA8FB101330CBE
:1004D000880B990B0F94E7251B012C01AC019B01A4
:1004E0006D2D7E2D8F2D902F0F94B02CD62EE72EB4
:1004F000F82E092F2B2D3C2D49AD5AAD0F94E02538
:1005000087FF04C0BD2CCE2CF9AE0AAFA201910129
:10051000672D782D892D9A2D0F94B02CD62EE72E8D
:10052000F82E092F262D3BA94FA958AD0F94E02591
:1005300087FF04C06D2CEBAAFFAA08AF862D9BA9EC
:10054000AFA9B8AD8B8F9C8FAD8FBE8F8B2D9C2D9F
:10055000A9ADBAAD8F8F98A3A9A3BAA3BE01695E56
:100560007F4FCE0143960E946F2E882309F4B0C1BD
:10057000BE01615E7F4FCE014B960E946F2EE82E2A
:10058000882309F4A5C12F89388D498D5A8D6F8D27
:1005900078A189A19AA10F94AF2C20E030E040E827
:1005A0005EE30F9446264B015C012B893C894D8903
:1005B0005E896B8D7C8D8D8D9E8D0F94AF2C20E090
:1005C00030E040E85EE30F9446266BA37CA38DA346
:1005D0009EA38FA298A6A9A6BAA689819A81181669
:1005E000190674F489EA9CE00E946C388F85882390
:1005F00021F08FE99CE00E946C388AE00E94333839
:100600000E94B1610E94121D80E00E944A6980E050
:1006100090E0A0E2B1E48FA798ABA9ABBAAB60E0E1
:10062000CE018F960E9404652091D4053091D505A6
:100630004091D6055091D7056BA17CA18DA19EA1BB
:100640000F94E025811130C02091D8053091D90553
:100650004091DA055091DB056FA178A589A59AA58F
:100660000F94E025811120C02091CC053091CD055B
:100670004091CE055091CF056B897C898D899E89EB
:100680000F94E025811110C02091D0053091D10543
:100690004091D2055091D3056F89788D898D9A8DBF
:1006A0000F94E0258823A9F00E94286F88E0FE01BE
:1006B000B396A4EDB5E001900D928A95E1F788E03C
:1006C000FE017396ACECB5E001900D928A95E1F7CE
:1006D000188A60E085E40E94A924882309F4FBC0FD
:1006E000F1E0FBAB1B861C861D861E861A8A9E2C9B
:1006F0004FE6C42E4CE0D42E5DE7A52E5CE0B52E6F
:100700001A8915300CF0F7C06B857C858D859E8528
:100710009B01AC010F94A22F8111EDC0992009F427
:10072000DDC031E03FAB35E0232E91E09926F12E7C
:10073000FF0CFF0CF10EF394898B19896A8912154D
:1007400009F4D5C0062E000C770B880B990B0F947B
:10075000E7252FA138A549A55AA50F9446262F892C
:10076000388D498D5A8D0F94B02C2B013C01612F8F
:10077000110F770B880B990B0F94E7252BA13CA148
:100780004DA15EA10F9446262B893C894D895E8937
:100790000F94B02C6B837C838D839E834F8258860D
:1007A00069867A8689819A81892B79F06F2D8BE809
:1007B0009CE00E94404169E170E089E89CE00E9471
:1007C0006A4186E89CE00E946C381F9299E19F93F1
:1007D0001F92FF92DF92CF92BF92AF921F920E9420
:1007E0002BF929814BA9BE01695F7F4FCE0103968A
:1007F0000E949CF92B013C014B865C866D867E86AF
:100800000FB6F894DEBF0FBECDBFAC019B010F94B5
:10081000A22F811169C089883A8825E0382D3203DA
:1008200080011124030D111D37FC1A95000F111FB3
:10083000000F111F0257184FA30192016BA57CA551
:100840008DA59EA50F94B02CD8016D937D938D93AB
:100850009C931397632D882D0E9400F8188A81E0DD
:100860000E94475AF3948989BFA98B0F65CF4D2DFC
:100870005E2D6F2D702F86E40E94FB241B012C013E
:100880004BAD5CAD6DAD7EAD8CE40E94FB246B8BFB
:100890007C8B8D8B9E8B2F8A388E498E5A8E4B2D5A
:1008A0005C2D69AD7AAD82E40E94FB246B017C0172
:1008B000462D5BA96FA978AD82E50E94FB246B8F62
:1008C0007C8F8D8F9E8FCF8ED8A2E9A2FAA246CEC2
:1008D0008FEB9CE0F8CC22E02BAB04CF8FEF8FABFB
:1008E00022242A9484E021CF88890E944A698A8937
:1008F0008F5F8A8B05CF0E9496E40E94DA65882379
:1009000059F088890E944A6980E090E0A0ECBFE736
:100910008B879C87AD87BE876B857C858D859E8503
:100920009B01AC010F94A22F811159C08F858111B9
:1009300026C082E0F82E02E094E0C92E12E0DC2C02
:10094000D11A21E041E0612F802F0E94AA2221E0EC
:100950004FEF612F8F2D0E94AA222FEF41E06D2DC6
:10096000802F0E94AA222FEF4FEF6D2D8F2D0E9416
:10097000AA22115020F70150F3940F3FF9F60E947C
:10098000B1400E94D81E8F85811124C08EE29CE068
:100990000E94C21D4B015C0186E29CE00E94681F20
:1009A0009B01AC01C501B4010F9446269B01AC012B
:1009B00060912E0C70912F0C8091300C9091310C25
:1009C0000F94AF2C60932E0C70932F0C8093300CEF
:1009D0009093310C8F858111E888E092370C0E944A
:1009E000F91C8091370C81110E94352B0E94C4673D
:1009F0000E94CE306B857C858D859E8511E09B01A4
:100A0000AC010F94A22F811160CC3ECB8F929F92AC
:100A1000AF92BF92CF92DF92EF92FF920F931F930C
:100A2000CF93DF9300D01F92CDB7DEB75C016B018F
:100A30007A01122F0023E1F10E943F4E88E999E0EC
:100A40000E946C3861E0812F0E94603A90901605F8
:100A500083E08093160581E08093250C0E94574027
:100A600082E08093901140E368E879E084E799E0C0
:100A70000E945C4040E069E171E18DE699E00E94EE
:100A80005C4061E088E699E00E943E408AE799E098
:100A90000E9466228091250C882341F060E0812F1E
:100AA0000E94603A81E00E94475AF4CF9092160566
:100AB00020E030E0A901F50160817181828193819C
:100AC0000F94E025882371F080E090E0A0ECB0E482
:100AD00089839A83AB83BC83BE016F5F7F4FC5015F
:100AE0000E948A6820E030E0A901F60160817181EE
:100AF000828193810F94E025882351F18090700CBE
:100B00009090710CA090720CB090730C80E090E00B
:100B1000A0E7B1E48093700C9093710CA093720CD9
:100B2000B093730C80E090E0A0EAB1E489839A83EB
:100B3000AB83BC83BE016F5F7F4FC6010E948A6892
:100B40008092700C9092710CA092720CB092730C07
:100B500020E030E0A901F7016081718182819381F9
:100B60000F94102F181674F480E090E0A0E4B0E425
:100B700089839A83AB83BC83BE016F5F7F4FC701BC
:100B80000E948A688091EB0429E131E1882311F009
:100B900029E439E047E559E061E679E081E00E9427
:100BA0007F400E94574081E00F900F900F900F9070
:100BB000DF91CF911F910F91FF90EF90DF90CF9039
:100BC000BF90AF909F908F900895CF93C82F809142
:100BD000E40B83FD14C080910109811110C0809144
:100BE0005F02909160029C01215031094091EC110B
:100BF0005091ED114217530714F40E94531FCC2358
:100C000029F061E080E0CF910C9408BD809101094A
:100C100091E0892780933C0280913C02882389F0EF
:100C20008091EA119091EB112091EC113091ED112E
:100C3000821B930B97FF03C09195819591090297B1
:100C400044F410923C028091E40B83FF06C0C1E0A3
:100C50001AC080E00E94475ADFCFC0910109C1113C
:100C600012C080915F029091600201972091EC1177
:100C70003091ED112817390754F70E943F4E8BE24F
:100C800099E00E946C388C2FCF910895AF92BF925B
:100C9000CF92DF92EF92FF920F931F93CF93DF9348
:100CA000CDB7DEB764970FB6F894DEBF0FBECDBFE9
:100CB0000E943E4F87FDAFC08AE50E94CB1E88236D
:100CC00009F4BAC040E050E0BA018AE50E94FB2472
:100CD0007B018C0120912E0C30912F0C4091300C17
:100CE0005091310C60E070E088EC93E40F94AF2CED
:100CF0005B016C019701A8010F94102F181614F0D6
:100D00007501860120E030E0A901B701C8010F9408
:100D1000102F181624F4E12CF12C00E010E0B7019C
:100D2000C8010F941C2E072E000C880B990B0F94F2
:100D3000E725698B7A8B8B8B9C8B20E030E0A901B7
:100D40000F94E025882321F0CE0141960E9408737C
:100D500080E090E0A0EAB1E48D879E87AF87B88BF2
:100D600019861A861B861C868CE40E947D1E8823A9
:100D700009F467C00E94D1246B017C0120E030E0BF
:100D8000A901C701B6010F94102F87FF04C0F7FA1D
:100D9000F094F7F8F094CD82DE82EF82F88620910D
:100DA000EC113091ED112430310574F08091EA118D
:100DB0009091EB11821B930B97FF03C09195819546
:100DC000910901E004970CF400E080E00E94E585C1
:100DD000882359F022E0AE01435F5F4FBE016B5F95
:100DE0007F4FCE0109960E94068569897A898B8991
:100DF0009C898B019C01305809831A832B833C8387
:100E000020E030E0A9010F94E025882321F0CE01F5
:100E100001960E94087364960FB6F894DEBF0FBE69
:100E2000CDBFDF91CF911F910F91FF90EF90DF9099
:100E3000CF90BF90AF900895E12CF12C00E211E427
:100E400049CFC090C705D090C805E090C905F09083
:100E5000CA0594CF7F928F929F92AF92BF92CF920A
:100E6000DF92EF92FF920F931F93CF93DF9300D007
:100E700000D01F921F92CDB7DEB76C015B014A0113
:100E8000722E7801009114060E945F1F8091EC1170
:100E90009091ED118E159F051CF4C7010E94531F00
:100EA00080E00E94E585882331F0272DA401B5015B
:100EB000C6010E9406851E141F043CF4C7010E944F
:100EC000531F60E080E00E9408BD81E00E94E5853C
:100ED00080E090E0A0E7B2E489839A83AB83BC838F
:100EE00080E090E0A0E8B0EC8D839E83AF83B8876C
:100EF000BE016F5F7F4FCE0105960E948A6887E032
:100F00000E944C2A811158C080912E0C90912F0C78
:100F1000A091300CB091310C4091F0045091F1044B
:100F20006091F2047091F304C090EC04D090ED0451
:100F3000E090EE04F090EF04C0927207D092730735
:100F4000E0927407F0927507409376075093770705
:100F5000609378077093790780937A0790937B0763
:100F6000A0937C07B0937D0780E090E0A8E4B2E412
:100F700089839A83AB83BC83CE0101960E94A172C0
:100F80008091F4049091F504A091F604B091F704D7
:100F900080937A0790937B07A0937C07B0937D079B
:100FA00080E090E0A0EAB0E489839A83AB83BC83BD
:100FB000CE0101960E94A172C12CD12C80E7E82EAF
:100FC00082E4F82EC982DA82EB82FC8280E090E033
:100FD000A0E8B0E48D839E83AF83B887BE016F5FC6
:100FE0007F4FCE0105960E948A6820E030E0A9017B
:100FF0006091F8047091F9048091FA049091FB04D7
:101000000F94E02587FF0BC0C982DA82EB82FC8255
:10101000BE016F5F7F4F88EF94E00E948A688091E5
:10102000F8049091F904A091FA04B091FB04809324
:10103000320C9093330CA093340CB093350C809306
:101040007E0790937F07A0938007B09381078EE778
:1010500097E00E94C2618091CB0581110E9446F702
:1010600061E087EB99E00E94A73F809122118150B7
:101070008093221140E758E16FEB79E085E00E9410
:101080001BE380912211882339F00E9441AB8091AB
:10109000221181508093221180E00E940DF90E945C
:1010A000C83180912311823011F40E947A380E9455
:1010B00096E428960FB6F894DEBF0FBECDBFDF9141
:1010C000CF911F910F91FF90EF90DF90CF90BF9045
:1010D000AF909F908F907F900895CF92DF92EF9284
:1010E000FF920F931F93CF93DF9300D01F92CDB742
:1010F000DEB77C016B018A0161E08CE399E00E941C
:10110000A73F40E758E163E479E085E00E941BE3F4
:101110009091221181E0890F8093221180913014E7
:1011200082FF06C08B7F809330149E5F90932211C4
:101130000E946C3980E1E6E2FCE0ACEEB4E00190A4
:101140000D928A95E1F70E94B16181E00E940DF94C
:1011500020E030E0A901F7016081718182819381F3
:101160000F94E0258823F1F08091010981110CC0D2
:1011700080915F029091600201972091EA11309175
:10118000EB112817390774F080E090E0A0E7B2E493
:1011900089839A83AB83BC83BE016F5F7F4FC70196
:1011A0000E948A6887E00E944C2A811103C0B60120
:1011B0000E94DE6720E030E0A901F80160817181C2
:1011C000828193810F94E025882341F080E00E9482
:1011D000E585882319F0C8010E94BA68129A64E66E
:1011E00070E080E090E00E943F2681E00F900F9039
:1011F0000F900F90DF91CF911F910F91FF90EF9083
:10120000DF90CF900895CF92DF92EF92FF92CF932D
:10121000DF936B017C01D42FC091160583E080938E
:10122000160581E08093250CC114D104E104F1047A
:1012300031F00E943EFDC60ED71EE81EF91E8091B9
:10124000250C882389F0C114D104E104F10421F4B0
:101250008D2F0E94475AF3CF0E943EFD6C197D09E5
:101260008E099F0997FDF4CF1092250CC0931605A7
:10127000DF91CF91FF90EF90DF90CF9008950F9383
:101280001F93CF93DF93C82F162F0E943F4EC1119B
:1012900094C0CFE8D8E0CE010E946C3861E0812F85
:1012A0000E94603A0E943EFD685370458F4F9F4FE9
:1012B00060931006709311068093120690931306A4
:1012C000109214060091160583E08093160530E015
:1012D00020E049E151E16DE179E082E00E947F4048
:1012E0008DE199E00E94662281E08093250C809137
:1012F000250C882309F464C060E0812F0E94603AC5
:1013000080911406882309F454C00E943F4E83E064
:1013100099E00E946C3830E020E04DEE58E064EF38
:1013200078E082E00E947F4084EF98E00E9466228D
:1013300041E060E070E0CB010E94038930E020E0F2
:1013400050E040E060EE78E085E00E947F4080EE73
:1013500098E00E94CF350E945F1F80E00E94E585E3
:101360000E943F4ECE010E946C380E943EFD6853A1
:1013700070458F4F9F4F60931006709311068093B6
:101380001206909313061092140630E020E049E113
:1013900051E164ED78E082E00E947F4083EC98E0C8
:1013A0000E94662281E08093250C61E0812F0E94DB
:1013B000603A81E00E94475A9ACFC4EAD8E06BCFE6
:1013C00000931605DF91CF911F910F910895CF9251
:1013D000DF92EF92FF920F931F93CF93DF93CDB7DE
:1013E000DEB7A0970FB6F894DEBF0FBECDBF0E9448
:1013F0003E4F87FDCCC085E40E947D1E882309F402
:10140000D5C00E94D1246B017C0120E030E0A9010D
:101410000F94102F87FF04C0F7FAF094F7F8F094B8
:10142000F7FAF094F7F8F094CD8EDE8EEF8EF8A2F6
:101430008CE0E4ECF2E0DE01119601900D928A95C9
:10144000E1F78AE50E94CB1E882351F040E050E08E
:10145000BA018AE50E94FB2469877A878B879C877B
:1014600088E50E94CB1E882351F040E050E0BA018D
:1014700088E50E94FB2469837A838B839C8389E5BA
:101480000E94CB1E882351F040E050E0BA0189E56C
:101490000E94FB246D837E838F83988785E50E945D
:1014A0007D1E882309F489C00E94D1246B017C0130
:1014B00020E030E0A901C701B6010F94102F87FF8B
:1014C00004C0F7FAF094F7F8F094F7FAF094F7F80C
:1014D000F094C98EDA8EEB8EFC8E1D8A1E8A1F8ACE
:1014E000188E8CE40E947D1E882309F46FC00E9430
:1014F000D1246B017C0120E030E0A901C701B601D5
:101500000F94102F87FF04C0F7FAF094F7F8F094C7
:10151000C98ADA8AEB8AFC8A62E070E082E40E947F
:10152000C224F82E80912211811131C021E0AE0138
:10153000475E5F4FBE016F5F7F4FCE014D960E94A9
:101540006D88882321F16F2D81E00E943F8982E51B
:101550000E94CB1E882309F442C00E94BE2440E0B2
:1015600050E060EA71E44D875E876F87788B209149
:101570002211222361F08C012F2DAE01435F5F4FBA
:10158000BE016F5E7F4FCE0145960E942A87A096CE
:101590000FB6F894DEBF0FBECDBFDF91CF911F9184
:1015A0000F91FF90EF90DF90CF900895C12CD12C38
:1015B00080E8E82E80E4F82E33CFC090C305D090A9
:1015C000C405E090C505F090C60572CFC090C70570
:1015D000D090C805E090C905F090CA058CCF90E086
:1015E00080E0BDCFCF92DF92EF92FF920F931F93D7
:1015F000CF93DF93CDB7DEB76C970FB6F894DEBF0D
:101600000FBECDBF8CE40E947D1E882309F4B0C0BC
:101610000E94D1246B017C0120E030E0A9010F94ED
:10162000102F87FF04C0F7FAF094F7F8F094F7FA58
:10163000F094F7F8F094C98EDA8EEB8EFC8E8CE085
:10164000E4ECF2E0DE01119601900D928A95E1F74B
:1016500088E50E94CB1E8823A1F040E050E0BA014B
:1016600088E50E94FB242091CE083091CF0840915C
:10167000D0085091D1080F94AF2C69837A838B8363
:101680009C8389E50E94CB1E8823A1F040E050E0B6
:10169000BA0189E50E94FB242091CE083091CF0841
:1016A0004091D0085091D1080F94AF2C6D837E8368
:1016B0008F8398878AE50E94CB1E882351F040E0F3
:1016C00050E0BA018AE50E94FB2469877A878B87FC
:1016D0009C871D861E861F86188A80912211811183
:1016E00038C020E0AE01435F5F4FBE016F5F7F4FA8
:1016F000CE0149960E946D88882359F18091CB05CF
:1017000081110E9446F760E080E00E943F89898D48
:101710009A8DAB8DBC8DB0588D8B9E8BAF8BB88F57
:10172000198A1A8A1B8A1C8A1D861E861F86188A99
:1017300080912211882369F010E000E020E0AE01E2
:101740004B5E5F4FBE016F5E7F4FCE010D960E94D4
:101750002A876C960FB6F894DEBF0FBECDBFDF911F
:10176000CF911F910F91FF90EF90DF90CF90089550
:10177000C12CD12C80E8E82E80E4F82E58CF2F928F
:101780003F924F925F926F927F928F929F92AF9211
:10179000BF92CF92DF92EF92FF920F931F93CF935E
:1017A000DF93CDB7DEB7E5970FB6F894DEBF0FBE77
:1017B000CDBF8DAB209116052CAB21E020931605F3
:1017C000809134058D3409F405C6843511F40C94E8
:1017D00012A1873409F091C18091320590913305AF
:1017E0008B31910509F4DDC108F079C18430910590
:1017F00008F030C12091E7068230910508F48EC1CF
:10180000213009F091C111E0029709F010E00E9427
:10181000122519821A821B821C821D821E821F823F
:10182000188682E50E94CB1E882309F490C10E948D
:10183000D1246B017C0120E030E0A9010F94E02568
:10184000882309F4EAC04090260C5090270C609041
:10185000280C7090290C80912A0C90912B0CA0914F
:101860002C0CB0912D0C8CA79DA7AEA7BFA7809084
:10187000720790907307A0907407B09075078091DD
:10188000760790917707A0917807B091790788AB98
:1018900099ABAAABBBABA5019401C301B2010F94F4
:1018A000E02581110DC028A939A94AA95BA96CA519
:1018B0007DA58EA59FA50F94E025882309F4ADC0D2
:1018C000A3019201C501B4010F94AF2C20E030E0D8
:1018D00040E05FE30F94462668A779A78AA79BA7F5
:1018E0002CA53DA54EA55FA568A979A98AA99BA9A4
:1018F0000F94AF2C20E030E040E05FE30F944626E9
:101900002B013C0120E030E0A901C701B6010F9492
:10191000E025881F8827881F181709F40FC180E069
:1019200090E0A0E8BFEB8CA79DA7AEA7BFA728A516
:1019300039A54AA55BA5CA01B9010F9446264B01FA
:101940005C01A3019201C301B2010F9446269B01E1
:10195000AC01C501B4010F94B02C0F945E2F4B0164
:101960005C01AC019B01C701B6010F94AF2C68ABC1
:1019700079AB8AAB9BABA5019401C701B6010F946B
:10198000B02C9B01AC0168A979A98AA99BA90F94E5
:1019900046266B017C0120E030E0A9010F94102F56
:1019A00087FDD1C0C701B6010F945E2F6B017C018A
:1019B000C301B2019058A50194010F94AA2D2CA542
:1019C0003DA54EA55FA50F944626A70196010F944D
:1019D000462628A539A54AA55BA50F94B02C698396
:1019E0007A838B839C83A501940168A579A58AA538
:1019F0009BA50F94AA2D2CA53DA54EA55FA50F94E0
:101A00004626A70196010F944626A30192010F9442
:101A1000B02C6D837E838F83988720E030E0A9010E
:101A200069817A818B819C810F94E0258111A3C00B
:101A300020E030E0A9016D817E818F8198850F942F
:101A4000E025811198C00E943B4E8BEB9FE00E94E5
:101A50006C386AC08531910509F466C08A319105F8
:101A600009F49CC0049709F048C080E50E94CB1E91
:101A7000C12CD12C7601882321F00E944B246B01CC
:101A80007C0183E50E94CB1E882361F00E94D12453
:101A900020E030E04AE754E40F9446260F94232ECA
:101AA0006B017C010E94B16180912411811105C0FC
:101AB00060E081ED9FE00E94DA3F0E943EFDC60E8D
:101AC000D71EE81EF91E0E943EFD6C197D098E0985
:101AD0009F0997FF29C080E00E94475AF4CF8A32BD
:101AE000910509F4ECC260F48D31910509F415C239
:101AF00008F470C04E9709F468C20E945FF914C0E0
:101B00008B35910509F4BEC38C35910509F4BEC32C
:101B10008A35910591F71092F20706C0213021F421
:101B20000E9412250E94EE6F3DA9311102C00F9450
:101B3000C5148CA9809316050C94739980E090E0ED
:101B4000A0E8BFE3F0CEC12CD12C760131CF89E4DF
:101B50000E94CB1E882331F00E94D12469837A83AE
:101B60008B839C838AE40E94CB1E882309F455CF83
:101B70000E94D1244ECF412FBE016F5F7F4F82E77D
:101B800097E00F9418150E943EFD609375117093B5
:101B900076118093771190937811C6CF0E94DD77EC
:101BA000C3CF87E00E944F4E8111BECF8CE0E0EDA5
:101BB000F2E0DE01119601900D928A95E1F770E056
:101BC00060E080E50E946B24BE016F5F7F4F0E9442
:101BD000DE67AACF87E00E944C2A811106C060E030
:101BE0008FE40E94A92481119FCF0E94B1611092BD
:101BF00046026091370C8CE40E94A924E82E80E014
:101C00000E944A690E943EFD60937511709376119F
